:20000000003B012089230100A1C10310A1C10310A1C10310A1C10310A1C10310A1C1031019
:1C002000A1C10310A1C10310A1C10310A1C10310A1C10310A1C1031079C10310B9
:200040009C482DE9F04F90F86B14ADF14C0D1091002190F8FC020D91974920B90846007804
:20006000002840F0A380109F81220846022F027002D19249FF2008700D98914CBF4A109E44
:20008000BF490B90DFF8FC8227781070012EA08109882069A77012D0007A801E85B2A942AC
:2000A000C0F2B283216A04F118000422083157F099FB0426A17E607EE27EA68129E0467A10
:2000C000027A06F0070302EB032295B2720938BF2D1F06D3427A057A02F0070205EB022567
:2000E000AD1E36F07F06ADB240F08E83A942C0F28B830A3029460FF001FF216A04F11800FF
:200100000522083157F06EFB0526A681227FE17EA07E04F11A0300EB01200C93C1F3011BD2
:2001200060816449227191F8FC12ED1EADB2002908BFBBF1020F00F06783BBF1020F00F366
:200140006383DFF8C09261B110F0070F00F05C8349460978862904D100F00701022940F0B2
:200160005383011301F00201022946DA637800F00700022833D1D8F804A0181C2FD1216A23
:2001800009A801228919083157F02CFB771CB8B2A081D047824699F800604648D8F808509E
:2001A0004768CDF82880862E14D10FB916F019F99DF9240016F065F978770B989DF92460E0
:2001C000B8775046FE77A847608900F0100010F085FF01E05046A84715F0E4FB18E399F8B3
:2001E00000000D9E862808BF0126CDF828803EB10D9812F011FEA77801E0CDF8288063785E
:200200008FB183B9012F00F0FC826089022F03D110F0070F40F0F582032F05D100F0070119
:20022000032901D0EDE26089010909D310F4405F00F0E7821F4991F82074002F00F0E18220
:20024000011301F00201022902DA810A80F0D9821099012905D0BE4ABD49921C89780C9236
:2002600001E0BB49C978C1F381098E11B9F1010F00F0C782012E00F0C482BF49BBF1020F5E
:2002800009D08A5D11F809108918CFB2F6B1C1091CD3BF1E0BE0721849441279097989186D
:2002A000CFB2C1090ED259EA06030FD0BF1CFFB20CE0C0462008002049360020AD1F002097
:2002C0006434002059EA060308BF0227C0F300217A1A61719542C0F29482ED1B00090D44EF
:2002E000A9B2218124BF25200D900D984018743080B215F00BF965786061002800F08182A7
:20030000DDF82C807422414610F044FB84F80380B4F80A804FF0FF0A1DB9184908F0200034
:2003200008700B9D154B60790E951D780F90002D39D0002837D108F00708B8F1030F06D08F
:20034000B8F1010F15D1BA4890F86A0488B11098012806D09F4805781DB115F059FDFE2873
:2003600005D014F025FE10B914F048FC08B10420E0701098012810D106E0C0464B36002004
:20038000101F00208C1A0020A94890F8FC0210B1BBF1020F01DA14F047FF6079B4F80A801F
:2003A0000F90E0780E90636903F174005860986525891D812089A3F85C005FEA181016D379
:2003C000109D0F98012DC0F1030082B2A3F85C2019BF5F49491CB3F85C200C99986D57F09F
:2003E00001FA6369B3F85C10986D401898651098A3F80C80012807D055490C98007849787B
:2004000006E0C0464D36002051480C99C07809780E9DC0F3011001F07801014345EA010009
:20042000187483F80EA00F9920790D9001B10B9883F8306083F83A9083F84900A089002F68
:20044000A0EB010085B2A58100F0D1817848BB46216A90F86B94E7805A464919CDF844909C
:200460006846083157F0BEF97F19BDB2A581B9F1010F07BF3648C0780C98007861690F7CC3
:200480004E46012E07F0400AC0F30110109007BF2F48C0780C9800786E46C0F38107002F45
:2004A00045D010980B9B022802D1BAF1000F0BD19DF801209DF8000000EB0220A1F8440011
:2004C0000DF10206A1F84200DFF82893B1F84400B9F86A20824203D04FF6FF72824223D17C
:2004E000032F12D07278307800EB022080B24886B9F86820B61C0121824204D04FF6FF72CE
:20050000824218BF191C08460DE0CD4800683146323057F02BFCCA48006809F15F013230D6
:2005200057F00CFC08360346002B00F065811198012807BF0648C0780C980078831123D023
:2005400010996069022905D0017CC90905D30BE07C3400205AEA070706D172783178B61CB9
:2005600001EB0221A0F84210032B07D07178327802EB0122028507E030890100B048006852
:200580003146283057F0F2FB08F00708B8F1030F07D0B8F1010F39D1254890F86A04002871
:2005A00034D023486669DDF82C80876FEFB17B7E33F07F0315D096F8300002280CD0032874
:2005C0000FD107F1700006F1280157F0B7FB40B11CE0C046181F0020B7F87000318D8842C9
:2005E00014D057F80C7C002FE1D1B8F1000F0DD1944F4046E0700C9BF878C0F301111878A4
:20060000CDF8388000F0780008433074119801285BD1074890F8FC0210B11098022854DA72
:2006200089480778002F50D00F9800284DD101E0200800200E98854E0746DFF8F891DFF808
:20064000F8810D9D96F86B04012813D04A4628460223911C0B9D0B70D57017B143F0100328
:200660000B7003228870404680F84720816414F0DBFD27E0E9200DF1260112F081FE9DF871
:200680002660052336B94846072200F10C010A70082204E0484600F10C010B70182242738A
:2006A000881C022202700B9ACA701FB1027842F0100202700D71C8F8DC10A8F8D030032133
:2006C0000FF01CFCA589B4F806B0606981890909C0F08D80806D5A46694657F083F8616909
:2006E000886D58448865276AB1F85C0001225844A1F85C000DF125007919083157F072F893
:200700006E1CB5B2A58161699DF82500896D087061699DF825709DF82530886D401C8865B4
:20072000B1F85C00401CA1F85C0007F0070081F82400C3F3C10781F8257091F82460208986
:200740008046002E58D03D497F183A78121D1646E280864250DC216A05A84919083157F0B3
:2007600041F838789DF817209DF814109DF8163040193D78001D01EB026180B201EB034154
:20078000A0819DF81530606901EB032181616DB12B4800686D1E06A92A461C3057F022F853
:2007A000397860696944C97D80F82610806D324605A957F017F86169886D80198865B1F8C7
:2007C0005C004FF0FF3706EB0642C8EA0040A0FA42F01FFAA0F217FA80F0A1F85C2082B2DC
:2007E0002281B1F85C000A818018A1F85C0000F02FF80DE02819002015F056FD11F092F9F0
:2008000006E015F09BFB03E015F098FBCDF82880DDF82880D8F804008047226A0B991368AC
:20082000197111682162D8F80810884713B0BDE8F08FC046B41C0020C8130020687A0100C0
:20084000783400207C3400204B360020200800202DE9F04FC34C60692689216AA589806D91
:20086000ADF14C0D32464919083156F0BBFF6169886D80198865C5480778216AAD19ADB2ED
:2008800001220DF13E004919083156F0ABFFDFF808836D1CADB2022F09D1216A40460122E5
:2008A000401C4919083156F09DFF6E1CB5B2216A04A804224919083156F094FF2E1DB0B2F0
:2008C0009DF813109DF810509DF81220A08105EB016063699DF8111000EB024000EB012077
:2008E000049015F0DBFAD863049814F0C1FFA3F84000EA2015F08DF8A548A64E0221022F4B
:2009000001700BD1A548801C007838B14146087810B94878FF2801D00420E0706569E0787E
:20092000297C084328749DF93E0015F0AAFD85F8460005F17407AF6529899DF93E006B680A
:2009400085F84800B5F85C004FF0000A401AC01801466860A88985F847A0820A18D2020929
:2009600055D310F0070F07D000F00700032812BF081C6868401C46E06968C87800F00702EF
:20098000401000F0380000EB42004018001D3AE00DB915F026FDA889800A2ED369684878E8
:2009A000C7112AD12F89696650464B780A7803F07F035B0003EBE2137E2B0DD07F2B09D046
:2009C00002F07F0280188918801C891C80B28742EBDC08E0514600E00121801C85F860105E
:2009E00080B2874201DA504605E06968091869602989091A2981A5F86800686E10B1B5F823
:200A00006800B0B168686861A889000918D295F86000002800F01081284611F0E1FE65699E
:200A2000E86C002800F00881B5F85000002840F0038104F1140015F01EFD504660611FE267
:200A40005046059095F82470069005A906AA07AB0790284605F0EEFD002840F0E280059A66
:200A6000D5F8148068682B89A8EB0001581A1FFA80F90AB915F0B5FCB5F85C000090CDF822
:200A80000480CDF808900698001D03900598A969AB6D3A4615300BF0EDF8002840F0C18022
:200AA000B04895F860202B89C15D581A288112B1284611F095FEA88900F00709B9F1030F92
:200AC00002D168680078E87395F80FB0732009A914F07EF9832010A908F01AF9B8464F469A
:200AE0005046514611900BE0C278012A04D1B8F1000F08BFDC2029D0001D491C0990C9B2F9
:200B00009DF84000884240F38B8009988378032F07D00278BA420DD096F8FC220AB1022F68
:200B200008D0032FE8D10278032AE5D1024652785A45E1D14FEAA802B2EBA30F05DA03F02E
:200B4000030308F003029342CEDD5046DDF814C08346604695F80FE090F8148039465046B7
:200B600004E0C04664340020401CC0B2804555DDDCF810704300032907EB030210D1FB5C1C
:200B8000032BF1D152787245EED112E08B0C00204936002020080020AC1F0020161F002055
:200BA00012788A4205D096F8FC22002ADCD00229DAD10698077D002F08BFBBF1DC0F2FD004
:200BC000A869B0F1FF3F27D0712008A914F000F9089B5046AA6905998B4207D10699074674
:200BE00001EB8701C9681197914213D8401C2C330228F0DB06981199521CB2F1FF3F00EBB8
:200C00008100C26002D107980121817085F801A0504607E0DB2005E0DB2002E0DC2000E078
:200C2000DD20687065696870A8696F7868651FB1F22014F0EEFE656996F8FC02002800F030
:200C4000A180A989DFF8448201F00702022A5ED16778002F5BD16F78002F58D161698DF887
:200C60003FA00DF13600283157F080F861690BA80A22283156F0B6FD414601F110026769F3
:200C8000D6F820331088401C1080786E04210DF13F029847454604F1140928B9706818B167
:200CA0009DF83F1080F86810676997F83000022811D1D9F8000006F57A71884602222830C4
:200CC000203114F0F9FA30B908F116010DF1360057F04CF867696E480078862807D1688A9E
:200CE000401C6882B88900F0100010F0F7F996F8FC0220B1D6F8441309B16069884748461B
:200D000015F0B9FB5046606114F04CFEBAE0614A177877B3C1F3013102292AD16878002863
:200D200040F0AE809DF83E105F484346E7780170988A05F128021C35002F00F101009882A4
:200D40000CBF51460821544B5046186000910195B6F80E34117A0D2005F060FB20B914F05F
:200D600063FA03E06C7A010014F0BAFD4B486569007838B1D6F8441321B1284688476569CD
:200D800096F8FC02AF890A9507F0070760B1A87BFF2871D0032F05D128464068007804288D
:200DA00002DD69E0012F67D1381C3AD0401E4ED0801E61D1A889C0F30130022803D1686816
:200DC000007807282BD02889002855D0284641684A1C42600F78AC46C7739CF824506DB973
:200DE000002F49D00A2F47DA2D490089C95D814209D0082F40D1082805D03DE0C07B0028C3
:200E00003AD00A2838DA60460189491E0181C17B0B3101700A99C87B401CC87319E03220BA
:200E200016E096F8F5030F280BD015F055F840B90A988189091301F00201022901DA31697D
:200E4000884796F82B040A9D2874152000E0162028700A9906F17C0056F00EFC114D68684C
:200E6000804796F88410491C86F88410A9688847202015F04FF945E70AA812F0B3FB41E7EF
:200E800010F050FE13B0BDE8F08FC0460C1E00204D3600204B360020BC1C00201C0B00204A
:200EA000737A01008C1A0020161F0020AE482DE9F04F14300168ADF11C0D31B1A548007823
:200EC000012814BF002001208847DFF894B2A24DA24FA44C9BF86B042979012863D0E868C9
:200EE00001290CD158B1002011F026FC386A4168E8688847D848012101700020E8600221F7
:200F00003E6A297148B9002E00F09180316A05F1140088474FF4FA70E88412F06DFDF86905
:200F20008069006860639BF92A040FF0A9FD4FF6FF720121824218BF60860026668404F1D8
:200F40002D026662107861F30300107015F0A0F930B9D448D44A102114230170501C0370C2
:200F6000E86858B9386A0668F96AD94804F1200205F11403B0472F46044612E0304611F039
:200F8000DBFB8DF80C6033468DF80D60386A0293066D08228DE80C00E8682034214602AA13
:200FA000B047FC60A7E1E86802290CD158B1002011F0C2FB386A4168E8688847A64801219D
:200FC00001700020E8600121297100260496B0468DF8148000288DF8158035D1C748C84945
:200FE0000068814217D0C749814214D0C649814211D0C64981420ED0C54981420BD0C5490B
:20100000814208D0C449814205D0C449814202D0C34981420BD111F067FE012812BF85F866
:20102000018001206870386A00F1200608B915F0D8F9316805F1140088474FF4FA70E8845B
:20104000B84EAE620623EB6212F0D6FCB649786A4DC88A468AE84D009BF86964F86981F871
:20106000008026B980690068C4F8FC0005E0C0690068C4F8FC0014F025FC632006A912F081
:201080007FF99BF83B0413F023FA04F1EE0201461078012363F3020010709BF83B94B9F12A
:2010A000800F05DDB9F1840F1FDBB9F1860F10DB0F2004F1F70284F8F000107868F30300EF
:2010C0001070887B052814BF2420292084F8F40019E00F2084F8F000292684F8F46004F1E8
:2010E000F700027868F303020CE00F2084F8F000212684F8F46004F1F700027822F00F02F8
:2011000042F00802027004F1F5021078B9F1800F68F38710107002DDB9F1840F26DB887AE3
:2011200080B904F1F5039DF818001A78401E60F3050204F1F6001A70027822F03F0242F01E
:20114000180222E004F1F5029DF81830107863F3050012E08B0C00204C1D00202819002034
:2011600020080020C81300204419002004F1F502107820F03F0040F00200107004F1F6004F
:20118000027822F03F0242F020020270887B8A890A2604F1EE03401D504390FBF6F21E8887
:2011A00062F3CD061E808889192204F1F006800390FBF2F3326863F31C2204F1F80332608F
:2011C000FA69187892F8246066F30200187092F8240004F1F806C310307863F3C300307056
:2011E0004AF63F33A4F8FA3008894B680E68401E434306EB53004FF47A73B0FBF3F0166A57
:20120000A4F800013078A4F8E28004F1ED0284F804014FF00008C4F8E4801078012666F3B7
:201220000300107015F034F8E8B988891D4EB9F1020FB3FBF0F0C1B21B483170B3FBF1F28C
:2012400042700BD0B9F1840F0DDBB9F1860F0ADA05225C2104E0C046CF1F00200222A82130
:20126000324B1A700170E8683E6A98B3404611F063FAA8789BF83B14884217D1E9789BF827
:2012800069243E6AE868914212D1022142468DE80600366DE034434604AA2146B047FC6045
:2012A00023E0C046301E0020141F00203E6AE8687168884701211E483B6A01701E681D483B
:2012C00004F1E002514605F11403B0470AE0C046B030002004F1E0021648346805F11403CE
:2012E0005146A047E860786AB8629BF83B04A8709BF86974EF7007B0BDE8F08F94120050A2
:2013000000F0022000F0012000F00020008002200080012000F0820000F082200080822031
:201320000080002005520100183600200C1E0020CF1F0020B03000202DE9F04FADF18C0D63
:201340001C9104461D920DF15700D1491E93082256F048FA2046694612F0CEFF1F9000285A
:2013600004BF0020229000F0098202200027A41CDFF824B32090C74E2297204602A911F016
:2013800000FB5FEA000900F0F68122990DF13900162256F043FA9DF809707F1E00F0888049
:2013A0007F1E40F0E081B9F10B0FC0F2E781A41C04A80422214656F015FA241D05A80222C1
:2013C000214656F00FFA42F20B000DF1160111F065FCBDF81600BDF81410884200F3CE81F1
:2013E000A41C14F8010B0DF1390214F8017B8DF8390014F8015B8DF83A7014F8011B8DF852
:201400003B50204606F08AFDC34909780028044400F0B4811F9D012905F1020500F09C814C
:201420004FF400500DF14F0111F038FC0DF14F000DF15701082213F03FFF40B11C990DF1E4
:201440004F00082213F038FF002840F0858142F2010004A906F038FE42F20B0005A906F08A
:2014600033FE42F205000DF1390106F02DFE0DF13A0142F2060006F027FE0DF13B0142F2AD
:20148000070006F021FE0FA942F2090006F01CFE9DF83C0028B1022840F05E8142F2030011
:2014A00001E042F20D000DF13D0106F00DFE53E1B9F1050FC0F26281A41C14F8010B0DF170
:2014C000390214F8017B8DF8390014F8015B8DF83A7014F8011B8DF83B50204606F01EFD45
:2014E0000028044400F04A811C9806A906F0BAFE9DF83600002840F011819DF83C00002802
:201500007DD1B6F84E70002F00F00481B6F85200874207D0308B718B884201D109F0C6FFBC
:20152000B06D21E0B76D4FF400500DF15F0111F0B5FB13F09BFF4FF6FF78229D2190AA460E
:20154000B6F84E00A84243DCB06D4FF6FF7141450AD04FEA480707EB88073818808812F0F1
:201560000BF9B06D3F1823D1B6F84E300746002B08BF229D19D05846229D40681946D8466A
:20158000BF1FBF1DFA782AB1491E05F10105F8D1BF1D0AE08047B6F85210491CA6F8521016
:2015A000D8F808108847B6F84E30AB4200F099801C980AF0A9FDB8800120F870FD788DF843
:2015C0003650B888ADF83700229B8DF82330A5E0B88811F04FFA014608220DF15F0013F0F4
:2015E0006BFE40B138880104219814F01CFF82453CBF8246A8466D1CBF1DADB2A0E7B6F883
:201600004C70002F00F08680B6F85000874207D0308B718B884201D109F048FF706D20E0DB
:20162000776D4FF400500DF1670111F037FB13F01DFF4FF6FF78229D2190AA46B6F84C0065
:20164000A84250DC706D4FF6FF71414509D008EB48173818B0F81F0012F08EF8706D3F185E
:2016600029D1B6F84C300746002B08BF229D20D0DBF80400229D1946D846213F2137BA7F54
:2016800062B1491E05F10105F8D1213711E0C046C0810100401100208C1A00208047B6F8CE
:2016A0005010491CA6F85010D8F808108847B6F84C30AB4215D022993846212256F0AEF84C
:2016C0001C980AF021FDA7F81F000123FF2039462122BB770546787206A8FD7256F082F837
:2016E0001CE0612060E0B7F81F0011F0C3F9014608220DF1670013F0DFFD38B1796821986A
:2017000014F091FE82453CBF8246A8466D1C2137ADB293E7642047E0220800209DF8360044
:201720000DF13901162240F004008DF8360008A856F058F81F9D9DF83C00AD1C48B19DF820
:201740004E700DF13D00394610F0C6FD3F1A8DF8357006A80FF06AFD209809EB0007BF1C29
:20176000B8B2209003E01F9D4C44A41CAD1C209885423FF702AE2098022803DC229A67202E
:2017800011460DE01F9F01460220C0EA014207EB0741A1FA42F21FFAA2F110FA82F2229804
:2017A0001D9B19801E990A8023B0BDE8F08F70472DE9F04F0320ADF1540D13F023F8CE4C3A
:2017C0000025022004F11C0141F80C5F401E8D60FAD104F14000A946062701467F1E21F8A8
:2017E0000C9BFBD10821C64FC44BC64A01803F1D04F11C082E468360964627F00301531A68
:2018000023628C46A1610846E161824200F2CC81B80823F00303AEEB8000E827801001EB5F
:20182000800040F8046CEC3BCCF800704846C1F8E830E831216154F021FD6061BC49D8F833
:201840000000DFF8F4A220610A680AF10C073A6049687960B7493846082213F02DFDB84623
:2018600028B9D04801683A46116040685060D048D04FC0F8B470D04BC0F8B830C0F8BC502B
:20188000C0F8CC50D04AC0F8D050D04FC0F8C020CF4BD0F8B410C0F8C470C0F8C83009B1CF
:2018A0004846884754F028FDCA4ECB460C224946CDF838B006F128000FF06CF8C64F41F205
:2018C000707308223363708DF762616AADF82020102309930227ADF8227040F019007085F2
:2018E00008A8884700280CBF0A9F4F4608200123ADF82C00616AADF82E300BA88847544631
:201900009DF830000D992070616077B1D021397087F80190B87087F8039087F8049039466D
:20192000BD600220FD6012F045F9AC491820012254F05AFCE220414614F094FB182054F049
:2019400037FF60706068B046C8F808000BF0FAFEAC4F08F18400A060D8F80850A04C4946ED
:201960006762F520A56014F089F814F09FF89D4D002807BF0F2205F10C010D2205F118011A
:2019800005F124006A700E22AA700DF0B9FDA860687814F051FA00280CBF08264E46A8784A
:2019A00014F04AFA08B946F010068F49A86814F045FC8E49C82205F1300056F071F98C483A
:2019C000102E686010D1606A70B1C26862B1FF208DF810004FF6FF77ADF8127004AEADF80B
:2019E000147096E803009047824F07F1140007F108010DF085FD7860484656F0C7F84E46AF
:201A0000BD1E824605F8029F02206870304656F0C3F8014678685246C9B212F025F9761C28
:201A2000022EEFDB744907F120004FF4FA7256F037F9724D05F10C00291D0DF061FD2860C8
:201A4000606A002845D00769DFF8B4A16FB10094514612A80A688988026012AE818096E8BA
:201A6000030001234A46B847606A002831D0C26852B1514612A80B688988036012AF818096
:201A800097E803009047606A18B307690FB306208DF80800ADF80A0010AEADF80C9002AD16
:201AA000009695E803004A460223ADF84020B847666ABDF840007769A08057B1BDF8400095
:201AC00002AE401CADF8400096E80300022210ABB8473AA014F064FAE820012113F0CEFF80
:201AE000E720092113F0CAFF606A0626002835D00769002F32D007E08C1A002045690500C5
:201B00004E360020003B01208DF818600425ADF81A500EA8ADF81C9006AB009093E80300CA
:201B20004A462B46B84748B90E9E1936B34615E0C87F050038890100D81E0020606A8DF848
:201B4000186006AFADF81A504469ADF81C9097E80300CDF83CB02A460FABA047CDF838B05A
:201B600058460EF023FDE0200C2113F087FF4F20032113F083FF5720052113F07FFF4E204F
:201B8000042113F07BFF5920032113F077FF13F029FE08F10200012156F054F800F0F8FBD1
:201BA000FCE7C046F012005040F8046B2DE6C04610010020793801002D3C010054492053CD
:201BC000656E736F7200C04675F100005940010055CF00005C18002020BF02003D480000BA
:201BE00058170020141B0020914001003D5B0100A55C0100001C00202D7A0500901E0020E4
:201C000078890100C40100202DE9F04FD04CADF13C0DDFF840A3DFF84093DFF840B3D04F38
:201C20000C90666894F86B04012800F08480002E00F08280012051464D4608702978012974
:201C400002D001F037FC6668358994F82B0476680BF0E4FB01F0A6FDC44CDFF8148304F188
:201C6000380908F1040089F80F500068A66400256587804782465A4607F120000C9B066867
:201C8000106833F0010335D104F1A00104F138024D8004F1AD03C4F8A4201A7822F00F0233
:201CA00042F002021A7004F1AC031A7865F303021A7004F1B7031A7822F00F0242F00402AB
:201CC0001A70658749F64043C4F8BC3004F144031A7865F303021A708DF814500495B94BE9
:201CE0008DF8155008248DE83000346D04AAA0474C460FE08DF8145038348DF815502A46C3
:201D00006580B04B049208218DE80600356D04AA2146A847AC4946460880B16800280A4669
:201D200007D4AA4991F90000FC60401C087050463EE150463FE10EB914F053FB4FF0000850
:201D400030897168A24BCDF82480C500097818781035890906D340F6485191FBF0F16D1854
:201D600005F5AF75337D68438500352B0CBF46464FF4FA560DF12E01E82011F001FB9DF854
:201D80002E00032808BF44F620666068007DAD19352803D1D4F860038047454302205E46E3
:201DA0008DF828003068089508A90CF0F1F94E46012051460870317887F80080012901D043
:201DC00001F078FB60680589466813F0CFFB3088BB46000942D394F8FC0200283ED061686E
:201DE0004B6A4F6E986AB0F1FF3F26D02FB3421C9A628862030E07F80139606890F82A00B0
:201E000007F80109606890F8290007F80109606890F8280038706268106A00950190801B12
:201E2000281A80B20290916A506A92F88C203346153008F07FFF074600E0DB27D4F840132F
:201E400067B119B9E4200DF011FD04E0624880F80080E4208847002F40F0B18029463046BB
:201E60000EF04CF864200BA911F08AFA5B4894F8FC72007837B994F82B040BF0CFFA0128B6
:201E800005D099E00BF0CAFA012840F09580544BA81C87B20DF12D01E9201F8011F070FAEC
:201EA0009DF82D00012805D13D46C5F3022040F0180005E02D1DADB2C5F3022040F008001C
:201EC00006F8010D06F8015D284D9DF82C00A5F8C2800028C5F8DC600CBF42484248CDF8C0
:201EE000188002238DF81D8005F168068DF81C3005F1C00AA6F8028005F17501C5F81801AC
:201F00001B4FCAF81800087820F00F0040F003000870786880470D90DFF8A8900C98012813
:201F200028D0042826D0E8B105280DD0032808D194F83B0412F0CCFAC07B022818BF564675
:201F40001AE005F1C00617E0DFF8A09014E0C04620080020EF1E0020CD1F0020581D0020BD
:201F60002819002005F1840606E0C046C81300208C1A002005F16806DBF82000154B046DAB
:201F8000414602208DE80300D86806AA31464B46A047BE680C490028324608800AD40B496C
:201FA00091F90000C035401C08700D98CBF80C50904704E00D9890471A200DF057FC0FB08A
:201FC000BDE8F08F2D590000B41C0020F61E0020301E00204C1D00204D360020171F002043
:201FE000981400204E9055550E7A5555A5C90000B7482DE9F04F0C46ADF1140DDFF8E0B21F
:20200000B54902920078B54A039301286ED0B14801230024029F0B7002264FF0E045894602
:20202000039B006814703E401D4008BF002E35D13A464FF4803114EA030701EA020108BF0F
:2020400000291CD113464FF400311940039B224612EA030708BF00290DD1039F029B4FF4E8
:2020600080013A4001EA030108BF00290AD004710FF058FD06E0047111F0D2F802E0047166
:20208000FDF7DEFF0299039B2020274608401F4008BF002814D013F023FC11E0594691F9D3
:2020A0000020B04B521E0A7093F90020521E1A7091F900700FB9AC490C8004710FF032FD8F
:2020C000A84991F9000040B1002D08BF002E09D091F90000002805DC39E1A4480470204626
:2020E00001F0E8F9A046CDF8009035E101204FF0000817460870029EDFF87492DFF878A212
:202100000091454687F80080202705EA06001F4008BF002878D1424630464FF0E04719460E
:2021200010400F4008BF002843D133464FF48601039EB9F80A01DFF844C2CDF8049012EA2B
:20214000060701EA030108BF002919D1894912EA060701EA030108BF002971D0374651469A
:20216000029E0C8101F138034881002F83E8C00004BF331CB3F1806F62D1022860D111E0BE
:2021800037465146029E0C8101F138034881002F83E8C00004BF331CB3F5803F50D1B0F56F
:2021A000505F4DD1086A6746436938682146984744E05E4696F90000401E30705646B6F901
:2021C0000800844217D1728906F1380003C8002904BFB0F5803FB2F5505F08D0002904BFEA
:2021E000B0F1806F022A02D00FF09CFC03E011F017F813F003FD5B4A92F90000401E1070B6
:202200006FF00101318117E0604E96F8FC7251466FF0010001F1080210806FB1584800784F
:20222000832802D0574A812010705646316919B1404688472146E5E7CDF80490B9F80A01C2
:20224000039B029A474F5E4641464FF0020B11EA03050BEA020208BF002A61D043F20142A1
:20226000554682423ED0D21C82423BD0B5F9083096F900209C42A2F10102327004D043F67C
:202280000401814239D136E005F1380090E800064FF4820311EA0A0403EA090008BF0028F4
:2022A00012D105F1380090E800064FF4003411EA0A0104EA090008BF002802D10FF032FC2C
:2022C0001BE010F0ADFF18E0FDF7BAFE15E0C0468B0C002074340020CD1F0020F01E0020FF
:2022E000F71E0020A87896F90040401CA870601E30700FF017FC13F001FB0198234B6FF0B1
:202300000104A0F80A8193F8FC022C8110B11E48007808B913F072FC97F90000401E3870F8
:2023200096F9000010B9114880F8008097F9000078B10299039D58464FF0E04608402E4047
:2023400008BF002808D097F90000002804DC14F048F8002001F0AEF8009805B080F80080DE
:20236000BDE8F08FF61E002002150020EE1E0020C813002000000C8C28190020581D002019
:202380004D360020493600204B360020200800202DE9F041C94CCA4DDFF828836088ADF197
:2023A000600D4108C0F083800CA808A90FF088F901286DD1404624300068D8B10769CFB1AD
:2023C000062002268DF808000022ADF80A600FABADF80C2002AE009396E803000C23B84774
:2023E00040B9BDF83C006085109FE7621198206313F0FAFC0226BDF82210BDF8200084F891
:20240000246009AAA1830FF015FD011C02D0B7A013F0DBFF30460FF023FABDF830009DF821
:202420002C70A5F840000DA985F8427005F1500055F02DFCBDF8320005F1460609A9A5F812
:202440004E00304655F023FCBDF82200B5F84010A5F84400502013F005FBB5F84E105320AE
:2024600013F000FB4A20314613F0FCFD95F84210E12013F003FBB5F844104B2013F0F2FA45
:2024800005F10A00102155F0DDFB0120207008E012F09CFFE06001200FF0E2F9002013F05A
:2024A00061FDA01C012155F0BFFB2046408880080FD3E06A12F0D6F99348006800688047BC
:2024C00000B2A082E08202F081FDA01C022155F0ABFB6F89780805D305F10A00012155F0D5
:2024E000A3FB6F89B80805D305F10A00022155F09BFB6F89780917D384491820422217AB22
:2025000053F072FE95F85A0005F10A06032818BF042802D1286E12F08DF911F0EDFA30469E
:20252000102155F081FB6F89B80907D30EF05CFB05F10A00202155F077FB6F89F80907D3F6
:202540000BF0D6FF05F10A00402155F06DFB6F89780A0AD395F85D0013F004FD05F10A0058
:202560004FF4807155F060FB6F89380950D395F85C0005F10A0600283ED0401E36D0401E44
:2025800002D0401E30D03EE095F85810472013F075FA95F85910542013F070FAB5F8441047
:2025A0004B2013F05FFAB5F84010502013F05AFA092701238DF8597095F842008DF85A3010
:2025C00016AA8DF85B3052498DF85800182053F00BFE95F85A00012815D1E87898B130461A
:2025E000202155F02FFB0EE003200AE05220012113F02CFA022004E05220012113F026FAB6
:2026000001200FF0F9F83046082155F00DFB6F89454617B1A86813F0FDFFE98868784908C1
:202620001CD3A97802094FF0000601D301290ED040090ED301290CD030A013F0B1FCA01CF2
:20264000012155F0FFFAA86813F0E4FF01E010F00FFD6E70A81D012155F0E6FA608800283D
:2026600040D10A2008252B4CADF812004FF0FF37ADF81050616A059704A88847002831D13E
:202680000720ADF84850616AADF84A0012A88847149E159630BB20499DF84E20087890428D
:2026A00015D19DF84C004A7882420DD089684B6C6BB100213246984709E0C0465C18002031
:2026C000E019002058170020304600F0EBF9159840B1ADF818500320ADF81A00616A079613
:2026E00006A8884718B0BDE8F081C04641757468204572726F723A20307800C05374617261
:2027000074696E672E2E2E00EC010010813301003F6301008C1A0020D81E00202DE9F04FF7
:20272000064692F808B0307D09AF8946ADF1240D04933528039205D0114606F170000A22C0
:2027400055F050F8DFF8C4C239F07F0506BF604600884FF6FF700590F08A800934BF002090
:2027600008203076F08AC00834BF102080207076F08A400903D260460E30007800E00020AC
:20278000B076F08A41082CBF20240024000928BF44F010047568002109F07F09307D069102
:2027A0006D1E02280EDB0D2808DA0C2803D1022044F40854069044F0030404E00D280CBFF1
:2027C00002200120044396F88C0008B144F00804210900D328B1DFF8C88298F8203413B9B5
:2027E00008B1DF204BE121096ED306F12401DFF8A4A296F88D50079100EB0A011AF8053011
:202800000A7999183389491DCAB29918A24B1A8808908A42C0F2358100284CD0049A03995C
:2028200006F184000AF0C8FC0799002808603FD0806AB0F1FF3F39D070680023401E8DB1B7
:2028400096F88E10524600F80119515D491EC9B241B18A1992F88320491EC9B2002900F84D
:202860000129F6D1079970660968896AB162090E00F8011996F82A1000F8011996F82910B0
:20288000089A00F8011996F8281005F0030500F8011902F0070141EAC501017071683589BC
:2028A000091ACAB27060A918318105E0DB2700E0F3277770E6E00023F08A7370C00828BF79
:2028C00044F0100475686D1E336DA3B9B36D93B998F83914012903D13089B0F5EE7F06DA5A
:2028E000200904D202290AD144F4005401E044F48054012002E044F408540220069098F87B
:20290000020001280CD098F8FC0248B196F86B00042805D1022024F48054069044F40054FE
:2029200044EA8934B9F1020FA4B20AD0B9F1030F10D1ED1F08F22C41284655F017FA6D1E62
:2029400008E0B8F81204001205F8010998F8120405F80109069802280CD0B9F1000F15D0C1
:20296000BBF1000F0CD004990598814208D144F040040BE0BBF1000F08D1B9F1000F05D065
:202980000599081205F8010905F8011944EA8B24BBF1020FA4B209D0BBF1030F0ED103995F
:2029A000ED1F284655F0E2F96D1E07E003990888001205F80109087805F80109BBF1000F84
:2029C00005D00498011205F8011905F801093878F0B932480178307D0D2814D068B9306D85
:2029E00028B998F8FC03411C88F8FC130AE098F82104411C88F8211404E098F80A04411CEB
:202A000088F80A14014605F8011903E02E0C002044F48074201205F801092C7070683789E4
:202A2000401BC1B2756078183081200926D3B06D00B1306298F8FC0210B1307D0D281DD111
:202A4000746A14F1150001D113F0CBFCA16A481CA0623289306AB162471B0092D21B019097
:202A600090B20290706A96F88C202B46153008F061F900281CBF7070071C07D10020707088
:202A800005E0E5277770F32012F0C3FFF8B209B0BDE8F08F687A0100101F00206834002012
:202AA00020080020B0B50446BA480768ADF1480D002F00F0A8812078401E112800F2A3812E
:202AC000DFE810F06A015201380123011B010401F100E300C300B2008D005D00530042002B
:202AE000A1012A001C001200F86B002800F08B81684621460DF01CF8F96B82E1386C00289C
:202B000000F081816846002101220DF043FF60788DF80000396C74E1F86A002800F07381CD
:202B2000684600210E220DF035FFA11C684613F011F8A57BA1890022ADF80A1005B10122EA
:202B40008DF80C20F96A5DE1B86B002800F05B816846002102220DF01DFFA5788DF801500D
:202B600060788DF80000B96B4BE1786B002800F04A81684621460CF0DBFF796B41E1386B4E
:202B800008B36846002114220DF004FFA5788DF80150A3680193A289ADF80820A17B8DF84A
:202BA0000A1060788DF80000E57B8DF80B50237C8DF80C3094F911208DF80D20616904912F
:202BC000396B684688476068002800F01C810146F22008700020487010F0ECFF13E1B86AAD
:202BE000002800F010816846002124220DF0D2FE6078A11C8DF800000DF1020012F0AAFF85
:202C000004F10C0103A812F0A5FF257EE08A04F119018DF818500B22ADF816000DF1190059
:202C20000CF076F9B96AECE0786A002800F0EB806846002102220DF0ADFEA5788DF8015047
:202C400060788DF80000796ADBE0386A002800F0DA806846002112220DF09CFE6588627903
:202C60006078ADF8025023798DF80520E11D8DF80000A5798DF804300B220DF107008DF82E
:202C800006500CF045F9396ABBE0F869002800F0BA806846002101220DF07CFE60788DF8ED
:202CA0000000F969ADE0B86910B120460FF0C2FDA07820B9A069002800F0A58003E0A069FC
:202CC000002800F0A08012F071FB9CE07869002800F099806846002113220DF05BFE6D46B3
:202CE000A01C0168406829600B22686004F10A0102A80CF00DF9796983E03869002800F0DF
:202D0000828020460BF09EFB7DE0F86800287AD0684600210E220DF03DFE6078A11C8DF837
:202D200000000DF1020012F015FFA089ADF80C00F96866E0B868002865D06846002114227A
:202D40000DF028FEA01C01686D46296040686860A07A0B2204F10B018DF808000DF10900A3
:202D60000CF0D6F8B9684CE0786800284BD06846002110220DF00EFE60786588211D8DF887
:202D800000000B22ADF8025001A80CF0C1F8796837E0C046E01E00203868A0B368460021D3
:202DA00019220DF0F7FDA01C01686D46296040686860A07A410824BF01218DF80810810888
:202DC00024BF01218DF80910C10824BF01218DF80A10010924BF01218DF80B10C10924BF87
:202DE00001218DF80C1030F07F001CBF01208DF80D000B220DF10E0004F10B010CF088F82D
:202E000039686846884712B0B0BD70472DE9F84FDFF844830F460646F80B80F05B81C24DB4
:202E2000CB4CDFF81C932878B90F80F0EA80B90880F0DD80DFF8F8A2DFF810B3F90A80F0A7
:202E4000B380B90B80F09E80DFF8E082790B50D2380C40D23809C0F0608111F011FF0028AD
:202E600034D055464446032128682170783013F0D4FA0BF0D7F8AF48007818B92868403061
:202E800013F0E9FA022011F087FA11200AF092FB2868007C10B90E200AF08CFBA6490878FD
:202EA00020B100200870052011F076FAA34813F0B3F900224846B0F91410B0F916002270AB
:202EC000814214BF022007200CF060FD27F008070FF096F821E14846416889684E88002ED9
:202EE000FAD04168896849880129F5D027F40047EEE720B1042011F04FFA0020287011F07F
:202F000065FA0146002001B10120002540B1B0696FF480712A464FF0007384463046E0470C
:202F2000884889492A4613F088FAB0684146022203880A70A3F602032BB141F21E015B1AF1
:202F400018BF183000D11030018821F47C7141F434710180757420685C46006B2668804788
:202F600052467C4912680B68934214BF01222A1C26B1801B01EB8201000B886027F4805730
:202F80002560A5E7404613F062FA011C09D0486838B14A68C868B1F92C1020231446002225
:202FA000A04727F40057B8E013F041FA8046484613F04DFA061C14D05546286810B17830AA
:202FC00013F02BFA2068F168006B296080475C462060624813F020F961484FF4006113F0F5
:202FE00042FA404613F012FB27F4806795E007F02FFF4846103013F02AFA08B927F002078D
:203000008BE0584A116841F08001116020B1042011F0C2F90020287013F009FA8046B068BA
:203020000188A1F602052DB141F21E016D1A18BF183000D1103001884B4D21F47C7141F42A
:2030400034710180286808B3606D0068014604208847D8B120682C68006B8047F168001B45
:20306000728AF060F068000BF060F0688018F060F068884203D240184008F060F06840F69C
:20308000C41181422CBFB0F5FA7FF160404613F0BDFA11F09BF990B1B0696FF48071002299
:2030A0004FF0007304463046A047484613F0CFF9002808BF47F0020701D00EF0A1FF7069E7
:2030C00000214FF0806304460A463046A04727F0005722E013F0ABF90146404613F0B7F91F
:2030E000061C15D0356AA80812D225EA05003062084613F08BFA706868B165B17168B6F98B
:203100002CC0F06800232A468E466146F04702E0084613F07BFA27F480471FB110483946F5
:2031200013F0A1F9BDE8F88F1235002040360020FC3400201035002011350020A9B3000052
:20314000C435002054350020D98F0000043500208C01001090330020CC35002021A4000086
:20316000FC330020CC210840003500202DE9F04F09AFADF13C0D08900A92388809911E4690
:20318000ADF81800101C08BF002000F08A81002700F101094FF0FF3A4FF0010BB84672E12E
:2031A000252940F069811078521C0A922D2818BFADF8068005D15846551CADF806001078A6
:2031C0000A9530281CBFC446424605D10A990878DC466246491C0A912A28CDF80080554696
:2031E00017D13068CDF808A00A99CDF810C0C01C4B1C20F00300001D306050F8044C0A9372
:20320000002C0878009419D5ADF806B06442009414E044460AE00A9B610001EBC4010918AB
:20322000A1F1300418780094591C0A91302801DB3A28F0DBCDF808A0CDF810C02E282BD1DF
:203240000A9908782A2801F101010A9111D13068CDF80880C01C20F00300001D306050F8BF
:20326000045C002D48BF454608782B46491C0A9111E0434645460AE0690001EBC501091813
:20328000A1F130050A9908782B46491C0A91302801DB3A28F0DB02930AB1224604926C2890
:2032A00004D04C2818BFADF8048005D10A990878ADF804B0491C0A910BA9CDF80C800FABB5
:2032C00007916428059300F08D80692800F08A80BDF818C0752874D0782870D06F286CD089
:2032E000702851D063283ED073281FD009980A990128A1F101010A9116D96D490C68B5F197
:20330000FF3F03D0A84288BF6D1C00D8099D029508A80AA932466B46A0470A99C019074691
:20332000039801F1010975E040462AE030680A99C01C20F00300001D306050F8040CBCF135
:20334000000F01F10109014608B957A00146079112F0EAFD0390B5F1FF3F5CD0A842C4BF8B
:20336000281C039057E03068C01C20F00300001D306010F8040C5D468DF82C000A99039564
:20338000584601F1010946E0082035680490E81C20F00300001D306050F8041C082210238B
:2033A0000FA80DF00BFF411E0791402400F8014C0A99079801F1010929E0082302E0102328
:2033C00000E00A230A99306801F10109C01C20F00300001D306050F8041CAA42BCBF2A1CF8
:2033E000049210E00A99306801F10109C01C20F00300001D306050F8041CAA42BCBF2A1C5F
:2034000004926FF009030FA80DF0D8FE0790059D281A0390009CBDF80650211A241A009162
:203420005DB906E008A8202109AA11F094FC009C7F1C641E0094F5D503980546401E03906D
:2034400075B9BDF80600F0B10098401E00901AD408A8202109AA11F07EFC00987F1CF4E741
:2034600007990846491C0791017809AA08A811F072FC03987F1CE0E708A809AA11F06BFC4E
:203480007F1C09F101094A460A9812F8011C401C00290A907FF484AE089808B1414601701F
:2034A00038460FB0BDE8F08F286E756C6C2900C0AC8901002DE9F04FB94C05466068ADF19E
:2034C000340D8047DFF884B2A44FAE4E012D0B9000F0C4809BF8F503A14D0F2850D09C4837
:2034E00090F9000010F1020F05D19A4890F9000010F1020F44D0984C20783B68099003F11E
:203500003C0000688047099F61680023401AB900B0FBF1F2E768A0680A9704F1180787E890
:203520000C000A9F98464146BA4271EB080102DA3946884206D807464146BA4271EB0801D8
:203540001EDA0A90B9469A4604F11801B9EB02097AEB030A81E80006099A04F1180003C8E1
:203560001346DB1712F0C2FB183440F6B832D317801A9941002984E80300BCBF01202870AB
:2035800012F054FB002864D076480078002860D17548007800285CD174480078002858D1E0
:2035A00073480078002854D12878002851D17148007800284DD170480078002849D16F4801
:2035C0000078002845D1002054F02CF9002840D16B4F9BF86B94387800283AD16A4C206A04
:2035E000436CF068022106AA98479DF8180080B3DFF85C81226AF06898F90010002511F1D2
:20360000020F18BF01254FF0010A2DB1926B98F900109047226AF0684E4D95F9001011F1E0
:20362000020F03D0926B95F9001090476FF00100287088F8000087F800A0002012F034F94E
:20364000206AC169F0688847B9F1010F04BF0020607053490B988968884774E0012054F06A
:20366000E1F821460B9889688847484800780F280DD007F08FFD38680C36436C30680221BC
:2036800007AA98479DF81C0000285AD05BE03C4D9BF86B842878012853D1012012F004F944
:2036A0003B4F97F8C2000028FBD1374C206A436CF068022108AA98479DF8200050B197F82E
:2036C000C20038B9287801283BD10020287012F0B9FA36E03248406880472E4B8146022193
:2036E0000022B8F1010FF068297003F11007256A294E7A8009D004928DF8141001238DF832
:2037000015308DE8060004AA09E002928DF80C108DF80D2003F110078DE8060002AA2D6D9F
:2037200039463346A8471E498D68002801D512F058FE1A4991F90000E760401C087048465A
:20374000A84711F045FA0DB0BDE8F08F20080020EC1E0020ED1E0020301E002048190020CD
:203760004C360020493600204B3600204D3600204A360020EE1E0020EF1E0020F01E00209D
:20378000CF1F00204C1D002028190020150C0020B0300020C8130020CD2D0100F61E0020C6
:2037A0008C1A00202DE9F04FAA4C6068ADF12C0D8047A94A1178A94D08911278A168012AC9
:2037C0000BD0A54A01241470884728780795012805D02046FFF76EFE01E088470795AA4D62
:2037E0009F4CDFF8888295F86B14E068012900F0B080DFF870B29BF9000028B19A4890F98E
:203800000000002840F0AF80924840688047099000268DF8146004964FF001098DF8159013
:2038200008F59C7AC8F8406108F5A271AAF80260087808F5A27766F303000870387808F2EC
:20384000531369F3C7103870187808F2531269F300001870107808F2531769F3410010704B
:20386000387808F2531366F382003870187808F2531266F3C3001870107866F304101070AD
:2038800098F8530108F5AA7140F0600088F85301F4200FF075FD206A754A076D764B754808
:2038A00031468DE803001068514604AAB8476949A08000288968AF78069148D46A496F4B2B
:2038C00091F90000401C087093F90000002F00F1010018709BF90000C4F80CA000F1010067
:2038E0008BF8000014BF8021311CB4F85C004FF67F7208F5A876024011430843A4F85C0052
:20390000307867F3C7103070B5F80E04B5F81234082204F15F0705F22C463146A4F86A0011
:203920003846A4F8683053F05DFFB5F80E040822B5F81244A8F86A013146A8F8684108F582
:20394000B07053F04FFF0699099888476CE0B146FAE708F5847108F58477814205D1424876
:2039600090F9000008B100265FE03A48406880470026824695F8FC32A8F80A61002B07BF0A
:203980004FF48600311C3E482021B1463D4A8DF80D601378CDF808909B0904D212781209D3
:2039A00038BF012200D302228DF80C20226A166D314B2F4A8DE803001068394602AAB0472F
:2039C000244900288E68A0802CD427492B4B91F90000AA78401C087093F90000E760002AD9
:2039E00000F1010018700CBF4F468027B4F85C00B5F80E344FF67F71082201400F433843E2
:203A000005F22C41A4F85C00B5F81274A4F86A3004F15F00A4F8687053F0E4FE5046B04767
:203A2000012602E05046B0474E460A48406880470849896816B9084B089A1A70884707989D
:203A40000078012802D00020FFF734FD30460BB0BDE8F08F8C1A0020EE1E0020CD1F002059
:203A600028190020F81E0020F71E0020C8130020581D002020004300F11F0000F61E002043
:203A800000004F8C4A360020200800202DE9F04FAF4C0746201DDFF8B48200688946ADF1A7
:203AA0003C0D4FF0000B017DADF80CB0252900F00781703005A904F0D5FB002818BFC0B24B
:203AC00040F0418101A804A90DF006F912F05AF800280CBF41F2081543F2C82504A901A893
:203AE0000DF0FAF898F82B0201993B684FF47A7A10FB0AF00AFB1100C01A8542C0F2DD80DB
:203B0000D8F80422521A0AFB02F1C91A8D4200F3D480854208DD002806DD95FBFAF04FF4DE
:203B2000916110FB013038609DF81F0000285DD042F204000DF136010FF0B0F811F076FC2F
:203B40000699441A42F206000DF135010FF0A6F89DF835009DF81D10FF2804BF0A208DF838
:203B60003500FF2908BF0A219DF835609DF81C507848B4FBF0F2701884B25646A8105443D1
:203B80007043A04298BF041C41F20810241805A811F049FA9DF81C103D68B0FBF1F24A4320
:203BA000821A11FB06F192B206FB02F3CA1AC91A521B491B8C4201D900290CD5614291426C
:203BC00016D2002A14D53968B4FBF6F24FF4916312FB031508E061003C684FF49163B1FB86
:203BE000F6F18AB203FB02453D6001E03D68584606460DF1120102A80DF06EF80298D8F8C8
:203C000004125C46B5FBFAF280180290814203D998F82B32834202D998F898712FBB9DF8E2
:203C20001C00B6180004B04298BF361A9DF81F00002808BF9DF8200024D09DF81C00B6FB4F
:203C4000F0F085B2BDF833000EF014FF9DF83120014628460FF008FB054611F0D1F9024659
:203C600008A928460EF0CEFF0CE0814204D8BDF81200401CADF81200BDF8120098F89B11F2
:203C80000DF084F989F80000314F88F8F5017868007D052812D1384690F8110470B999F8F1
:203CA000000003A9ADF80C0042F20C0004F00CFABDF80C00A8F8F00100E06524204642E02A
:203CC00011F060FF00280CBF41F2081443F2C824214800784FF47A7510FB05F13868091B49
:203CE000A1F5FA62824206D2A1F57A61B0FBF1F24A43801A386068460DF10E010CF0ECFFD6
:203D00003868009998F82B6205FB0102009216FB05F18A1A944211DCA1F5FA619142BCBF0B
:203D200000F5FA60386098F89B11B8F878010DF02DF90146584689F8001002E099F800101B
:203D4000652088F8F5110FB0BDE8F08F4011002020080020A08601006B1300202DE9F04FA2
:203D6000002898461446ADF12C0D00F0F38011F47C1F40F0EC8011F00F0F00F0EB800746A6
:203D80000591002006900A904FF0000A0990554608954FF0010BCDF810B0054650460790DB
:203DA000059805990BEA000021EA0B014FEA4B0B401E059100F0AB80401E70D0801E5DD0B5
:203DC000001F40F0BE8042F205000DF10E010EF065FF9DF80E00002800F0B3801CB1276666
:203DE00094F86B0006900720152607F8010B022301A907F8016B42F2010007F8013B0EF021
:203E00004DFF684603A90CF067FF06980EF020FF0146019A00983E4640180090824206D857
:203E2000801ABDF80C300090581CADF80C00009B50085146814609041804030C1943000459
:203E4000534610EB090041EB0A0103F00DF80090BDF80C309DF80C009DF800209DF8011019
:203E600006F8010B181206F8010B9DF8023006F8012B9DF803200935BF1D42E002201526C2
:203E800007F8010B042307F8016BB8F1000F07F8013B0CBF099898F800002D1D4EE01CB151
:203EA000E76594F86B00069005201526049B07F8010B0DF10F0107F8016B42F2040007F86F
:203EC000013B0EF0EBFE02A80FF076FC06980EF0BFFE02999DF80F609DF80F30069AED1D2E
:203EE0004018000200EB6600B0FBF3F03E4602903F1D06F8012B9DF808109DF809309DF8DD
:203F00000A2006F8011B06F8013B327018E00320152607F8010BB8F1000F07F8016B0346B4
:203F200007F8013B04BF0A9807F8010B05D098F8000007F8010B98F801006D1D07F8010B40
:203F4000ADB2059800287FF42BAF2E4661E011F00F0F01D000205DE080468A4602264FF4ED
:203F6000803908F1020509EA0A002AEA090A4FEA4909B0F580301AD0B0F5803014D0B0F5BC
:203F800000300ED0B0F5802009D0B0F5002004D0B0F580102AD1072404E0062402E00524E8
:203FA00000E00424002704E00224012701E001242746A81C214600F08FF947B104F00F048B
:203FC000C0F30A0141EAC42141F4004105E004F07F0400F0FF0141EA042105F8011B0912CD
:203FE000871929702D18B81C6D1C86B2BAF1000FB9D1022ED8BF00260BDDB01E4FF6FE770D
:2040000008F8010BF019C0F3022040F0A00088F8000030460BB0BDE8F08F70472DE9F04F05
:20402000AA4C07466068ADF1340D80470B900AA9822004F06DFEA64EBDF8280038BB002498
:204040004FF6FF75ADF8284017E0ADF80450BDF82800ADF80650FF210822ADF8000002A839
:2040600053F0DCFB8DF81840D420694603F0E6F9BDF82800401CADF82800301DBDF8281094
:2040800000888842E1DC82200AA903F0D7F9DFF844920020B246ADF828009DF82800002684
:2040A0008DF8000069468DF80160D02004F030FEB0460126F0B99DF80B30012B07D19DF8A5
:2040C0000A0020B90DF1020011F0E0FD90B97D7B002D0CBF0522092246469D420AD10DF150
:2040E000020007F10E0153F041FB002818BF4FF0010809D1002E40F0D780B8F1000F03D1D6
:20410000787F002800F0D080564600240CE06F490B98896888471A20D4E0BAF804006D1C4C
:20412000ADB24BE0641CA4B2B088A04242DD9DF82800ADF8224008A98DF82000D12004F0E7
:20414000E7FD0028EED19DF82400FF28EAD0ADF800006946D42004F0DBFD002837D102A80C
:20416000391D082253F002FB0028DBD038887D88ADF80400B8F1000FADF8065008D0387B00
:20418000BDF82810BD698DF818000DEB81010D61D420694603F052F9B8F1000F0AD0387F5D
:2041A0009DF82510884205D08DF8250008A9D12003F044F9B088A04276D10025A84270DD5D
:2041C000ADF80050D420694604F0A2FD28B13F490B9889688847192074E00DF1080B5846B4
:2041E00011F054FD002300B101233C1D181C06D158462146082253F0B9FA00288DD07B8864
:2042000038883A7BADF80630B8F1000FADF80400BDF828308DF818200DEB830101F11001A4
:204220000CBF0020B86908220860214602A853F0D9FA99F8FC0230B1D9F84C231AB1BDF889
:20424000001020469047002401E0641CA4B2B088A0427FF762AF9DF82800ADF8224008A920
:204260008DF82000D12004F053FDE82803D09DF82400FF28E9D19DF8000000228DF8240087
:204280003B7F8DF8262069468DF82530D42003F0D5F808A9D12003F0D1F8B088A0427FF76E
:2042A0003CAFA8423FF433AFBDF82800401C80B20228ADF82800FFF6F0AE04490B9889683E
:2042C000884700200DB0BDE8F08FC0468C1A0020081F002020080020F0B504460846ADF1D8
:2042E0006C0D401E70D0401E0DD0801E00F00981401E00F0EF80401E00F0E180401E00F09A
:20430000AD80002042E142F2010007A90EF0C6FC42F20B0008A90EF0C1FC42F206000DF1A5
:2043200065010EF0BBFC42F207000DF166010EF0B5FC42F2050019A90EF0B0FC04A80AF0C8
:20434000CBFA06460DF1670142F209000EF0A6FC9DF86700002808BF002503D0022010F004
:2043600086FB0546204607A9042253F03BFA241D08A90222204653F035FAA71C9DF8640013
:204380009DF865309DF866109DF8674007F8010B9DF8672007F8013B2B4607F8011B610756
:2043A00006F0070444EA916005F0030404AD40EA8410314607F8010B012400953846019423
:2043C00007F06EFA0A309AE042F206000DF165010EF064FC42F207000DF166010EF05EFCD6
:2043E00042F2040019A90EF059FC04A80AF074FA05460DF1670142F208000EF04FFC9DF891
:204400006700002808BF002303D0012010F02FFB03469DF864009DF8657004F8010B9DF8BC
:20442000666004F8017B9DF867209DF86770790704F8016B03F0030705F0070646EA9160AE
:2044400004AE40EA8710294604F8010B002700962046019707F024FA001D50E042F215000C
:2044600011A90EF01BFC13AF42F2160039460EF015FC15AD42F2170029460EF00FFC17AE89
:2044800042F2180031460EF009FC204611A9082253F0A8F9083408222046394653F0A2F9FF
:2044A00004F1080708223846294653F09BF9082207F10800314653F095F9202066E042F2DE
:2044C00014000DF122010EF0E9FBBDF8221002200A1258E009A80021202253F09FF942F245
:2044E000130009A90EF0DAFB09A853F099F9024609A9204653F076F909A853F091F980B2DC
:2045000044E042F20E0002A90EF0C8FB0DF10A0142F20F000EF0C2FB0DF10B0142F20A007A
:204520000EF0BCFB03A942F210000EF0B7FB0DF10D0142F211000EF0B1FB0DF10E0142F2EA
:2045400012000EF0ABFBBDF808009DF80B209DF80C709DF80D609DF80E509DF80A1004F877
:20456000010B02F00102001204F8010B07F0010042EA400206F0010042EA800205F0070019
:2045800042EA4012042004F8011B22701BB0F0BD2DE9FE43A44C80460F46B8F1450F08D11F
:2045A00004F50F753422284653F01CF9C4F8F05337E111F079F8FF2808BFF42000F0328134
:2045C00094F86B14022907D1B8F1E80F00F02981B8F1E70F00F02581944D05EB8005A878E8
:2045E00010B9E978002937D0E978814208BFFB2000F01881B8F1580F24D0B8F1600F1AD0CC
:20460000B8F1E00F0ED0B8F1E80F05D03A7890421FDC91421DDB1FE0387894F83B14884211
:204620001AD1FEE097F900000CF02AFA4FF6FF7181420ED010E038880A280ADBB0F5804F70
:2046400007DA09E038888F2803DB47F60251814202DCE820BDE8FE83774E706880478146B1
:2046600028786A783946201800F57A7053F0BAF8B168484688474046503800F0C680801ED5
:2046800000F0AD80401E00F0BD808D3800F0B580401E00F09B80401E00F0AC80801F1ED018
:2046A0000D3840F0BE800E2094F869748DF8020017B11B208DF8020094F92A149DF902003C
:2046C000884204D0E0200DF10201FFF761FF11F0F9F894F86904002800F0A38073E001214A
:2046E00003208DF8051030278DF8030000258DF808704FF4FA568DF8065094F83B14ADF80E
:204700000060052080298DF8040009DD842907DA8DF8030014278DF8087008208DF80400FD
:204720009DF8030094F80D14884204D04F200DF10301FFF72DFF9DF8040094F819148842E7
:2047400003D0572001A9FFF723FF94F83B04842808DB862806DAC0208DF808004FF4FA4774
:20476000ADF800709DF8080094F81D14884203D05A2002A9FFF70CFFBDF80000B4F81A1478
:20478000884203D058206946FFF702FF94F83B0478B902208DF805000B278DF8075024493B
:2047A0008DF806707D260E80E7200DF10701FFF7EFFEF7200DF10501FFF7EAFEE1200DF1E5
:2047C0000601FFF7E5FE0DF063FB2AE094F82B040EF0F0F9012824D01A20BDE8FE8394F8E9
:2047E000110418B902200FF011FB1AE0022011F081FC16E00FF0F4FC09E094F92A0411F082
:2048000057FB0EE010F0C0FB01E010F0A9FB94F86B04022805D107480078012801D00BF061
:20482000F5FB0020BDE8FE83200800208C7D0100101F0020181F00208C1A00202DE9FE4F21
:20484000DFF83892074609F1040000688047DFF8248200248346002F88F8034064D010F0AD
:20486000A1F908F26C402146AC22054652F0D6FFDFF804A20AF104000188C80000EB011098
:2048800080B253F01FF8C8F80C0560B105F18C070226BAF8040000EB400080B253F012F899
:2048A00047F8040F08B911F09CFD761EF1D1E81DFF21082252F0B2FFFF2105F11000082263
:2048C00088F87B1452F0AAFF022703234FF6FF7C012288F88C3405F19400A8F88EC40421CB
:2048E00000F8042F417083707F1EC170F8D105F1A0000526022700F8042F417086707F1EF9
:20490000C270F8D1BAF8047085F8A8304FB12146D8F80C057F1E084401F11801A0F802C08B
:20492000F6D1022088F8700498F8FC024D4618B1D8F8000300B180470DF058F998F92A0458
:2049400011F0B6FA0EF048FC10F00AFB10F01CFB0FF046FC4A4F072657F8040B00B180476B
:20496000761EF9D111F07AF9464606F14C00016809B10EF037FE4348006886F85640C0B1C8
:2049800012E0384652F042FE029002A80EF02AFE20E0384652F03AFE019001A80EF022FE73
:2049A00014E068460EF01EFE52F02EFD00280090F7D135480078012802D02046FEF77AFD8C
:2049C000324896F86B8406F178070470B06F0028DFD13F1DF06F0028D3D1B467F46786F884
:2049E000824086F88340B8F1020F86F8844004BF2748C6F890002748C6F88801264FC6F84F
:204A00008C71264BC6F89031B470254AC6F894212449C6F89811244FC6F89C71234BC6F865
:204A2000A031264B224AC6F8C0302249C6F8A421234A214FC6F8C420244BC6F8A81121495D
:204A4000C6F8AC71204FC6F8C8105846C6F8CC70A968C6F8D030884706F211415220FFF78E
:204A600097FD96F82B040EF0A5F80DF0BFF82046BDE8FE8F20080020081F00208C1A0020A9
:204A8000280900203C360020CD1F0020483600207B640100070A0100E9630100C14E01003A
:204AA0006D7D000021C700002D5501009D4401009DA70000A98B0000A9410100D7ED000098
:204AC000E9970000711301000DF20000C11A01002DE9FE4F0546287D012808D195F91700FC
:204AE0000BF0CEFF4FF6FF71814200F016819548EF7B017894481FB990F883208A4208DBA1
:204B0000012F03D190F882208A4202DBF120BDE8FE8F80462E6A95F83500B5F8289095F869
:204B20003470AC8B4FF0000A5FEA060B029017D098F8FC32002B2FD0D8F8141300292BD07B
:204B400006F0FF008847D8F8141306B20BF47F008847361830B2001D00B2C83086B200E086
:204B6000C8260CB1241DA4B298F82004012809D147B1764802993F1897F804A0405C80192C
:204B8000401D86B209EB040080195044801C80B252F0BAFD071C02D11A20BDE8FE8F09EB3E
:204BA0000A0033193881002C03EB070078600EBF0020B819801C00217822C7F8A40007F17D
:204BC0000C0052F02BFE09EB0600FF2110220019A7F84C0007F13C0052F020FE07F12C0056
:204BE0000F21102252F01AFE00243C707C707868696A2A8D52F0F6FD07F1840005F12C01FF
:204C00000B2252F0EFFD07F19000294610F0F4FE6889A7F89A00287B87F89C00687B05F18F
:204C20000E0687F89D00326869460A60706848609DF800102046012908BF01209DF801104E
:204C4000012908BF40F004009DF80210012908BF40F008009DF80310012908BF40F0100086
:204C60009DF80410012908BF40F020009DF80510012908BF40F040009DF80610012908BFA3
:204C800040F080009DF80710012908BF40F48070A7F89E00A87D87F8A000E87D87F8A1009D
:204CA00095F8380087F86C00AA8BA7F8A82022B1D7F8A400A96952F095FDA87F87F8AA002C
:204CC000286AC7F8AC00B7F8A800C0B1D7F8A400A8B17868401E7860F82101707868401E65
:204CE00078600470B7F8A810B7F8A8607868401A786038898019801C38817868B865B7F8DD
:204D00009E00410A16D395F83710042905DD00F0040100F00100084302D0E820BDE8FE8FA1
:204D200008F1880630460BF0C1FB95F83710304610F000FE98F80000394652F0DBFB2046EA
:204D4000BDE8FE8F081F002020080020687A01002DE9F04142F20400ADF1280D0DF123013B
:204D60000DF09CFF42F205000DF122010DF096FF42F2010069460DF091FF8C4C8C489DF8FD
:204D80002310C4F8A801642011FB00F1C4F8A0118849C4F8C4119DF8221011FB00F0C4F8AC
:204DA000BC018548854EC4F8E001B07888B342F203000DF106010DF071FF10F021F9054688
:204DC0000DF1060029460DF087FA2D1A9DF8220084F89B5170B1009860B104F5DC700DF070
:204DE000F9FD04F5BA700AF02DF9012084F8940184F8980142F202000DF106010DF04EFFAE
:204E00000DF1060010F0C2FA04F5CE700DF0E2FD11E042F202000DF106010DF03FFF0DF15A
:204E2000060010F0B3FA04F5CE700DF0D3FD04F5BA700CF0CFFF96F83B040FF049FBC07B83
:204E4000022804BF012084F8F40194F8F801002840F0A88004F128000021382252F0DEFC1A
:204E60000026A681E08900EB800080B2804652F029FD04F12805074627610FB911F0D1FA26
:204E800038463146424652F0C9FC4D484D4FE06305F1080067630DF09DFD42F21B0001A9C2
:204EA0000DF0FCFEBDF8040001A9A4F84C0042F21C000DF0F3FEBDF8040001A9A4F84E0025
:204EC00042F21D000DF0EAFEBDF8040009A920835D200EF055FA9DF8240000280CBF301CCC
:204EE000012084F85C00B4F84C0038B100EB401080B252F0E7FC0028606551D0B4F84E003E
:204F000040B1410001EB800188B252F0DBFC0028A06543D0208B38B1C00080B252F0D2FCC9
:204F2000606108B911F07DFA27490DF11A00082252F058FC01273546208BA84223DCB4F84C
:204F40004C50668355B1606D4FF6FF720146A0F81F206D1E8E7701F12100F7D1B4F84E5070
:204F60004DB1A06D4FF6FF71024681806D1ED67002F10600F8D1201D3146062252F04EFC2D
:204F800084F8F8710EE060690DF11A01082200EBC50052F027FC6D1CADB2CDE711F041FA45
:204FA00011F03FFA0AB0BDE8F081C04640110020252A010091BA00008F630100200800209A
:204FC0004DA50000002A7515C0810100F0B500215022ADF15C0D02A80BF0DCFCF22016A95C
:204FE00011F038F88F4DBDF8580016A9A5F87000F32011F02FF8BDF858000DF10901A5F8DE
:205000007200E22011F016F8688DADF81200410806D305F11401096805A80160BDF81200EE
:20502000810805D3291D098806A80180BDF81200C10807D305F1180109680DF11A000160A6
:20504000BDF81200010908D30DF11E0005F15401302209F05DFFBDF81200400903D3286B1D
:205060001590EF6A14977048007800280CBF01210021012052F032FDBDF8120041082CBF94
:205080000F240B24810824BFA41CA4B2C10824BF241DA4B2010924BF3034A4B2400924BF16
:2050A0000834A4B220460FF07FFE071C00F0B78005260DF1090100F8016B0A680260496816
:2050C0004160BDF81210083052F0D5FDBDF81210844648080BD3BDF81410604652F0CBFDB4
:2050E000BDF8161052F0C7FDBDF812108446880807D3BDF81810604652F0BDFDBDF812106E
:205100008446C8080BD3BDF81A10604652F0B3FDBDF81C1052F0AFFD8446BDF81210434AA3
:205120009388080961D3BDF81E10604652F0A3FDBDF8201052F09FFDBDF8221052F09BFD20
:20514000BDF8241052F097FDBDF8261052F093FDBDF8281052F08FFDBDF82A1052F08BFD5F
:20516000BDF82C1052F087FDBDF82E1052F083FDBDF8301052F07FFDBDF8321052F07BFD5F
:20518000BDF8341052F077FDBDF8361052F073FDBDF8381052F06FFDBDF83A1052F06BFD5F
:2051A000BDF83C1052F067FD194652F064FD117852F061FDBDF8421052F05DFDBDF8441071
:2051C00052F059FDBDF8461052F055FDBDF8481052F051FDBDF84A1052F04DFDBDF84C104F
:2051E00052F049FDBDF812108446480906D31499604652F0FBFC159952F0F8FC05F11C01D9
:20520000224630463B4604F075FD0820ADF80260074D01972968ADF800006846884717B034
:20522000F0BDC0465C180020021C002058170020B01A00202DE9F04F8146D9F800600C46D1
:205240005FEA0208ADF11C0D14BF00214FF0FF3106F14805284610F0DAFEAA46002818BF58
:205260000B2040F00B8188480025F460B8F1010F057007D0657002200FF0C4FA06200FF020
:20528000C1FA01E0012060702078012840F2AB80801E012868D9801E012832D9801E0128C2
:2052A00000F2DD8011F0C3F84FF080578346D7F8DC11A0784E6A0090217807F5EE77284680
:2052C000062908BF0120019001200290A068228A6368E168B0470646584611F097F9002E0B
:2052E00040F0BF80B8F1000F02D010F03FFC02E048460FF0A5FB002800F0A4803868806AA5
:205300002BE011F094F883464FF0805CDCF8DC0101270068009726786368A168A278AE46B9
:20532000042E0CF5EE7408BFBE46064618467346B0470646584611F069F9002E40F09180F7
:20534000B8F1000F02D010F011FC02E048460FF077FB002876D02068406880474949C1F825
:20536000B0510D6006467CE011F061F807464FF08053D3F8DC01E18A80690091E1680191F6
:20538000218B0291A1780391217D04910122059221782E4603F5EE75022908BF161CE1784F
:2053A0006268A36884463046E0470646384611F02DF9002E55D1B8F1000F02D010F0D6FB11
:2053C00002E048460FF03CFB00283BD02868006A8047061C45D12868A168E28A2369C5693C
:2053E000E078A847BEE711F022F883464FF08052D2F8DC01E18AC0680091E1680191218B7A
:205400000291A1780391217D04910121059127782E4602F5EE7507B90E46A368E1786268B2
:2054200007463046B8470646584611F0EFF8C6B9B8F1000F02D010F099FB02E048460FF0CC
:20544000FFFA08B9142019E0286840698047061C07D1286802692169E078904782E74FF00F
:20546000FF36B8F1010F05D002200EF095FF06200EF092FF504610F0EEFF304607B0BDE8AB
:20548000F08FC04650450240473600208E492DE9F04F06460822ADF16C0D15A852F0A2F9C0
:2054A0008A4C94F8F30106F1280A06F12807002800F007817078002840F00381FF20844BF5
:2054C0008DF818001D78F06C012105AA02F086FADFF80092DFF8008228B99DF8180008B9EA
:2054E0009DF81C5070BBB08900F00700022814BF04200520B073B08900F00700032807D1B4
:2055000073684046001D01681878042800F09C8096F83000022815D149468878012811D075
:2055200001F57A710D4606F12800022220310FF0C3FE38B905F116010DF13E0052F016FC55
:205540000DF13E07706E002800F0BB80012102AA0AF04BFC002840F0B4809DF80800B0737C
:20556000F06C40B1394612AA0DF14A03FBF7E4FE002840F0A6800DF14A000090706E3946D1
:2055800012AB06F0DBFC002840F09B804946891C0878012854D04FF4005013A90DF07EFB48
:2055A00013A815A908220FF087FE30B113A8394608220FF081FE002842D194F89901002878
:2055C0003ED0D4F88851B4F8846142F2010004A90DF064FB049A4FF000410020E5FB021019
:2055E000051CD4F8900110F0EEFC2D180498A84202D8761C2D1AB6B24746786880475FFAD0
:2056000080F8D4F88001A84205D1B4F87801B04208BF00260BD0C4F88051A4F87861002004
:2056200084F875010FF002FF0126C4F88C01B968404688470EB10BF071FC012084F8980135
:20564000002084F899013CE0CDF85CA08847AB46224D0A274FF00008CDF864A096F8309079
:20566000189014F809A0287A484505D11999524628460FF021FE20B17F1E05F10C05F2D1BA
:2056800000E0A8465FEA08070ED194F87001134A0C2110FB0127401C84F87001C0B20A285E
:2056A00004BF002084F87001179938460A2252F099F809491898896887F80AB088470420CE
:2056C000B0731BB0BDE8F08FC081010040110020171F0020200800208C1A00203812002037
:2056E0002DE9F043071CADF1240D00F01381F86B002800F00F81B7F84020002A00F00A812C
:20570000007817F130014FF0000603D097F83810052902D0002E00F0FD80DFF80482401E93
:2057200069D0801E55D07F4CC01E3DD0001F40F0F1807A4DA878002800F0EC8003A831466A
:2057400004220BF027F9B7F840002A78032840F0E180F86B401C52F094FA434603F17C072C
:205760003988012A01F10101398009D0D988421A022A05DBB3F87E108918491EA3F87E1084
:20578000D880E7782E70400808D2012F00F0C2800121E170304652F0A1F9BBE0002F00F0B1
:2057A000B980E6703146F5E7012A40F0B3800725E0788DF8205000280CBF0121311C304628
:2057C000E17052F08BF9E07802228DF8210028460CE0012A40F09E804346B3F85C0001220A
:2057E000401CA3F85C0004208DF82000394608AB04F080FA8EE0684631460C220BF0CAF86F
:20580000B7F840000B285ED1FC6B14F8010BC14689F82800204652F034FAA41C03462046C3
:2058200052F01EFA0546201D52F01AFA8046387A4C4689F82400022806D0396804F11C00CF
:2058400001607A68426001E03888A08303F00100190928BF40F00800590928BF40F01000E1
:205860006085834218BF0226B5F57A7FADF8020016D32D48A84213D3E56210F0A1FA81465E
:2058800010F09EFA00EB092910F09AFA00EB0920B0FBF5F16943401A0A300EF0E3FF00E01A
:2058A0000226E06AB8F57A7F019008D342F21070404504D3C4F8308010F096FA00E0022650
:2058C000206B029001E04446012602258DF8016068468DF800500DF037FC0DF111009DF8B5
:2058E00001108DF8105052F0C6F9BDF8021052F0C2F9019952F07AF9029952F077F93946D2
:205900000D2204AB284604F0F5F9B4F86200401CA4F8620009B0BDE8F083C046E019002001
:205920005C18002058170020407E05002DE9F84F86468448DFF820C2DFF80C92834F844EBA
:20594000DFF81082DFF814A2DFF814B20478012C64D04D4601242C7000244FF0E0453C704F
:2059600004EA020015EA0307347008BF002843D10820274610401F4008BF002833D04246C9
:20598000654692F90000B5F8A230401E107042F201429A4202D0121D9A4209D1504600686C
:2059A000826C70469047008842F6014181420CD1688FB0F5105F1BD16A480068594600F525
:2059C000C07008600EF0ECFD1DE0E12009F04EFF98F90000002800F0A98098F90000002879
:2059E00000F3AB80A0E0454695F90000401E28701D2009F03BFF06E0454695F90000401E2D
:205A0000287010F037F998F90000002800F08E8098F90000002800F3908085E04D4601242E
:205A20002C7000243C70504834700688022707EA020514EA030708BF002D15D120464FF088
:205A4000E04700EA020117EA030008BF002903D11D2009F00BFF50E0454695F90000401E83
:205A6000287010F007F948E0424692F9003065465B1E137043F20842B24208D0B5F86A70AA
:205A8000931CB34203D0BA4218BFBB4216D150460068826C70469047008843F603018142D7
:205AA0000AD007F021FD98F9000000283ED098F90000002838DD40E0B5F86A70B5F8C2103C
:205AC00043F60400884220D0B8421ED0B5F8862090421AD0B1F5505F05D0080B0BD31D2080
:205AE00009F0C4FE07E01F480068594600F5C07008600EF055FD10F081F898F90000A8B156
:205B000098F9000000280FDD17E018480078022810D003280ED007F0E7FC98F9000028B1BA
:205B200098F90000002808DC10F05BFC2046FDF7C1FC02E0204609F099FE89F80040BDE81C
:205B4000F88FC0468B0C0020CD1F0020F01E0020EF1E0020F61E0020C813002048190020EA
:205B6000401900200C0100214E1400200E1E00202DE9F04781498B4E0F7896F86BC4002F4D
:205B800040F0F7807E4C894601210128A070756889F8001040F29780DFF8E881DFF8ECA10F
:205BA000801E47D0401E35D0401E00F0A180401E1FD0401E40F09A8095F86D00608195F801
:205BC0006E00002806BFE170081CE0706E4A514609781278474612FB01F148438100396416
:205BE00007F14401087820F00F0040F0030008708BE0BCF1010F40F088800020E98A60715A
:205C0000C90934BF96F80D1496F83614617010F0A9FA56E0BCF1010F09D196F83B040EF02C
:205C200057FCC07B022802D1002009F023F90EF0D1FC46E056480568BCF1010F1DD09AF86C
:205C400000008700E86B8047DAF804103C23401AB0FBF7F1B1FBF3F25A43891A227812FBF9
:205C600003F0401A3C301FFA80FAE86B804707FB0A014046016444301DE09AF8000087003C
:205C8000E86B8047DAF804103C23401AB0FBF7F1B1FBF3F25A43891A227812FB03F0401AF3
:205CA0003C301FFA80FAE86B804707FB0A014046C0F8C810CC30017821F00F0141F00201DE
:205CC0000170756821E00021EF8A6171F90934BF96F80D1496F83614617088B996F8EB03FF
:205CE00070B10229C4BF0220607009E010F079FB95F86900607195F86A0060700027A771B9
:205D000000F0A0FD7568002D35D02248007868B9002D2ED06968087800F0200020718878C7
:205D2000E0710878800901D210F0B8FAA078032803D0022818BF06281DD1174D6868804756
:205D4000A17802290CD015490F7817B914490F7837B1022189F80010A9688847BDE8F087F2
:205D6000832189F80010A96888470AF093FDBDE8F08710F036FBBDE8F087C0464D36002072
:205D80000C1E0020C8130020151F0020301E002048190020453600208C1A0020493600207B
:205DA0004B3600202008002001282DE9FE4F40F0F480DFF820A2DAF8DC00012840F0EA80C0
:205DC0000220CAF8DC000FF02BF801200DF02CFC5FEA000805D00120CAF8DC000FF034F88B
:205DE000DDE010F03CFB704D6E49029000200860A86A0068014601208847012818BF002050
:205E000003D100200BF048FA0120684F00903868112010F01FFA00280CBF00240124102093
:205E200010F018FA08B144F002040F2010F012FA08B144F004040B2010F00CFA28B1286893
:205E40005B49006B0246088890470A2010F002FA28B128685749006B02460888904756489D
:205E60000126066028688069014644F0200088475248066010F0E8F900F00101DFF844B113
:205E80000191400816D2286A806801464C4888478146B9F1040FF6D0B9F1010F05D1286AB0
:205EA000406802464648032190475946086820F0030008604448006842F2107240F2AA2336
:205EC000B0FBF2F15143401A83422CBF40484FF040403E49086028683968806B80470198E4
:205EE00001280ED0B9F1010F05D1286A40680246334831469047DBF8000040F00300CBF8F7
:205F00000000286840690146204688470B2010F0A1F928B128682649C06A02460888904756
:205F20000A2010F097F928B128682249C06A0246088890472048032206602049CAF8DC20E0
:205F400000230B602868406B0146204688470128F8D1386804200DF067FB04461148009DA7
:205F600006603868012D02D130460BF095F910F05FF908200DF058FB07460298CAF8DC6066
:205F800010F040FB0EF060FF57EA040018BF4FF0FF3804E06FF0040801E06FF001084046B9
:205FA000BDE8FE8F0C400940B80100102C200940428701003E8701002820086080010443B4
:205FC00000400340242208401C1400501C00094008E7A4803C1500207B4A2DE9F84F81465E
:205FE000854C5068800806D2106804F15001000C40F0F0000870D2F808B0DFF8D081754FE8
:20600000641E5E46B00E11D2700E0FD3802084F820004FF6D801A4F861103D462074A5F145
:2060200070000068C0F304600AF032F8684D55F8180CBA46C0F3400018B96749002008602B
:2060400001E046F040666549F00EB70E80F001004FF0805300F00100086087F0010000F0CE
:2060600001008860D3F8F06103F5F87072680090594648469047DFF86891DAF80070594B97
:2060800039F83B2C07F0FF06101280F0C000B04211D002F0FF021968B04234BF01214FF08D
:2060A000FF3140180102864281F4404142EA010129F83B1CEFD13809C7F30331C7F384467E
:2060C0006FF4017200F0F000014304F80810F90CA65401F0F00040F47040A4F86300DAF81D
:2060E000046028681F4620F0100828F4F070286057F8080C5FEA9B6002D25FEA5B6017D2B3
:2061000055F8180C800834BF300AF00800F0F80040F47840A4F86100207800F07F002070F9
:20612000207840F080002070C6F3044009F0B0FF46F3050321783A6841F30500984211D072
:206140009842B4BF01224FF0FF3201F04001801800F03F020A4322702178834241F0800175
:206160002170E7D138683868C5F800801E4957F8080CDAF814004026C0F3053089F8A30F28
:2061800043F61803E675009A0B8010688168584688471649164A0AE0105C9378141D834247
:2061A00099BF204410F8010C20444078086008684B689842FCD10228EED1012048620D4FB0
:2061C0003860BDE8F88FC046AC4F0050FEFDFFFF28000940F813005094042A43000220437B
:2061E0006BA00C40342009406AB00C4000600C402889010094046042066208402DE9F043B4
:20620000002B08BF002A10D10029BCBF00204FF0004106DB50EA01071CBF6FF000006FF081
:2062200000410BF084FBBDE8F0835FEA530898EA610803D50026404266EB01015FF00009D1
:2062400013F0004E03D00026524266EB03031C461546002C08BF8D429CBF2C1C0025070CAF
:2062600047EA01470E0CB44208BFBD429EBF240444EA15442D04070A47EA01670E0AB442DA
:2062800008BFBD429EBF240244EA15642D02470847EAC1774E08B44208BFBD4200F2928011
:2062A000870847EA81778E08B44208BFBD427BD8C70847EA4177CE08B44208BFBD4265D8FA
:2062C000070947EA01770E09B44208BFBD424FD8470947EAC1674E09B44208BFBD4239D83E
:2062E000870947EA81678E09B44208BFBD4223D8C70947EA4167CE09B44208BFBD420DD886
:20630000E60146EA5566EF01B14208BFB84201D3C01BB14159EB09094EEB0E0EA60146EAE4
:206320009566AF01B14208BFB84201D3C01BB14159EB09094EEB0E0E660146EAD5666F0170
:20634000B14208BFB84201D3C01BB14159EB09094EEB0E0E260146EA15762F01B14208BF71
:20636000B84201D3C01BB14159EB09094EEB0E0EE60046EA5576EF00B14208BFB84201D37F
:20638000C01BB14159EB09094EEB0E0EA60046EA9576AF00B14208BFB84201D3C01BB141A0
:2063A00059EB09094EEB0E0E660046EAD5766F00B14208BFB84201D3C01BB14159EB090937
:2063C0004EEB0E0EA14208BFA84201D3401BA14159EB09094EEB0E0EA34208BFAA423EBF83
:2063E0002D0A45EA0465240A8AD373464A465FEA080803D50026404266EB01015FEA480835
:2064000003D50026524266EB03031E4617460B46024631463846BDE8F08370472DE9FE4F12
:206420000CAF9946934604467D680291294604F0F3FB061C00F0EE803888F082774F3475B5
:2064400097F8FC0218B1012C04BF1520307506F1840029460B2251F0C5F9012C04D00D2CCC
:206460001CBF7068401C00D170683062002597F8FC0235650028B5654ED0052C18BF012CF1
:2064800045D14FF0040A86F86BA0F08A86F86950C00934BF97F80D0497F8360459460A226F
:2064A00086F86A0006F1700051F09CF99BF8080003282CD1032097F8113402903BB3DFF8A6
:2064C000608108EB8408D8F8000010F47F0F0ED086F82CA0D8F8000006F12C01012200F4C7
:2064E0007F003063304602F0E1F9D8F8000010F0FF0F0CD02A2086F83C00D8F8000006F1C3
:206500003C0100F0FF003064304606F0EFFD97F8FC0208B10D2C13D0009502994B463046CA
:206520005A46FCF7FBF8071C75D1E41F012C03D8707E40F020007076304606F05DF96AE031
:206540000520374C86F86B0004F13400016811F0F70F18D02A2186F83C10BA78006806F183
:206560003C01012A00F0FF0030641CBF20F00800306497F8110418B9306C20F002003064F2
:20658000304606F0B3FD009502994B4630465A46FCF7C4F85FEA00083AD122480660348970
:2065A000756801A964200CF0EBFE1F4EA01C0DF1050187B206F1D0000780E9200CF0E0FE54
:2065C0009DF80500012806D13C46C4F30220022140F0180006E0241D0421A4B2C4F30220E0
:2065E00040F0080005F8010D671A05F8014DB9B2C6F8DC50AD1C284609F080FC9DF80400F2
:2066000000280CBF09480A48C6F81801C6F8D800474600E01A27F8B2BDE8FE8F20080020A5
:20662000447B0100BC1C0020C81300204E9055550E7A55552DE9F047044694F830900F46B5
:20664000984615468B20ADF1300D0DF10A0102F05FFB8A20694602F05BFB94F825000028AC
:206660003ED1B9F1000F19D1BDF80A104FF6FE70884205DCBDF80A1088422FD1694615E0FE
:20668000B4F844009DF80A608DF80C0000128DF80D00BDF80A008DF80E601BE0B9F1020F6E
:2066A00009D0B9F1030F19D104F1280103A851F05DFB092612E0207CC00934BFB4F8420092
:2066C000B4F844008DF80C0000128DF80D00208D8DF80E00001205268DF80F00002013E071
:2066E00002280CBF05260926012818BF04F11C0104D1892006A902F00BFB06A9324603A842
:2067000051F070F894F826000DEB0601C8723A4603A831460AF0A4FA002840F08F80B9F19A
:20672000000F19D1BDF80A104FF6FE70884205DCBDF80A1088422FD1694615E0B4F8440006
:206740009DF80A608DF8200000128DF82100BDF80A008DF822601BE0B9F1020F09D0B9F1DE
:20676000030F19D104F1280108A851F0FFFA082012E0207CC00934BFB4F84200B4F84400C5
:206780008DF8200000128DF82100208D8DF8220000128DF8230004203E6881460BA98220A7
:2067A00002F0B6FA9DF82C10307B8142D8BF9DF82C00002842D0074600244FF0180A722002
:2067C00029460EF005FBB0689DF82C100019C8F80000007881422DDD296810FB0A10286007
:2067E0000146D8F800004278012A1FD083782BBBB9F1040F06D0091D08A851F09FFA012861
:2068000016D017E008884B888DF82800042208A98DF82A3000128DF8290018128DF82B003B
:206820000AA850F0A3FF012802D003E0807828B9002004E07F1E04F10304C0D1F3200CB010
:20684000BDE8F0872DE9FE4FDFF8E0810025804C98F86B048DF80050667801900FF062FDEF
:206860004FF0010B0BFA06F2DFF8C891744E4FF6FF718918014098F8FC02618138B3D8F81C
:20688000342322B342F21A0069469047684867790378B3B1AFB99DF8003093B1D8F85803ED
:2068A00078B1804707464946701C097800783FB16389083010FB01F0B7FBF0F15818608193
:2068C00067799DF80010608907FB01006081A078002840F09280607898F86B14574C012930
:2068E00066D155480068C06B804782460BF0E2F9074604F1900299F8000011780223800039
:2069000063F3030107FB00AC11707178C4F88CC0083189B200FB01C204F17401087863F38B
:206920000300087004F1CC032267187865F30300187098F86B04012836D10FF02FF998B37B
:206940004946226F486890422ED204F19002107865F30300107004F17403C4F88C50187817
:2069600020F00F0040F0030018700978707804F1780608308B0082B203FB02F0206730784B
:2069800004F178026BF3C300307010786BF3041010704FF4FA53A4F8865007FB01F0C4F89C
:2069A00080300EF019FB2AE01C2008F05FFF26E0A4F8AE5098F8191484F8B01098F80C74D0
:2069C00084F8B17094F8B21004F1B20241F0200184F8B210117804F1B20621F01F0141F0FB
:2069E00002011170317865F38711317084F8B35084F8B40084F8B55001E002F04DFE0198F2
:206A0000022810D10F481149007848B90E48007830B983220846027009F03CFFBDE8FE8FBF
:206A2000022208460270BDE8FE8FC0462008002045360020301E002048190020C81300206D
:206A4000141F0020493600204B3600204D3600200C1E00202DE9F84F7E4C074694F8610154
:206A6000002800F0E980B4F80E04B7F84210884240F0E28007F128000EF04AFA002800F000
:206A8000DB80002594F8110484F8615110B102200EF07CFD94F8070210B101200EF076FD65
:206AA000387C400905D310200EF070FD80200FF031FB20200DF0AAF904F5067009F0F6FC61
:206AC0007A685178107800EB0120C0F30321C0F3003684F85D11C0F3031384F8143400F050
:206AE0000F0184F85E6194F8370484F862110F2804D0884202DDD67806B9014684F8F51309
:206B000094F8F58384F83852B8F10F0F0AD194F85F01022840F090800DF0A6FC07F0E6FBFC
:206B2000BDE8F88F4C480078012802D00120FCF7C1FC4A48001D0068804783460EF098FB19
:206B40003E483F4B94F86BC48246426801789E6C3C48BCF1010F04D09E6D00F58A79034614
:206B600002E0034603F58A79B01A94F8F523890003EB820390FBF1F0D3F814110CF09CFF92
:206B8000CAF8046059F8280020630E4660630BF0FDFDA16A30460DF0CFFC0BF079FC2A489C
:206BA00081685846884794F85F01022810D1284809F07CFC94F8F50304EB4001B1F8242105
:206BC0004FF4707606FA00F12148891A0EF062FB94F814643889294609F036F8C4F85401C8
:206BE0000F2E14D094F8F51394F85D01B14208D0401C6FF00F07B0408101A1EB8005ED19D1
:206C000005E0401CB0408501A5EB8005A03DC4F85851022004F5A27584F85C01284609F0F4
:206C200045FC0A48C4F84C01D4F8581128460EF031FB10200FF06EFABDE8F88F301E0020BA
:206C400028190020687A01008C1A00209D070100280A002020080020CD1F00208C1A002019
:206C60002DE9FF470546DFF8FC81687898F86B14002840F0EB8095F89A20022A1CBF032AEC
:206C8000E82095F88F20802AC8BFE820012911D195F89010092901DB0A2900DDE82095F88B
:206CA00091700FB1042F05DB802FC0F2CE80882F80F2CB80002840F0C98098F83B0495F8E0
:206CC0009110884204D005F19101E820FDF760FC05F19001E720FDF75BFC05F18F01E12035
:206CE000FDF756FC05F19C015020FDF751FC95F89A0002280CD04FF6FE70A8F8080405F188
:206D0000920108F2FE3051F031F805F1920604E005F192063088A8F8080408F5FE7005F189
:206D200084010B2250F05EFD4FF001090220A5F816903146287501A80EF05EFE95F89E70A6
:206D4000B5F89CA0686805F19E01002FA0F1010068600CBF002048464F780FB140F002002A
:206D60008F780FB140F00400CF780FB140F008000F790FB140F040004F790FB140F08000E9
:206D800069684A1E6A6008702F7D69680024481C2862781E087028892C6598F8FC32AC65CA
:206DA000801C002B288141D0042785F86940E88A85F86B70C00934BF98F80D0498F8360410
:206DC00031460A2285F86A0005F1700050F00AFD95F89A00032829D105F1700005F1920141
:206DE00050F0C4FF98F8110400B31D4E306810F47F0F0CD085F82C70306805F12C014A4663
:206E000000F47F002863284601F050FD306810F0FF0F0BD02A2085F83C00306805F13C0179
:206E200000F0FF002864284606F060F900942846832101AA5346FBF771FC071C02D128466D
:206E400005F0DAFC381C01D106E0E82068701820287028460AF0C2FA0090BDE8FF87C046C6
:206E60004C7B0100200800202DE9F0411C4615468C4208BF854282BF00230022E5E0002C2B
:206E800008BF002D0AD100290EBF00286FF000006FF0000100F0E1F8BDE8F0815FF0000810
:206EA0005FF0000E002C08BF8D429CBF2C1C0025070C47EA01470E0CB44208BFBD429EBF2C
:206EC0005FEA044444EA15445FEA0545070A47EA01670E0AB44208BFBD429EBF5FEA0424BB
:206EE00044EA15645FEA0525470847EAC1774E08B44208BFBD4200F29380870847EA8177F1
:206F00008E08B44208BFBD427CD8C70847EA4177CE08B44208BFBD4266D8070947EA01778A
:206F20000E09B44208BFBD4250D8470947EAC1674E09B44208BFBD423AD8870947EA8167DF
:206F40008E09B44208BFBD4224D8C70947EA4167CE09B44208BFBD420DD8E60146EA5566EF
:206F6000EF01B14208BFB84201D3C01BB14158EB08085EEB0E0EA60146EA95664FEA85176D
:206F8000B14208BFB84201D3C01BB14158EB08084EEB0E0E660146EAD5666F01B14208BFF8
:206FA000B84201D3C01BB14158EB08084EEB0E0E260146EA15762F01B14208BFB84201D3F4
:206FC000C01BB14158EB08085EEB0E0EE60046EA5576EF00B14208BFB84201D3C01BB14107
:206FE00058EB08084EEB0E0EA60046EA9576AF00B14208BFB84201D3C01BB14158EB0808B1
:207000004EEB0E0E660046EAD5766F00B14208BFB84201D3C01BB14158EB08085EEB0E0EBE
:20702000A14208BFA84201D3401BA14158EB08085EEB0E0EA34208BFAA423EBF2D0A45EAF8
:207040000465240A89D3734642461E4617460B46024631463846BDE8F08170472DE9F04F8B
:20706000754C6068ADF12C0D002840F0E28004F178063068002800F0DC80DFF8C89109F14D
:2070800023000078022800F0D4806D4D281D006880470A90A06F074678B3684E4FF0000A99
:2070A0004FF01D083B7D0820711E11F8012F9A421ED0401EF9D164483946524650F088FA4D
:2070C000787E30F07F0005D194F88300401E84F8830004E094F88200401E84F8820087F80C
:2070E000018057F80CBC384608F068FD5F4602E0BA4657F80C7C002FD4D1352007F056FF4A
:20710000A9684E46002862D1452007F04FFFA968002856D1684601A909F0DEFD4A4800683F
:2071200038B1017D252904D050F80C0C0028F8D113E090B196F89801002838D00EF022FDCD
:2071400000280CBF04210D21009F96F82B02401AB8421FD8012086F89501152007F026FFBE
:20716000A968A8B10A98884760680DF10601703001F078F810BB96F82B020099884203D9A1
:207180001C2002F035F954E0002086F896010AE00A984DE0252007F009FFA9680A988847AB
:2071A000002086F895010420FEF7E2FC41E0252007F0FCFEA9680A988847192001F01EF98A
:2071C00037E00A98884708200BF0BAF931E00A98884796F8F401B8B10EF008F9B18901B9F0
:2071E000F1893269491E89B201EB81018918D1F801100FF018F942F21071814292BF0020F6
:207200006431081AC0B200E000206968002808BF0620D9D0C6F8D80188470446D6F8E01147
:20722000D6F8D80106F5F4720DF082F8A968204688470BB0BDE8F08F20080020B881010028
:207240008C1A002040110020980800202DE9F843784C714A7248734DDFF8CC81744E94F87B
:20726000E430591E0B2900F2C980DFE801F0954F6629466629466629C806106842F2107243
:2072800040F2AB27B0FBF2F15143401A874204D98020383D286000272F6067485F490026F8
:2072A0000125001D06600E200D6006F083F902200DF072F884F8E45084F8E360BDE8F88300
:2072C000042B07D001220A2B40F8252C14BF0221032104E02023012140F8253C0A4684F8FF
:2072E000E210002140F83D1C0827C0F8FB7FC0F8FF7F40F83D2CBDE8F883052B14BF092066
:207300000620002684F8E4002E607EE094F8E17001213C38002FC0F81B1004BF0621002244
:2073200002D00022EA62032184F8E410032140F8011C2A602868800867D294F8E40001268E
:2073400003281CD04FF08059D9F8A40140680027702204233946844600974046E047D9F8A2
:20736000A401C06870223946134684464046E04794F8E400062814BF0A200720C2E72B4881
:20738000006840680221702204230746009140460021B8470420B5E7116842F2107340F25B
:2073A000AB27B1FBF3F25A43891A8F4202D90821403D296001270F213038376042F62A2274
:2073C00040F8011C4FF08059C0F80320D9F8A40140680225072300214FF4C0728446404610
:2073E0000095E047D9F8A401C06800214FF4C072072384464046E047376004E0FEE700207C
:20740000306070600C2584F8E45004F178000FF002F8BDE8F883C0461C14005004800C404F
:207420003D400C4058600C4000A00C40A401001054600C403C15002038500C402DE9F04152
:2074400007460C467148DFF8DCC1DFF8CC81DFF8D0E1724902883846D12810DCD12879D0CA
:20746000713800F0B180401E00F0AB80401E00F0A480113810D04C3800F0868007E0D238C3
:2074800054D0401E41D0401E33D0401E28D038460EF0C6FDFF2802D1F420BDE8F0815C4D96
:2074A00005EB8005A97809B9E87850B1E878884208BFFB2000F0A7802278914269DC90426C
:2074C00067DB544E70688047074628786A7841464018214650F086F9B1683846884791E07E
:2074E0002278022A55DA0846641C00EB8200042285E021888A424CDDC8007746182200EB89
:20750000011039684018241D79E02678304602283FDA2C2505FB0680611C1022393050F041
:2075200061F9616905FB0680C1646BE02178607802292EDA02282CDA2C2200EB410602FBE0
:2075400001C3471C0CEB460C022283F8A4740CF2045030E02178608802291ADA824218DD49
:207560002C2303FB01C595F89C340CF26C429842A4BF431C85F89C3402EB8102D2F890102C
:2075800000EB40000322BDE720786778022800DA17B1E820BDE8F08161462C223D187E1CB2
:2075A00002FB001368000A2283F8946400EBC500401800F59D60A41C21E01CB308460822B2
:2075C0001DE0FCB1704692E7B4B90CF26C400CF264410CF2FC44022700F17C02983041F841
:2075E0002C2F54F8043B08617F1E02F10A0200F104008B60F3D105E040465822243021465C
:2076000050F0F0F80020BDE8F081C0460C1F0020E87A01008C1A00208C0C0020300D00207D
:207620002C0D0020200800202DE9F843DFF8C0810026054688F8A96298F86B24687D062812
:2076400003DBE82088F8A902687DA97D0E2905DD032803D0E82088F8A902687D032806D1DD
:20766000B8F8540040083CBFE82088F8A90295F8287017B1E82088F8A902012A12D1E87DFD
:20768000092801DB0A2802DDE82088F8A902287E08B1042806DB802801DB882802DBE82014
:2076A00088F8A90208F52A77294638460DF047F8291D112207F12C0050F094F895F82800BA
:2076C00008F52A74002804BF88F8F062A87D04D095F8290088F8F002688DA8F8E602687ECE
:2076E00088F8E802A87E88F8E902E87E822788F8EA02287F98F82B6488F8EB0298F83A34E3
:2077000088F8EC723B4F88F8ED6298F83B24C8F8CC72042688F8D06205F11D0188F8EE32B5
:2077200004F1490088F8EF220B2250F05BF898F8A902002855D16878002852D1287E98F8D0
:20774000AA728DF8000017B1EA2088F8A90205F11701E720FCF71CFF98F8F00228B1287E67
:20776000022808BF01208DF8000098F83B049DF80010884203D0E8206946FCF709FF1E4C45
:2077800098F8AA3298F86B94277867B9B8F80E041A490880EBB1032B17D0052B05D0012BA0
:2077A00003D0022B01D00EF01CFE0220207004F06FFE4FF6FF701249A8F80E04B9F1020F51
:2077C000088004BF0F49088005E004F061FE032000E0012020702720287030460DF0D6FE6C
:2077E00001E02A202870284609F0F8FDBDE8F883200800201561010064340020561D002040
:2078000092190020321500202DE9FE43DFF8C081704D0E46B00958D3444604F17C074DE0A3
:207820000178D0290EDBD02909D181783970C17879700179B97085687D60C168B9604FF068
:20784000DDFF48E004F15005286009F0C7FD28460BF0C8FE3FE0884794F88410491E84F875
:207860008410A9688847009801788DF8041020654378CBB1DC2B0DD0DD2B0BD0E42B09D07F
:20788000F32B07D0DE2B05D0DF2B03D0E82B18BFDB2B0BD104F044FF9DF80400162805D188
:2078A00068460BF09FFE01E009F098FD9DF80400162803D004F150000BF094FE38464FF0DA
:2078C000A5FE002869680090C5D1F00BA9464446C00305D0404F4FF097FD002800909FD150
:2078E000700905D32E208DF8040001A809F076FD700805D325208DF8040001A809F06EFD20
:20790000B00805D326208DF8040001A809F066FDF00805D327208DF8040001A809F05EFD66
:20792000300905D329208DF8040001A809F056FDF00908D300208DF805002D278DF80470A4
:2079400001A809F04BFD300A08D300208DF8050030278DF8047001A809F040FD700A08D3FA
:2079600000208DF8050035278DF8047001A809F035FDF00A08D300208DF8050023278DF8E6
:20798000047001A809F02AFDB00A08D300208DF8050036278DF8047001A809F01FFDE06C0B
:2079A000D9F8041080B18847E16C00270091D9F80810E7648847009804F15006306009F06E
:2079C0000DFD30460BF00EFE0020BDE8FE83C046200800208C1A0020FC1E00202DE9F04343
:2079E000894614460546ADF12C0D69460CF084FC5FEA000800F0C580AD1C0226284602A981
:207A00000AF0BFFF071C00F0BC809DF80900814509D0ED19BF1908F10200BF1CAD1CBEB235
:207A2000B042EBDCADE0401E05F1020500F08D80401E50D0801E33D0401E26D0401E20D0E7
:207A4000401E18BF622040F0AC80202F40F099802046294608224FF0C5FE083504F1080040
:207A6000082229464FF0BEFE05F1080704F11000082239464FF0B6FE07F108051834082251
:207A80000BE0022F7DD1022207E0202F79DC2046002120224FF0C2FE3A46204629467DE053
:207AA000042F6ED12046294602224FF09BFEAD1C15F8010BA070287800F00100E070287810
:207AC000C0F3400020712878C0F38000607128784011A07164E00B2F53DB0DF1120000219F
:207AE00016224FF09BFE2046294604224FF07AFE2D1D201D022229464FF074FE42F20B00BA
:207B000004A90BF0CBF8BDF81000A188884238DCA81C10F8011BA17110F8011BE17110F8B6
:207B2000011B217210F8011BC1F3C202A2720DF1120200F0F3F920B39DF82700A0819DF8B3
:207B40001670E78104F1100025E0052F19DB0DF11200002116224FF061FE15F8010B207055
:207B600015F8010B607015F8010BA07015F8011B0DF11202C1F3C2002071284600F0CEF98C
:207B800008B967200DE09DF82700E0809DF81670278104F10A0011220DF116014FF022FE2B
:207BA00000200BB0BDE8F0832DE9F04F8246ADF11C0D02F06DFA5D4800780BF095F85C4D47
:207BC0000024012808D90A380FD0801E04D0401E0ED0401E09D006E00DF074FF022804BF2E
:207BE00001210C1C06D0296806E005211F2401E003210724284601604E4AD068C0F3815032
:207C0000012804D112680120120E904004430EF051FADFF828B1DFF82081FF2240185B4609
:207C2000401E471CC8F800007F1E03F8012BFBD1DAF80020002702F0FF03FE2B1CD0D446F7
:207C40003B46012602F0FF05FF2D0ED0A84205D3A94203D806FA05F52C4201D0022062E057
:207C600002F0FF022F430BF802305CF8042F5B1C02F0FF05FE2DE7D1092005F0C5FD30483B
:207C8000C0F800A0374801210CF01EFF364D00264FF00109B04609FA06F0044214D107427D
:207CA00007BF06F0FF0141F4C0411BF806005AF82010244804F00CFBF0B24FF0FF310DF0C2
:207CC00067FDC5F8008001E0042028601A480068761C2D1D8642DED904A80EF0DBF91A4C6D
:207CE00020781B4A05901948102104AB0BF024FF68460EF0E7F96068174902901548CDF82B
:207D00000C806A460BF0CEFF144951F80D0C20F4F85040F4005041F80D0C114AC1F8FF9FBC
:207D20004046C2F8009007B0BDE8F08F46360020401F0020A84F00503C1F0020D83400208F
:207D4000AC300020007FC767488901008C350020AD570100C8330020093401000D300940E3
:207D60002C000940A8350020C0320020F8B507466848B0F854200021930804D2B7F89E30AA
:207D8000DB0828BFE82112F0600F04D1B7F89E20920828BFE821604E3B8906F108021288C6
:207DA0009A42B8BFE82197F89C5035B997F89850002D08BFF52100F0A880002940F0A580E7
:207DC000D7F8AC5090F8FC1215B9012903D026E0002900F0998097F89840002C18BF032CA6
:207DE00005D1D7F8AC5045F00A05C7F8AC5015F0FF0F07D02A21D7F8AC5087F83C1005F023
:207E0000FF01396415F47F0F07D00421D7F8AC5087F82C1005F47F01396390F8FC120024DD
:207E200049B397F89850426804216DB925223A754268D28AD20934BF90F80D0490F83604B5
:207E400087F86A00801C08E015233B75D28AD20934BF90F80D0490F8360487F86A0087F8E0
:207E60006B100A2207F1700087F8694007F190014FF0B8FC01E00120387597F8A050B7F872
:207E80009E00FD7697F8A130F8827A683B7797F82C103A622546BD650F293D650AD0B7F80C
:207EA000A80007F12C01224600B90122384600F0FDFC04462CBB97F83C00FF2801D1B86D30
:207EC00028B107F13C01384605F010F90446C4B9009597F89C10B7F89A3007F19002384600
:207EE000FAF71CFC041C0CD130893989884203DB384604F081FC04E0E5207870384607F024
:207F00005DFE211C01D1F8BD1821384607F042FBF8BDC04620080020081F00202DE9F04FB8
:207F2000154601F00708C1F3C2074FEAA119044683460C22ADF11C0D002168464FF06EFCF6
:207F40005FEA080034D0012879D101A8594603224FF048FCE41C14F8010B022200F00F002E
:207F600021468DF808000DF10A004FF03BFCBDF80A60A41C0721DDF804C052486E754268C8
:207F8000624507D1027A9DF808309A4202D14289B24206D0491E00F10C00F0D10020014649
:207FA00001E0017840788DF800108DF801001FE014F8013B07218DF8003014F8016B404870
:207FC0008DF8016010F80C2F9A4202D14278B24205D0491EF6D100200246114603E04268CC
:207FE000017A4089687501928DF80810ADF80A0003A806F071FC9DF800009DF80110B8F18F
:20800000000F10D0B8F1010F19D10198049A9DF814109DF80860424071408918BDF8160042
:20802000BDF80A2004E09DF80D309DF80C2059405040081803D1EF701FB1022F07D0002076
:208040003BE0281D214602224FF0CCFBA41CB9F1010F27D0B9F1020F2CD1BDF80A10281DF2
:20806000C91DCA1021464FF0BDFBBDF80A00C11D04EBE104F0B1401E811000EB5171C9105B
:20808000C9B249190E798210012700EB527222F00702801AC0B2401C07FA00F0FF30304000
:2080A000087107E0291D20460AF042FC207804EB8004641CA4EB0B04A0B207B0BDE8F08F26
:2080C000D8110020E41100202DE9F84F0F4680460DF025FB4FF6FF71814208BF682000F036
:2080E000B8805D4E440004EBC004A419D4F8026016B9D4F8065025B3D4F80610B14208BF56
:20810000692000F0A6806078401E13D0401E09D0801E16D13868864200F295808142C0F009
:2081200092800EE03888864200F28D808142C0F08A8006E03878864200F285808142C0F073
:208140008280464E7068804742F2020BDFF8109100904046A0EB0B0001282FD90A380128E9
:208160001CD9C01F49D1207862784D460021281800F5FE704FF052FB637838464FF050FBD9
:2081800005F5FE798342D8BF181C02DD38464FF047FB2178024601EB090034E00CF030FFEB
:2081A000B668398888424CDD207862784D463946281800F5FE704FF015FB28E00CF020FF54
:2081C0000546384629460AF087F8B6682D1A5FFA85FABAF1000F34D0207862784D4639466F
:2081E000281800F5FE704FF0FDFA5846404514BF85F89BA185F89AA109E0207862784D4651
:20820000281800F5FE7039464FF0ECFAB6680BF11900404504BF0020A5F884020BF11A0043
:20822000404513D1B5F88472B5F88202C119322901DC07430AD10220A5F882023027A5F893
:2082400084720098B0476A20BDE8F88F0098B0470020BDE8F88FC0464C8201008C1A00206D
:20826000401100202DE9F04F80465F4C98F80800A7780D46ADF1140D0228CDF80C8014D19E
:20828000012F12D004F57A71404602220C4620310DF012F838B903208DF8080004F11601E7
:2082A00068464FF063FDCDF80CD02FB3DFF848B198F808904D4CDBF8040014F809A080470A
:2082C0000A266427F8340490207A484505D15246204641460CF0F0FF20B1761E04F10C044C
:2082E000F2D103E00027EF72A07A2873DBF8081004988847002F73D03C49DDF80CA04FF08E
:20830000000864278B468E6DB1F84E0085F81E804446D9460AE0BAF80010761C2134B6B248
:2083200033E0B9F84E00641CB61DA4B2A04218DDF0780028F5D0B0880AF09CFB51460822CC
:208340000CF0BAFF0028ECD1F078A877308800046860B08885F80B80A5F81F00B0784746C7
:208360002873DBF85440002F3AD085F81E8042F219000DF10A010AF091FC0DF077F8814697
:208380001B480188642746468246B14228DDA07F0028C0D0B4F81F000AF06CFB0399082251
:2083A0000CF08AFF0028B6D1E07A022803D0E07A80B161270FE0BDF80A000E4A61684243CB
:2083C00048460DF0F7FD28B9A07F6C2740F00800A07700E047462846214621224FF002FA7C
:2083E000384605B0BDE8F08F20080020401100208C110020808D5B008C1A00202DE9FC412F
:20840000634C064694F8FC0294F86B84002798B1D4F8342382B1D4F8540368B142F21A000C
:2084200069469047D4F85403804728B19DF8000010B1E12E08BF0127B8F1010F04D194F885
:208440003B040CF045F801E00DF01CFFC07B02280CBF052501256068002800F09180002E0C
:2084600076D01B2E06D1017D052903D094F86A34002B6DD0E92E29D047BBE12E16D10DF080
:20848000BDFC90B16068C18AC9080FD294F81C14817694F80A144A1C84F80A244068817017
:2084A0002846FDF765FBBDE8FC8160681C2E50D1616A002951D088473249002009786060E5
:2084C00001295DD0FAF7F6FFBDE8FC81F1200DF0A0FA6768B87E48B90DF090FC20B160686D
:2084E000C18AC90835D2D1E7606832E0B8F1010F03D17868398907F001FD78680088000932
:2085000005D394F8FC0210B10CF030F86768F88AC00811D3387E00F07F003876387D032864
:2085200003D1787E40F004007876F0200DF071FAE168606888470FE013490126B87E0E70D1
:20854000401EB876F0200DF064FA10480078A8E70026467007F032FB6068C08A000A0AD3CC
:2085600094F8FC0218B994F82B040AF023FB94F92A040DF09DFC0020606010200DF0CAFDA8
:20858000BDE8FC81CD1F0020453600200E1E002020080020F8B5074661485F4C001DC26AE7
:2085A0000168B7F5C067C2F30722C4F8B870C1F38441C4F8BC20C069C4F8C010C0F38120A3
:2085C000C4F8D00000F0A38094F8D8606EB9C4F8D470D4F8C000C4F8C800D4F8BC60C4F85D
:2085E000C460D4F8D050C4F8CC50D4F8D400D4F8BC50002854BF02236FF0010304F1C80299
:20860000116800EB4000C018431000EB937001EBA0011160D4F8C810C4F8C45000291CDD09
:208620001E293DDDD4F8CC0030B93429B4BF15391E21C4F8C81025E02A29BABFD4F8C80002
:208640000B381E20C4F8C800D4F8C4003E28D4BF401C3F20C4F8C4001FE0D4F8CC0003288F
:2086600012D011F10A0FA6BFD4F8C8000B300120C4F8C800D4F8C4000028CCBF401E002063
:20868000C4F8C400032009E011F1140FA6BFD4F8C80015300120C4F8C8000020C4F8CC009E
:2086A0004FF08057D7F8A401B4F8C4101B4D40684FF47F4208230646009128463021B047DE
:2086C000D7F8A40101214FF40032112340680091064604212846B047D7F8A401B4F8C81054
:2086E00040684FF4F80212230646009104212846B047D7F8A401B4F8CC1040684FF4406270
:208700000A230446009120212846A047F8BD002084F8D800F8BDC0463C15002000A00C407A
:2087200000A00C402DE9FE4F9A469146884604460DF07DFEDFF86CB10CAFABF1350529688D
:208740000290A14208BF69680DF1050042464B460090204600F08EFB061C11D195F83400BC
:2087600040F0040085F834000298AC620DF04EFF9DF80500022873D16FF00200BDE8FE8F87
:2087800004F178000DF049FEC6F80880464899F80430F460B18D86F82E30143001803E48D6
:2087A000C6F804A097E80C00202100271940B846104086F82F7006F1100383E8030006F131
:2087C000180282E8800199F80500012805D196F82F0040F0100086F82F0002980DF016FFA9
:2087E00095F83500042806D1E86AB5F9301095F832200DF0A8FD0DF01AFE804695F8350056
:2088000002280BD196F82F0040F0800086F82F0084F8C27040460DF0F9FE39E01F4D012862
:2088200012D11F480DF0F9FD96F82F0040F0800086F82F00686884F8C2700028EAD14046FA
:208840000DF0E4FE5846007830F004001ED12846314601AA0AF06EFA30B940460DF0D6FEDE
:208860006FF00100BDE8FE8FB08DA4F8C0009DF8045096F82F0040F0800086F82F00012D9C
:2088800084F8C270C6D140460DF0C0FE0DF05EFAB6F92C00BDE8FE8FFDEFFF9FC43500204D
:2088A000B4340020C5330020C43500202DE9FE4F07461046002F00910CBFE8210021019132
:2088C0000099002900F0AC800199002940F0AA8060B17868401E7860F82101707868401EAE
:2088E0007860002606703889801C3881DFF83C81009C4FF000094FF0020BCDF80890C246C5
:20890000083C14F8080F00F00F010F2900F08580012821D004287AD19AF8FC02002876D034
:20892000DAF8141360688847061C26D03889B7F84C108019801C81421FDB7868DAF818C344
:208940006168029B3A46801BE047B0B178683989801B8919786059E0009A029804254A4433
:20896000D21C12F8011FFF2941D021293DD13989B7F84C300B318B4202DA1A20BDE8FE8F10
:208980007968B8F82434491E79601B120B707968491E796098F824340B707968491E796061
:2089A000029E0E7098F826147B68197098F8223479681B01491E796043F00F030B7098F8F0
:2089C00014C498F8F5337968491E796043EA0C130B707968491E796021260E707968C01D7B
:2089E00080B2491E796005260E706D1EB9D17968C0F30122491E796042F088020A70796839
:208A0000491E7960087039890918891C3981BBF1010B09F108097FF474AF7868B86501E025
:208A2000E82001900198BDE8FE8FC046200800202DE9F0470446880FC0F0A38000200AF069
:208A400069F851480DF0E8FB504A002140F60A00108002F10C0551802B7802F10D0661F3DF
:208A600003032B704A4B516035784FF0010A6AF3030535701F78A6688C460D46718007B993
:208A80005546637C1D4318BFD446338891466546A3F602076FB141F21E02BF1A09D006F110
:208AA00019031A7861F382021A707DB106F1180208E006F111031A7861F382021A702DB1A2
:208AC00006F11002138861F309131380C21F6174354602F1010800E03D466F6837B13B88DD
:208AE000984203D09A4218BF9845F5D1C5F8049005F10D03187861F30300187025480DF043
:208B0000A6FC8068008882421CD04246824219D0278DCFB104F12800E16204F134034180DD
:208B20001A78353461F303021A7022786AF30302227009F10D07C9F80400387861F30300EF
:208B4000387001E0144801601448007880B914480068006801465046884701280ED00D35A1
:208B600028786AF3030028700E480DF055FB05E00AF0A2FE0028FBD00AF0BEFE30460DF01F
:208B8000D9FABDE8F087C0460D2E00000436002041360020C43500200035002011350020E0
:208BA000E0010010912601002DE9FE4F4D48DFF84481476890F86B1490F8FC22002F51D0CC
:208BC000494C4A4FDFF828A1012A11D0606880473F7847B95246A16817782FB9832342462F
:208BE0001370884767E0A1680223424613706EE0012981460BD199F83B040BF069FCC07B1D
:208C0000022804D14148C01C007806F033F90BF0E1FC394D286A394E016CF0688847834682
:208C2000606880473F780290002F47D150460078002843D1D9F8481300208847F42001A9F2
:208C40000AF09EFB2E4F9DF9040058451ADCBB79C3B9A16802988847D9F84863B878BC79D4
:208C6000042801D00DF0BDFB04214046641C0170E0B2B8710EB10320B0470320788100F006
:208C80000BFD25E0832140462A6A0170536CF0686A4600219847B5F90600BDF9001088428D
:208CA00014BF0020012009F047FDA16802988847387A1449087007F0EDFD09E002214046F7
:208CC0000170A16802988847D9F84813042088470D480078012802D00020FAF7EBFBBDE82E
:208CE000FE8FC046200800208C1A0020493600204B3600204D360020281900204C1D002006
:208D00000C1E0020171F0020CD1F00200E1E00202DE9F041074651480C460188384671382C
:208D2000022840F29880133828D0514A4C387CD0401E65D0401E4FD0DFF82C81401E3BD014
:208D4000DFF828C1401E2BD0401E1AD038460DF067F90646FF2E11D0414D68688047414ACD
:208D60000746B000115C801842784346C91820464EF038FDA968384688470EE0F420BDE8EF
:208D8000F0812178022966DA6046641C0422001D00EB810120464EF025FD0020BDE8F0818C
:208DA0002088814257DDC100674601EB001138681822241D0918EDE72678022E4BDA2C2555
:208DC000601C05FB0681102239314EF00BFD05FB0680C06C6061E0E72378022B3BDA6078BF
:208DE00002F26C412C2505FB032292F8A424824231DD00EB430001EB40010222983128E0E8
:208E00002378022B27DA618802F26C402C2505FB032292F89C248A421DDD00EB8300D0F844
:208E2000900001EB41010322C3E72178022912DA607802F26C432C2505FB012292F89424C4
:208E4000824208DD401841000A2201EBC001C9187C31A41C9EE7E820BDE8F0810C1F0020BB
:208E60008C1A0020E87A01008C0C00202C0D0020200800202DE9FE4F554E04468A4690467A
:208E8000002006F1350108700C9A0192834682F800B00CF05DF90093071C08BF012000F001
:208EA0008A804C4DB16AB5F914008C4200F101006FF31F30B88507D196F83400410824BFBE
:208EC00000F0FE0086F834001846006800B95846B86298F80C0000F00F00022814BF584685
:208EE000D8F80800BAF1000F78626DD00AF19C000DF0C8F800285DD1204629460BF072FDE0
:208F0000041C0DD12B685BB169682A68384605F09BFB28B1012386F83530286838602F60B1
:208F200096F83590B9F1000F4ED10CB92C6894B122683846214605F087FB18B92468002CF9
:208F4000F6D108E00221206886F835103346386093F835902760B9F1000F35D1009801793B
:208F6000504603F005FB014601292AD096F83500002829D1012927D0296809B10868F0B993
:208F800098F80C0000F00F0002281DD198F80C00C011400818D241B96868A8B1696838460D
:208FA0005A4605F051FB28B10EE038465A4605F04BFB48B9022001995F46087004E0096881
:208FC000DCE7042086F835003846BDE8FE8FC04690330020C43500202DE9F843554C676884
:208FE0004FF0FF300CF01EFF002F00F09980DFF83C81010925D2810801D3E6680EB307F1B9
:20900000100191E86000002105EA00020E4008BF002A00F085803A6A284007F118061043AB
:2090200096E80C0007F118053862386AA7601943104385E8030040464FF480410DF013FA9B
:209040006EE039693E6A07F1180595E80C0041F00A0108403043364D3862386A00211943A7
:20906000002610433A69666007F1180383E80300286807F110039043286093E80300083DD4
:2090800028683246091C88433946286004F11000814609F04FFE404602210DF0E4F9E068F4
:2090A00000283DD0E068F968C068884238D1E06890F82F1097F82F00084310F0070015D0D3
:2090C000410806D2810804D2E16891F82F20104304E0E16891F82F0040F0010081F82F00DE
:2090E000E1683246484609F025FE18E0E0686060E0680069C0436860E0680069A96808437C
:20910000A860E068103003C8081CC04345F8040CE068103003C82F68081C38432860E66029
:2091200009F0C6FE05F08CF8BDE8F883FC33002014100440C43500202DE9FF41044666689B
:20914000A7680D460DF073F93178012903D10DF05DFA00208DE0012131700DF057FA28780B
:2091600070706878B07068687060A868B060E868F06028693061287D3075687D7075A87D54
:20918000B075A869B061287F3077687F4FF000087077A87FC6F82080C6F83080B077454680
:2091A00075627563B562B56386F82C5086F82D50786804F029FB204604F07CFE204604F0B6
:2091C00085FB78B92C480068C068014638688847786804F0EFF90DF02AF935700DF016FA96
:2091E0002C4645E068460CF055FF3A7B06F17C00B9680192214A00946B460AF09DFC68460D
:209200000CF060FF396902911D49009406F198006A460AF047FDB07830B906F1CC00294604
:209220000BF052FC17483061707830B906F1E80029460BF049FC1448F06068460DF09BF8AC
:2092400001958DF8005006F58270104902940A226B4609F0E9FEB969FA6906F13C000CF056
:20926000CDFE0B4A06F16800042123460BF000FE20460090BDE8FF81D0010010299E000025
:20928000E13C0100676301005F630100D5FC0000756101002DE9F04F06464FF00108ADF1F3
:2092A000640D0922B07D8DF84C8006F117018DF84D000DF14E004EF095FA4B4D686880476B
:2092C000179016A98120FFF723FD707D002840D09DF85800022817DA042000238DF8030075
:2092E000347D8DF802809DF858708DF8013069468DF80040781C8DF85800D220FEF79EF841
:20930000812016A9FEF79AF8DFF8E0A000274FF0FF0B3C46B94618E0307D69460DEB800052
:20932000C0F81090D420FEF789F801E08DF824B08DF82670307D8DF8257008A98DF82000F9
:20934000D120FEF77BF8641CE4B2BAF80000A0422ADC307D00279DF84D208DF840000DF16B
:209360004E018DF841700DF142004EF03BFA8DF84B80D02010A9FEF761F8071C0FD1307DBE
:20938000314610228DF828000DF129004EF02AFA30690AA90F90D320FEF750F80746A96875
:2093A00017988847F8B21CE0307DADF8224008A980F001008DF82000D120FFF7A9FC00285A
:2093C000B4D19DF82400FF28B0D0ADF800006946D420FFF79DFC00289ED0A96817988847AC
:2093E000192019B0BDE8F08F8C1A00200C1F00202DE9F843504C80466068002800F099808A
:20940000DFF83891B8F1000F18BFB8F1E90F17D14D46AE892F690CF019F806EB8606F61999
:20942000C6F80100A88995F8F521014601EB81017A54E989401C80B28142D8BF0020A88173
:209440003F4D6868B8F11C0F37D0B8F1000F0BD099F82300032807D1B8F1E10F04D00020FE
:2094600089F8F201072000E0052009F069F8676899F8230003280FD077B10020FE8A87F816
:209480006900F00934BF94F80D0494F8360487F86A004046FEF7B2FF99F89701012848D194
:2094A00068688047044608F03BF8A96820468847002089F89701BDE8F88380470646616825
:2094C0002048C98A0078C90804D294F88310814204DB28E094F88210814224DA616804F14C
:2094E00078004EF053F96068C08AC00805D294F88300401C84F8830004E094F88200401C01
:2095000084F88200A968304688476068007D252819BF012089F89601012089F895010020FC
:209520006060BDE8F883A96830468847F120FEF765FFBDE8F883C0462008002040110020AC
:209540008C1A0020081F00202DE9F04FFF25ADF1140D8DF800504FF6FF79ADF80290ADF858
:2095600004900AF0CDFDDFF82CB104900BF1020000880027001F84B2082C64DBC84646463C
:20958000C246201F02A9082280B24EF015FABDF80800814508D1BDF80A10894506D1BDF8AB
:2095A0000C20924502D107E0BDF80A1051EA000314D1BDF80C308BB9BDF80E00C10BCB036A
:2095C0000AD100F108018C4238DA4EF027FA04980CF032F9002058E0241F31E0C20BD30365
:2095E0002AD1C20B28D3BDF80C3000F0FF02954203D1884508BF9E421ED0C5B28DF800506D
:209600008846ADF802801E46ADF804609DE80600384607F077FE78B9BDF80E20A01A07F1AD
:209620008851001F083280B292B24EF0C5F9BDF80E00C019083087B2BDF80E00241A083C34
:20964000A4B2082C9DDA09F023FF3FB110484FF088513A464EF0D0F90CF07AFC04980CF0FD
:20966000EBF859464E78002E1CBF0020021C0BD104204FF40052C0EA0740C2EA0742A2FA44
:2096800040F01FFAA0F280B24A8005B0BDE8F08F04400500241F0020F8B5504C4C4E4D4AF4
:2096A00094F86B3470897178012B6AD102F174031978002565F30301197002F1CC031567F3
:2096C000197802F1780765F3030119703B78012161F3C3033B7002F178073B7861F3041378
:2096E0003B704FF4FA57C2F8807008B9718108463B493C4F491C94F8FC320978083148430D
:209700003978002B01FB00F0009036D0D4F83C23002A32D0D4F8400300282ED006F108015F
:20972000684690477179737862682B4E65281AD0A8B9107D052820D194F81104E8B96068FF
:2097400090F82C00211D042817D10968D4F81843906D096B2B46A04778B91A2000E03570B2
:20976000FEF74CFEF8BD82F8691082F86A30D4F8401335701C208847F8BD00980BF02CFCAF
:20978000F8BD002394F81904A2F8AE3094F80C7482F8B00002F1B20682F8B170307802F1B9
:2097A000B20563F345103070287802F1B20720F01F0040F001002870387863F3871038701E
:2097C00082F8B41082F8B33082F8B530F8BDC0460C1E0020C81300204D36002020080020A4
:2097E000141F0020301E00202DE9F04705466C78ADF1180D002C40F08B804A48B5F89A1019
:209800000088884218BFE82405F1900101A888460CF0F2F8444E01A80BF07AFB30B995F80E
:209820009D0030B1707820B9E82471E0002085F89D00002C6CD195F89D0000280CBF0120AB
:20984000052004272F754146E8820DF10E000CF0D3F8686895F89C40401E6860411E6960C9
:20986000B5F89A9004702B7D69680024481C2862581E087028892C6596F8FC22AC65801C89
:20988000002A288136D085F86B7005F1700041460A224DF0A7FF95F8980005F1700A0328DB
:2098A00028D105F1900150464EF060FA96F8110400B31E4E306810F47F0F0CD085F82C7019
:2098C000306805F12C01012200F47F0028632846FEF7ECFF306810F0FF0F0BD02A2085F816
:2098E0003C00306805F13C0100F0FF002864284603F0FCFB0094284603210DF10E024B46C9
:20990000F8F70CFF041C02D1284602F075FF2CB16C701A202870284607F060FD06B0BDE8DE
:20992000F087C0462E0C002020080020547B01002DE9F04705464B4890F8009028798028AC
:20994000D4BF0020E820494C0027B9F1010F0DD16979092901DB0A2900DDE820A97909B114
:20996000042903DB80297ADB882978DA002876D194F8F5030F2872D0B4F80E144FF6FF70ED
:2099800088426CD0B4F80814884268D0E87901280BD040B1FF2862D194F85F0100285ED104
:2099A0000126374602E0012600E0022604F50670824606F07BFD04F5027006F077FD04F57F
:2099C000A27006F073FDDFF8A88008F104000068804784F85F6166680246FF210020C4F896
:2099E0005801002E84F85C110CBF0121011C84F86111012F84F8607108BF032084F83802E2
:209A00004046816810468847A91DE820FAF7C0FD691DE720FAF7BCFD291DE120FAF7B8FD12
:209A200094F86101012802D120200CF063FB0E48B9F1010FC4F8200207D094F8F5134FF406
:209A40007070884000F2564106E094F8F5134FF47070884000F2636150460BF06BFFBDE81A
:209A6000F087C0468B0C0020B5140100200800208C1A00202DE9F0474E4C4B496FF00100FF
:209A8000383CA76B087027B994F8F5030F2840F089804648DFF818810121002F814601706D
:209AA00072D0206B7968884221DB0AF0B5FB7968884267D394F8F503A56B0F2812D1002DC8
:209AC00062D00AF0A9FB696888425DD3A66B706800280CD4304606F0E9FCB168307B884716
:209AE000A56BECE7002D4FD06E68002E01D50CF078FCAA462F7BAD680AF08EFBB0420DD2EA
:209B0000A06B30B1216B4068814202DD09F0B4FF3AE00BF0ADFB0020A06335E03846A84775
:209B20004646301D006880475546824604F1280128460BF0D7FD20B904F12C0128460BF0FB
:209B4000D1FDA06BA84218D10027A06AA76387420BD0216B4068814207DD0AF05DFBA76A3C
:209B600079688842C8BF7860A763E56A2DB11FB178686968884200DDA563B16850468847F6
:209B8000A56BAFE708F084FC464670688047044603F042F8B168204688470BF0BDFE0020E1
:209BA00089F80000BDE8F087ED1E0020CD1F00208C1A0020580800202DE9F8434A4D4B4C0C
:209BC000686894F86B8480478146A9686068002840F08680E0698047A76F40F01000002FE0
:209BE0007DD00022797E0140884205D03A4657F80C7C002FF6D172E004F1780039464DF057
:209C0000E7FCB8F1020F02D1384604F0AFF9002F65D06760787E30F07F0005D194F8830015
:209C2000401E84F8830004E094F88200401E84F88200A9684846884761680889C98A06F068
:209C400003F8B8F1010FA4F8800004D194F83B040AF03EFC01E00CF015FB05466068C18A15
:209C6000090A08D3C07E08F0A5FF606890F91C000CF01EF96068B8F1020F04D1C18AB4F84E
:209C80008070490A10D2E97B012906D0022929D10520FBF76DFFBDE8F883007E401080F035
:209CA000010000F00100F4E797B190F86C607EB196FBF7F10E4F068980F86D10791C0A789B
:209CC000122ED4BF0C21282191FBF2F1C9B202E0012180F86D1080F86E100620D9E7A9686B
:209CE00048468847BDE8F8838C1A002020080020141F00202DE9F04F994692460C46804662
:209D0000ADF13C0D0BF062FB444D3C2205F1100108600021684606F03DFE20686E463060DA
:209D20006068706020893081207A032804D0022003248DF80C0002E003248DF80C40287844
:209D400018B105F134000CF07DF9A88EADF80A0068781E28D4BF411C00210027B8F1050F9E
:209D6000697040F080000BD0B8F1040F05D0B8F1020F08BF40F0600004E040F0200001E0C8
:209D800040F040008DF80D00ADF828A04FF0010BCDF8249022498DF80EB00A680BA802605B
:209DA0004968416005238DF83540B8F1050F8DF83640B5F858008DF8343012D0B5F85E009C
:209DC000B8F1040F08D0B8F1020F0ED1B5F86400401CA5F8640008E0401C80B2A5F85E0077
:209DE00003E0401C80B2A5F858000E4918206A464CF0FAF9C0B258B1B8F1050F09D1E86A2B
:209E00000AF030FDB5F85800401CA5F8580000E05F4638460FB0BDE8F08FC0465C18002045
:209E20004D850100D14A00002DE9F0478046D8F808603068076CD8F8045047646A6CA96B25
:209E4000286C17F4F06FA0EB020935D1F8091ED278096AD3B1B196F821003E4A145C601E32
:209E6000814294BF0C1C641E404621460AF0F0F9A86B001BA863A86B002856D105F1980029
:209E80000CF0F3FA404649460AF0BEFB4DE00029F8D040460AF0DCF9014695F82D00A96391
:209EA00018B9A86B002840D101E00020A86305F198000CF0DAFA38E0F80A1AD24FF00009CD
:209EC0004C4603E0A86B401EA863A96B49B3404601210AF0BDF93068446814F00F04C0F816
:209EE0000490EFD0296B686B491E2963401E686317E0306844680022202904F00F0442603D
:209F0000CCBF4FF0200A8A46404651460AF0A0F9CAF120008145C8BF8146494640460AF0CF
:209F200073FBEC77404607F0FFFBB80910D3AF6A77B1404639460AF0C3F9A862AD6A3DB922
:209F400096F820000449095C4046C91908F0FCFFBDE8F087608901006C890100F0B5494D0F
:209F6000014695F807020027ADF1140D002855D195F8EA03002851D0087ACF68C0F3021689
:209F800000F0070100E0BF1C0846411EC9B248B17A783878B5F8124400EB0220A042F2D196
:209FA00002270FE005F57A74443400E008373046411ECEB2A0B3204639464DF0BFFE00285B
:209FC000F4D0032795F8070240F0040085F8070202A80AF0B1FF01200BF0D8FA05F5FE7198
:209FE0008720FEF795FE05F501718520FEF790FE05F205218620FEF78BFE05F20621882097
:20A00000FEF786FE0120009005F5FE760196B5F80E34394602AA0520FCF700FA002F2ED1B7
:20A0200095F8F5030F282AD095F81414814226D095F8110418BB95F8560000BB1248007817
:20A04000012802D00120F9F735FA104C6068804795F85F11022910D195F85C11FF290CD0D3
:20A06000696851B9A96F41B9A168884705F5A27006F01CFA06F092FB01E0A168884705B012
:20A08000F0BDC04620080020CD1F00208C1A00202DE9FF47494C94F8E700002879D10125F7
:20A0A0003E4E84F8E750307B84F8E6007768C4F8107101A80CF05FF9002704F10C0002977A
:20A0C00001AB8DF80470364903973A4608F0ACFF344904F1300001AB3A4608F0A5FF3249BA
:20A0E00004F1540801AB3A46404608F09DFFB0680146284688472D48DFF8B4900078767B34
:20A10000D9F80400C0F3815A26B1BAF1030F04D184F8E150BAF1030F20D0BAF1020F1DD070
:20A12000BAF1010F2ED14FF08058D8F8A401214C406803214FF040521C2306460091394634
:20A140002046B047D8F8A401406839464FF400720923064600952046B04713E002200AF0D8
:20A1600051FBBAF1030F0CBF4FF47A7142F2107111480068B1FBF0F140460CF04AF940468F
:20A180000CF049F9D9F80000C00802D238460AF039FB00200090BDE8FF87C046D48801002A
:20A1A0000BDB000085FF00004DF7000046360020B04F005000A00C40303600203C15002023
:20A1C000F0B5477EADF1140D37F07F0700F08A80017D012918BF032940F0848042490988B4
:20A1E00001F0020201F0080111437BD041684878C0F38102022A8DF8082006D0032A10D175
:20A20000491D68464DF0B2FD09E08A79487940EA0220ADF80000C8780A7940EA02209DF8FC
:20A2200008200446022A18BF032A19D16846214606F078F8FF284ED19DF8080002460BF0F1
:20A2400041FE0026012505FA06F1084202D0761C052EF8DB052E09D1022A18BF032A05D1B6
:20A260000BF0D6FDFF283DD1012039E01F48022A06D004466946082204EBC600903012E0AE
:20A28000BDF800108DF80C40271204468DF80A1004228DF80D7004EB8600091274308DF825
:20A2A0000B100DF10A014DF09DFA9DF808102046022914BFD0F88C30036F05FA06F202297D
:20A2C00043EA020314BFC0F88C3003670A463046294609F0B1FB0BF09BFDFE2802D1002015
:20A2E0000BF0E4F805B0F0BD740800202819002030B5ADF1140DFFF7CBFE3049314A086861
:20A3000040F0020008602E48026068460BF0DAFE2D4DA8782E4902902C486A4609F0C2FCCC
:20A3200068460BF0B7FE28782B4A002419216B46019028488DF8084009F0FEFB68460BF032
:20A34000C1FEE8780290264924486A4609F0AAFC68460BF09FFE01206B788DF808001A2110
:20A36000214A204801936B4609F0E6FB1F4820492246134608F058FE1E481F4A04212346AF
:20A380000AF076FD234804701C4A1470072554701B4B94701B491D701D480C7005250560CC
:20A3A0001A4A1460184D1C492C704FF4FA728A601A48CA600BF030FF05B030BD0020094005
:20A3C000CC210840110000E07E890100FC330020ED550100543500209519010030340020E1
:20A3E00041DD00007035002099010100B434002075510100DC350020C52A01004036002059
:20A40000883300201135002012350020003500200C350020F834002090330020A9B3000053
:20A420002DE9F8430446080B7CD3474804273E49077001250D7038460AF0E4F93B4E30684E
:20A44000016AC90804D3C16900220B46394698473748384900220BF0F0FF37480BF0DCFE8E
:20A4600030684168886808B9C86810B133480BF061FE284608F04EFBD4F808900021A9F84F
:20A480000210A0680288A2F602072FB141F21E02BF1A18BF183000D11030038840F60A066A
:20A4A000F21F61F3091302F1010803804B46657400E03B465F6837B13888864203D0824203
:20A4C00018BF8045F5D103F10D065960307865F3030030701A480BF0BAFF8068008882426D
:20A4E0001BD04246824218D0208DC0B104F12800E16204F1340641803278353461F3030263
:20A500003270227865F30302227003F10D075860387861F30300387001E00A48016048467F
:20A520000BF008FEBDE8F88312350020FC34002054350020ED5401000D2E000051000706BF
:20A54000C435002004350020403600202DE9FE4F0AF08CFF434C04F1280202901168E06210
:20A560004FF40050491C1160694608F097FBDFF8FCA0DFF8FC90B4F8520000285FD0A66DFB
:20A58000B4F84E0000254FF6FF7BA0462F4654E0B07F800822D3B6F81F0008F06BFA014631
:20A5A000082268460AF088FEC0B1716802982E4A0BF000FD90B9B6F81F00B77709F0DCF8DE
:20A5C000A6F81FB0DAF800008047B4F8503013B15B1EA4F85030D9F808108847B8F84C003C
:20A5E0006D1C2136ADB235E0F078800821D3B08808F040FA0146082268460AF05DFEC0B1D4
:20A6000030880104184A02980BF0D4FC88B9B088F77009F0B1F8A6F804B0DAF80000804749
:20A62000B4F8523013B15B1EA4F85230D9F808108847B8F84E006D1CADB2A842D4DCB4F8AD
:20A64000500048B1A046666DB8F84C0000254FF6FF7B2F46A8429BDC04F1300008F0BAF972
:20A66000BDE8FE8F4011002000A493D6901A00208C1A00202DE9F041394A43483949167835
:20A680000778ADF1180D002E60D04048067836F07F065BD1C88A344D012F00F10100C882FE
:20A6A00009D000248DF80C4002948DF80D4005F144002C6404E0002405F1CC00C5F8C8400B
:20A6C00001782A4E2A4B64F303010170012030701978012901D0F8F7EDFE012F01D10AF025
:20A6E00045FF2B48001D006880478046294B2A48DFF880C006681868012F05D005F1380172
:20A70000082302AA4C8008E0049402238DF8154005F1C0018DF8143004AA8DE81800346DBB
:20A720006346A04714490880144900280AD4144A92F90000401C10701248012F14BF3835B2
:20A74000C035C56089684046884706E0088B401C0883002010700BF0C3F806B0BDE8F08117
:20A760004B3600200C1E0020C8130020EF1E0020CD1F002029F60000B41C00208C1A0020E5
:20A78000F61E0020281900208B0C00204D3600208C1A0020581D002048190020B0B504463F
:20A7A00045480078002800F0828094F88F00002871D13520207504F19101112204F17000EC
:20A7C0004DF010F804F13C00FF2110224DF026F804F12C000F2110224DF020F894F8900062
:20A7E00004F13C0500283ED0401E29D0401E14D0401E5AD12A20287002272764042305F811
:20A80000103C4FF410222263032184F86B10204607F01EFA071C3BD137E02A200A27287009
:20A82000042327644FF44C1205F8103C02212263204684F86B1007F00BFA071C28D124E05B
:20A840002A2002272870042327644FF4102205F8103C01212263204684F86B1007F0F8F991
:20A86000071C15D111E02A2002272870042327644FF4502205F8103C00212263204684F89B
:20A880006B1007F0E5F9071C02D1204601F0B4FF381C0DD1B0BD01280CD10848D0F80C039C
:20A8A0008047002808BF002002D0192000E018200BF01CFBB0BDC0461C0B0020200800208B
:20A8C0002DE9FC4706467568D6F80880A86B002818BF4FF0FF307ED129630024EC77171C8B
:20A8E0006C631BD005F13C090BF0A1FD82466946484609F021F8002820D450460BF086FE82
:20A900009DF80000296B0870686B296B7F1E00F10100686301F101012963E5D169786A6BE9
:20A92000286B0129A0EB0200286305D1E868296B0346304698476A6B14464BE0AF635046E8
:20A940000BF064FE0BF073FD244E0746307820B9022009F057FF0120307038460BF056FEF0
:20A96000D8F80010086B40F400700863D8F80010886B40F4FA608863687808BB696805F1BF
:20A98000E80738460BF043FBB8B1AC63384621460BF03DFB88B10BF04AFD0746307818B148
:20A9A000022009F0F9FC347038460BF02FFE1022696B286BEA77401A2863686BBDE8FC8763
:20A9C00095F82D0030B1686B20B1AC6305F198000BF04BFD2046BDE8FC87C046433600202B
:20A9E00070B50546434C2878ADF1200D002858D1B4F8400004F150066B88ADF80000314656
:20AA0000ADF81030E2200BF015FB0DF1120031464DF03DF9698853200BF024F8B4F84000E3
:20AA200004F146063146ADF80E004A200BF002FB01A831464DF02BF900268DF80D60B4F804
:20AA40004400ADF8020094F842308DF80C30304609F020FF522031460AF0F8FF94F8580000
:20AA60000F2807D00120A070B4F8441020704B200AF0F8FF606928B102681AB10DF10E00C8
:20AA800069469047032006F0EBFE94F85A00032818BF042827D104F10A0010214DF0D2F8EB
:20AAA00021E0154E01280FD002280DD00020A0700BF058FA41F2883009F0ECFEB6F85600D4
:20AAC000401CA6F856000EE005200BF04BFA062006F0C6FEB6F856000021401CA6F856007E
:20AAE00052200AF0B3FFA16E09B12846884708B070BDC046E01900205C180020FEB506469B
:20AB0000434C3178B4F86800E1292FD0B4F86A00E92926D0B4F86C00D9B93E4D30696F6A1B
:20AB200002903FB37F692FB3A96A1931814221D806208DF800000422ADF802200023ADF84E
:20AB400004309DE8030002ABB84708B90298A86210E0401C80B2A4F86C002AA00BF035FCAC
:20AB600008E0401C80B2A4F86A0003E0401C80B2A4F86800717831F07F0042D001F06000F8
:20AB800040282AD1307840BBB4F85A002569401CA4F85A000AF01AFC854203D80AF016FC0B
:20ABA000401B03E00AF012FC401B401EB4F8827080B26421B0FBF1F080B2B842A8BFA4F886
:20ABC0008200B4F85A10B4F880304A1E02FB0300B0FBF1F0A4F88000717801F060012029ED
:20ABE00006D1307820B9B4F86000401CA4F86000602906D1307820B9B4F86600401CA4F8AE
:20AC00006600FEBD64617461436E663A2000C0465C180020581700202DE9F84F05464248AD
:20AC2000DFF80C81814646192D3698F8FC0234780F46C0B1D8F81413A9B109EB850ADAF881
:20AC4000DC0000F0FF0088478346D8F81413DAF8DC0000F47F008847584480B218B131786A
:20AC60000818001DC4B298F8200401280AD1387A40B148447B7A067919F803002418641DF5
:20AC8000E4B200E000260D2D19D0A01900F1020A50464CF039FD071C19D102204CF034FD9B
:20ACA000011C09D04D4495F8490008701A274F7098F800004CF01EFC0020BDE8F88FA719CD
:20ACC000F82F01DD0BF08DFB07F1020A174F3846002152464CF0A2FD07F10C0000217822B1
:20ACE0004CF09CFD07F13C00FF2110224CF096FD07F12C000F2110224CF090FD38197860B2
:20AD0000022D3E810BDB0B2D09DA7868401E78606D1E05703889641EE4B2401C3881A7F8A1
:20AD20004C403846BDE8F88F687A0100B02F0020200800202DE9F04F09AF9A46164688469C
:20AD4000ADF1440D3C893D88D7F8049010900020AC428DF83C0001DACA4501D30BF041FBB3
:20AD6000002E6BD03748875D042EA4EB07044FF00000A4B2B8BF01205FEA000B0EBF2D1BA5
:20AD8000A1440024314807A90823ED1B2530ADB210F801295B1E01F8012BF9D14FEA18604F
:20ADA00001F8010B4FEA184301F8013B4FEA182201F8012B01F8018B0E70234E109A306C73
:20ADC0009DF83C104369F06B98478046B8F1FF3F24D00BA9049101208DF801009DF83C301A
:20ADE0008DF8023007AA01928DF800B08DF80370CDF80890CDF80CA0ADF81640316CADF820
:20AE000018500223F06B0A6A8DF81430694690478046306C8269F06B0FA99047B8F1000F98
:20AE200018BFE4200BD14FB109EB040138460BAA12F8013B401E01F8013BF9D1002011B0AB
:20AE4000BDE8F08F6C7A0100200800202E0C00202DE9F041424C04F1100528460BF0F7FA0C
:20AE6000071C7AD009F0CCFA7B683A6A00263E6243B397F82F0000F00700401E0BD0401E17
:20AE800006D0801E18BF002308D14FF0805304E04FF0804301E04FF00053324697F82F00CA
:20AEA000000908D397F82F0010F0070F03D04FF08070324303437968B7F92CE0F8688C464E
:20AEC0007146E0470BF0B3FA8046B4F91600401C6FF31F30E082206980F82F6028460AF0FC
:20AEE00009FE40460BF092FBB4F91400B4F91610884232D1F86890F8C20000280CBF05201A
:20AF0000072004F043FD1748F96805688D4208BF456891F8C240002C0CBF0C68341C81F8A7
:20AF2000C2604DB195F8C23023B92868A04228BF041C01E085F8C26064B1B4F1FF3F0CD0C9
:20AF40000949F86809687830B4FBF1F10AF021FFBDE8F081082009F071FBBDE8F081C046BC
:20AF6000C43500209033002030360020F8B53A4D0646287800286DD03F4CB4F91600B4F9CF
:20AF80001410884214D03046214609F02BFD021C06D1616830460BF09DF800B162683AB1B7
:20AFA000B2F92C1030464FF0E043002200F0EAFD0BF03DFA074629480168B14219BF002491
:20AFC0004460002404602878401EC0B22870244D58BB244800782E6002280ED1082009F01D
:20AFE0002DFB38460BF012FB06F140004FF0FF310BF00DF80BF01BFA074620480BF02DFA16
:20B0000019480BF012FA1E480BF027FA17480BF00CFA17480BF0F7F916480AF057FA307C47
:20B02000012802D10E2002F0C5FA2846016806F140058E4208BF046038460BF0E7FA28465F
:20B040000BF007FA06F178000BF0DDF906F19C000BF0D9F9F8BDC046103500209033002051
:20B06000FC340020403600205435002070350020B4340020DC350020C4350020FC330020DB
:20B08000303400202DE9F04F06460020ADF1140D00903E4F02917868019680473C4D0390A2
:20B0A000303D286A334CC36CE06804216A469847DFF8C4A0DFF8C8B0DFF8C88026F0010621
:20B0C0002AF0010AB24519D02C4820F00100B04212D19BF900102F6AE06811F1020F08D0A1
:20B0E0005946BA6B91F900109047812819D1E0682F6A2549083118E00BF073F998F9001000
:20B10000E0682F6A11F1020F81460CD04146BA6B91F900109047812804BFD4F80C902F6A0E
:20B1200001D00BF05EF948461749FF6A029A019BB847002818D4B24507D0104921F0010110
:20B14000B14204BF5946087001E04146087001202F6A0090E068FB6C04216A4698470B4941
:20B1600003988968884701E00BF03BF905B0BDE8F08FC0464C1D002085D20000759A000096
:20B18000ED1E0020EC1E0020C81300208C1A0020581900202DE9F04F3F48384C90F8009090
:20B1A0002078ADF12C0D012864D101200AF07CFB3A4E343E306A324F436CF868022108AA37
:20B1C00098479DF82000A24600284AD13148001D006880470025022409902A48039502A952
:20B1E0000290F8688DF8104002F0D2FF2649B3462846B9F1010F254B8AF8004001F11008F9
:20B20000DBF82060A8F802000AD006958DF81C4001218DF81D1041468DE8300045460BE06D
:20B2200006958DF81C408DF81D0001F11005024621468DE806002946346DF86806AAA047B8
:20B24000294600280BD4124A124FCBF80C1092F90000B968401C1070099888470AE00BF0FF
:20B26000C0F89AF80000012804D100208AF800000AF0E8FC0BB0BDE8F08FC046CF1F002013
:20B280004C1D002000093D00C8130020CD2D0100F61E00208C1A00208B0C00205C190020A3
:20B2A0002DE9F04105463E4804780F46002DADF1280D42D03B48466A002F3ED08046D6B1D6
:20B2C0007069C0B10123ADF8223006208DF8200029460C2200236846ADF8243003F018FECE
:20B2E00003A839460E2203F013FE766908A803C81A226B46B047787B012668B9002C14BF78
:20B300000FA013A06988102207F06AFE397B13A00A2207F065FE08E0002C14BF12A017A00C
:20B320000AF03EFE19A00AF03BFE88F80260002031464CF0D3FB88F803600AB0BDE8F081B5
:20B340005265737461727465643A20307800C046537461727465643A203078004368616EE4
:20B360006E656C3A2000C0464465766963652052657374617274656400C046C044657669C2
:20B380006365205374617274656400C04672657175656E637920486F7070696E6700C04681
:20B3A0005C1800205817002070B50C46A00852D2E0085ED32F4801250570042009F022FAC3
:20B3C0002E480068006B80472B49086036480BF03EF82B4C216870B1C068064649B18E4273
:20B3E00007D0316AC90804D3C16900220B460421984731462160486822490078086002207D
:20B4000009F000FA112002F0FFF922681E49107C0D7008B1487818B90E2002F0F5F9226842
:20B420005168886808B9C86810B118480AF082FE174A07201749106000260E60164D4E60DA
:20B440000A6845EA0200086014480AF0E5FE19200AF0EFFF70BDFFF7FBFC11480AF0F7FF24
:20B4600010B906F0CDFD70BD0E4844F002010AF0FAFF70BD12350020003500208C01001010
:20B48000FC340020D0210840403600205100070600000460141004400A000040318A00005E
:20B4A000D4350020FC330020C43500202DE9FF473A4CA11D0888401C08803949082268468D
:20B4C0004CF090F909F0D2FF4FF000084FF6FF7746464546824618E09DF80830616D2BB985
:20B4E00002EB421040184068010403E002EB42104018416850460AF096FF804503D29DF891
:20B500000890804616466D1CADB2208BA84238DC254D281D006880478046B4F85200B9F18C
:20B52000000F0DD1A26D7100002301EB8601401E8918CB708A888F8080B2A4F852000EE09F
:20B54000606D06EB461600233618B377B6F81F20A6F81F70B4F85000401EA4F8500011487D
:20B5600067690088121A91B2082207EBC10069464CF038F9608BA968401E60834046884779
:20B5800008E0284602A903F071FF02469742A3D10AF047FF0090BDE8FF87C0464011002040
:20B5A000C08101000C1F00208C1A00202DE9F84390460F460AF03BFF814641463648DFF8E5
:20B5C000DC8002788324381C06D0401E5AD0401E52D0401E0CD009E04246101D0768002F46
:20B5E00008BF802451D05068808D4DE003244CE00D6850220021284605F0CCF928480227B1
:20B6000029462B46844610305CF8042B1A60027A1A7345685D6050F80C2B1E467F1E06F159
:20B6200010032A44B260EFD142465768002F08BF02200ED05068C36857680B6297F82E307E
:20B64000566881F82C30736A55684B62AB6A03208B621768CFB1052817DAFB6801EB00126D
:20B66000136097F82E3013737B6A5360BB6A93603F68401C40B2EDE70020022A08BF012037
:20B68000087002E007480078088048460AF0BEFF2046BDE8F883C04640360020C435002081
:20B6A00090330020883300202DE9F04304463B48083000680E1C1F461546ADF12C0D16D06F
:20B6C000ADB131784FF0010808FA01F108420ED0104600210AF0B9FE6660A5600AF0A7FE6D
:20B6E0002A4D2E788146022E03DB0AF08FFF002048E016B9FEF7FCFD2E782948711C40F8EF
:20B700002640C9B2297048460AF080FF1FB903AF38460AF09BFB386820607868E060387C1C
:20B7200046462074B96966742162788A6082184DA561E5616561F86800B1A061786900B16B
:20B74000E061B86800B16061A022002104F1280005F020F904F14000002109F0B5F968465D
:20B760000AF009FE04F178000A49029400226B4607F05AFC084904F19C0000226B4607F0A6
:20B7800053FC20460BB0BDE8F083C046103500201B6400001D580100DD630100CC2108404B
:20B7A000903300202DE9F04707467D68D7F8088091460C460AF03BFEAE6A8246002E65D130
:20B7C00005F582700AF029FE2C620024EC7750466C620AF01BFF0AF02AFE304E33788246BC
:20B7E00023B9022009F00EF80120307050460AF00DFFD8F80020106B494640F4807010635E
:20B80000384608F05DFDA862C0B93846494607F09BFBA878D0B9A96805F1CC000AF0F7FBD3
:20B82000E8B1AC621020E8774146284604F066F80AF0FDFD8246307840B323E0D8F8001051
:20B84000886B40F020008863A87810B12046BDE8F087A96805F1CC000AF0D9FB10B9686A1B
:20B86000BDE8F0873846494607F06EFB1020AC624146E877284604F041F80AF0D8FD8246E9
:20B88000307818B1022008F087FD347050460AF0BDFE4FF0FF30BDE8F087C0464436002080
:20B8A0002DE9F04106AF3D793E68984604460B1CADF1180D074611D0012B15D13079737949
:20B8C000641C3870B17904F8013B337A04F8011BB17A04F8013B7389181201E0317870781E
:20B8E00004F8011B04F8010B8AB9002D0CBF42F20C0042F20D00694607F0D0F99DF8000068
:20B90000BDF8003004F8010B181204F8010BB8F1010F34D0B8F1020F39D1002D0CBF42F25B
:20B92000020042F203000DF1020107F0B7F97589CDB1681E01468B100DF1020201EB537190
:20B94000C910CBB2811000EB517121F00701401AC0B20121401C01FA00F0D15CFF3080F039
:20B96000FF000843D054E81DC2100DF1020120464BF038FF7089C01D04EBE00407E0002DEC
:20B9800014BF02210121204602F008FE2418E41B06B0A0B2BDE8F0812DE9F04390460A6847
:20B9A000D8F800401678814600271D463846ADF1140D531C242E0B6053D112F8016F5B1C1A
:20B9C0004C2E0B600ED1AA68E41C24F00304241D54F8040C494606F0F9FB2968EF60012758
:20B9E000091A2960462E1AD1E41C24F00304241D54F8040CE41C029024F00304241D54F84A
:20BA0000040C002749460390AA68ADF8047001A803F092F92968EF600127091A2960532E46
:20BA20001FD1E41C24F00304241D54F8040CE861C8F80040288B0090A968EA69D9F800009D
:20BA40004346F7F793FBD9F80040002714B12418C9F800402968D8F80040091AEF6001276C
:20BA60002960662E0AD12B8B23B9E41D24F00704083403E0E41C24F00304241D1FB9E96977
:20BA80000E700127EF60C8F8004005B0BDE8F0833EB542F2050002A907F000F99DF8080080
:20BAA000002865D042F20100694607F0F7F8314D95F89401002836D0202009F0C7FB9DF801
:20BAC0000800002464229DF80810C5F88001009B85F89441581A02FB00F105F5DC70C5F879
:20BAE000BC1106F077FF2648007868B995F8960130B92148007800283AD104F097FC3EBD63
:20BB000010200AF007FB3EBD01A807F055FE95F82A020199451EB1FBF0F24243891A01910D
:20BB20008D4225D918E09DF80810642011FB00F0C5F8BC0105F5DC7006F04CFFB5F87801EC
:20BB40000124401CA5F878010023C5F88031202085F8944109F01AFD084991F811142046B6
:20BB600021B94FF400700AF0CDFA3EBD06F0E8FC3EBDC04640110020CF1F002020080020DA
:20BB8000310C00202DE9F8439946904604460E1C44BF0020011C68D40AF061FC0546314639
:20BBA0008022204608F0D8F8071C04D097F82F0030F07F0003D128460AF024FD53E097F842
:20BBC0002F0010F00F0F46D100200A2107F1180640EA090941EA080896E8030008EA0000B6
:20BBE00019EA010608BF002820D028460AF00AFD07F1180003C804F1700604F1700508EA4B
:20BC0000000809EA010986E8000395E80C0007F1180696E8030007F118059943904385E85D
:20BC20000300703494E80300BDE8F88310487968884202D07968A166786004F1600080E86C
:20BC4000000328460AF0DEFC04F140004FF0FF310AF0DDF9E5E728460AF0D4FC97F82F0069
:20BC600010F00F0FFAD102200021BDE8F883C046C91801002DE9F04F09AF3C897D6816467D
:20BC80004FF0000A0246002EADF1440DA04610933C888DF83CA05CD0304810F80690042ED4
:20BCA00003DAA8EB0900C8464519F868A4EB080407AB0827A4B2C01D10F801C97F1E03F826
:20BCC00001CBF9D1080E264F03F8010B080C03F8010B080A03F8010B386C03F8011B9DF8B8
:20BCE0003C101E704369F86B98478346BBF1FF3F2AD0042E04DA03208DF80000022002E013
:20BD000002208DF800008DF8140002959DF83C608DF8026001218DF80110386C8DF80390C0
:20BD200007ABADF816800BADADF81840026A0193109E04956946F86B039690478346386C2B
:20BD40008269F86B0FA99047BBF1000F18BFE42000D1504611B0BDE8F08FC0466C7A010037
:20BD60002008002039482549C0F870122449C0F874122449C0F878122349C0F87C122349DA
:20BD8000C0F88012304AC0F8E421C0F8F4212049C0F884121F49C0F888121F49C0F88C1226
:20BDA0001E49C0F890121E49C0F894121D49C0F898121D49C0F89C121C49C0F8A0121C4935
:20BDC000C0F8A4121B49C0F898101B49C0F89C101A49C0F8A0101A49C0F8A4101949C0F8B5
:20BDE000A810002180F8041280F80712022180F8E811012180F8F8117047C046616C00008A
:20BE0000E526010019350100652B0100F919010071410100BD510100A1350100B9200100B0
:20BE2000B9390100E55B0100A1020100853E0100155C0100E56001008D580100A5F2000031
:20BE40005D1A01007F640100156101002008002070B5394D064695F8AA02ADF1180D80B99B
:20BE600095F8EC0282280CD031480068314C016C2068884709F010F995F8EC12D5F8C02263
:20BE8000505495F8EC02822814BF401C002005F52A7485F8EC0295F8EC0204EBE00292F8B1
:20BEA0002C00411082F82C10400807D295F8EC02401C85F8EC02C0B28128ECDB95F8EC028F
:20BEC00081282EDA04F14401E120F8F761FB02204FF6FF738DF8100095F8AA12ADF8083097
:20BEE00031F0020019D0012919BF072083210820802100224934009202AA0194FAF78EFAB5
:20BF0000DB2807D0E52805D0F32803D0DF2818BFE8280BD185F8A90203E0304604F000FC3C
:20BF200004E02A203070304605F058FA06B070BD48190020581D0020200800202DE9F04FE0
:20BF4000DFF8D89000240646ADF13C0D4FF0010B2546A0460D9318980C91DFF8C4A00E90E9
:20BF600047E016F8020FA41CA4B2401E1CD0401E09D0401E04D0401E35D1022F33D135E004
:20BF8000032F30D132E0072F2DD1B1787078042240EA0120AAF88401F11C0AF5C4704BF004
:20BFA00021FC8AF899B121E0052F1CD1CDF80880B11C02A803224BF015FC0C9803A9FCF7FE
:20BFC00051F99DF82A0088B1029BD9F80020039340F00200049200F0F7008DF82A0003A8F2
:20BFE00005F024F902E07819801C85B2E419F619A4B23046694608F089FB071CB1D1022C13
:20C0000003DC44466720254600E040460D990C800E990FB00D80BDE8F08FC046D01200200E
:20C02000401100202DE9F84F0746344800788B4620B93846F7F72AFDBDE8F88F304DE98999
:20C04000002405E03868E989641CA4B280193860A14201DC0AF0E5F938465946F7F716FD08
:20C0600095F8F411002847D19BF80080D7F800A0002940D023480168C88AC2083BD28009AD
:20C080004FF0000602D3087D152834D009F0AEF9AB898646002B06BFB5F80EC06346B5F85F
:20C0A0000EC05B1EBCF1000F9BB224D0D5F810906146184600EB800048440278904506D0AE
:20C0C00003B963465B1E491E9BB2F2D113E0D0F8011070460AF0A7F942F21073642101FBB7
:20C0E0000A018B4205D942F242706423401AB0FBF3F6002EA6D10020BDE8F88F34130020D7
:20C10000401100202408002036492DE9F04F0822ADF1140D039001A84BF064FB324C606889
:20C12000804780466946722008F052FE2B4EB0884FF6FF7590B10746002400990398091D73
:20C140004BF0FCFD012808D000987F1E04F1010400F118000090F0D100E02546224989687A
:20C1600040468847B0884FF6FF71A94218BF281C30D183461A4800F118010F88002F08BFB4
:20C18000002425D081461849D9F81450D1F8048000263446AA46504601A9082209F08CF865
:20C1A00040B17F1E06F108060AF1080A04F10104F1D10DE00399701908224BF013FBC04797
:20C1C000B9F81A10084F491CA9F81A10B96888475C44A0B205B0BDE8F08FC046081F0020F5
:20C1E00040110020C08101008C1A00202DE9F0410AF018F84FF08058D8F8E8014068804736
:20C200000AF022F8044604F00C000C284FD0E0081ED208F04BFD294E37680546012001468C
:20C2200009F033FA31686943884211D2244CF020B0FBF7F0291A20460AF0E0F920460AF0F8
:20C24000D9F90120F9F7B0FD20460AF0CFF930E020092CD208F5EC75286880680146194871
:20C2600088470428F8D01849620905D220B10846016821F0010103E00846016841F00101F0
:20C280000160D0F8981041F00301C0F89810D8F8B80180690146202088470C4CD8F8B8018F
:20C2A0002168806B804701202060206801E009F0BDFB09F0BDFFBDE8F081C0469C89010091
:20C2C00048150020004003408C2108402C2009402DE9F0470D4606465FFA85FA280824BFFD
:20C2E0002F4845402F494FEA8A032F4AC85806EA0504224085EA000706F4E0243740B4F57C
:20C30000E02F20EA0600C7F3006742EA000201D1500E14D306F4E020074310D002F4E02777
:20C32000B7F5A02707D0B7F5803704BF22F4003242F4A02203E022F4803242F4C022DFF8B3
:20C340006C80CA5008F1D00739680122002002FA0AF40C4218BF101C5FEA000906D1F00DB2
:20C3600004D34146C5F3805001F80A00300E0BD30AF05DF8290E34BF0021211C3A68A2435A
:20C38000114339600AF042F9B9F1000F06D0F00D04D34046C5F3805100F80A10BDE8F087DB
:20C3A000006000A000100840007F077F002002403448FEB5002406782B48334D0470203D29
:20C3C0002C706C702948047028696C6110B128690AF051F82D48801D0088012E14BF103031
:20C3E0000E3080B209F092F807462F610FB909F0F8FF00978DF804409DF805001C4B64F3FD
:20C4000001008DF805009DF8050064F383008DF805001889012E05F1100112BF1030154A4C
:20C4200010809DF8052064F307128DF80520ADF806000868082269464BF0D4F92F626C623D
:20C4400000F026F80C4D2878012802D02046F7F731F80A4804700A4F3C702878012802D0F7
:20C460002046F7F727F8FEBD493600204B360020081F0020E8140020CD1F00204D3600203C
:20C48000453600208B0C0020843400200A1F00207CB53148354E314D314C0078012813D17C
:20C4A0006420694606F06CFF4036C5F830419DF80000C5F8346100280CBF2A482A48C5F8C9
:20C4C000D800C5F818017CBD3246C5F8484105F2471302F14C00C5F84C011978012605F26E
:20C4E000471466F3000119702378002005F2471160F3410323700B7866F382030B7005F2F7
:20C5000047110B7860F3C3030B7005F247110B7866F304130B7005F247110B7805F24714CB
:20C5200060F345130B70217805F2471066F386112170017866F3C7110170052385F8563126
:20C5400085F8573102F18804C5F8584102F16C06C5F85C617CBDC0468B0C0020C813002031
:20C56000843400204E9055550E7A555528190020334B2DE9F04188465968044609F0AAFD8A
:20C58000002750B1586890F82E00414609F02DFD3E46051C18BF5F6801E03D460126186805
:20C5A00000B31A681CE02046114609F093FD28B192F82F0040F0080082F82F0012682BE00C
:20C5C0002046114609F086FD48B192F82E00414609F00BFD002608B10DB917460546126822
:20C5E000002AEDD1002E18BF022027D1002D14BF002F002022D058683A4690420CD1596843
:20C60000204609F067FD38B1596891F82F0040F0080081F82F001A68002AC4D1094905F08D
:20C6200001058C62BB8DCC6291F8340081F8325040F001020B86012081F83420BDE8F08110
:20C64000C4350020903300207CB5344C054694F8F5030F285DD0697E6078890959D2297ED7
:20C66000002841F00201297639D069684A1C1078801010F0030F32D000F0030002280ED157
:20C68000B4F808344FF6FE70984208DD56791179002001EB0621994208BF012004E004F217
:20C6A000FE30491D4BF04AFBC8B9687E696840F0010068764A78C2F38102022A2DD1491D95
:20C6C0004A7809784FF6FF7601EB02218E4224D1297E00F0EF0041F0200129761CE0687E30
:20C6E00040F00300687694F85F01B0B994F82B048DF80000FF238DF8033094F83A648DF80B
:20C70000016094F83B548DF80250684609F017FE7CBD687E40F0010068767CBD200800205B
:20C7200070B5064600210B22ADF1280D0DF119004BF074F82E4D3078C01E15D0801E04D051
:20C74000143811D0801F01282FD801208DF8180006F18F0103A84BF009FB032495F8FC02FC
:20C760008DF8144070B113E000208DF8180006F18F0103A84BF0FAFA032495F8FC028DF877
:20C78000144028B9B5F812040224ADF8020005E00DF1020005F22C414BF0E8FA8DF80A409F
:20C7A000B5F80E04ADF8160017E002208DF8180006F1320103A84BF0CFFA0DF1020006F179
:20C7C00028014BF0C9FA0B48008806F11C01ADF816000DF1190009F010FE0B208DF80000BA
:20C7E00075788DF80150684600F046F90AB070BD200800202E0C00202DE9F843324C94F8B5
:20C800006B94054609F040FB297E2E48090902D2297D012900D0401CDFF8B0800778464689
:20C820007068804704F178010B68002B08BF0D600CD07F1E0026FFB202E07F1E1346FFB240
:20C8400053F80C2C22B92FB143F80C5C012601E0002FF2D1D8F8081088475EB3B9F1020F7A
:20C8600002D12846FDF7ACFCA16928468847E88AA168C0081AD2D8F80400804794F88310AB
:20C88000491C84F88310D8F80810884794F8FC0210B1D4F8100330B9E88A400A0FD2FDF7C9
:20C8A0008BF9BDE8F8838047BDE8F88328468847BDE8F883F1206870284603F07FF9BDE829
:20C8C000F883C046081F0020200800208C1A00202DE9F043DFF8BC808946054617464FF070
:20C8E000FF31ADF1140D404609F091FB2A4C04EBC5046668256809F09AFD8446206800686B
:20C900004946002807D42868002803DC41B14FF0FF3107E021B1604609F078FE002431E08A
:20C920002968491C2960604609F070FE2868022828DA1FB903A809F0FAFC03AF3868686023
:20C94000B768684609F0A6FB317B009405F12C006B46124A0191394607F0EEF805F16400B9
:20C96000002108F0B1F805F14800012108F0ACF8706800F049FF0A4A05F1180023460421F9
:20C9800008F076FA404609F066FD204605B0BDE8F083C0463835002040890100C1500100AB
:20C9A0004F6301002DE9F843324D0120002428702A48DFF8AC80DFF8B0900470294800F1B5
:20C9C000C2010F8814EA03064FF0020101EA020108BF00290FD120464FF0E04710401F407B
:20C9E00008BF002827D0424692F90000401E107009F040F91FE0424692F90010491E117024
:20CA000067B900F071FD46464846047096F90000E8B196F90000002817DD1BE0B7F5505FE1
:20CA200007D113481149006800F5C070086007F0B7FD09F0E3F848464246047092F90000E0
:20CA400028B192F90000002804DC09F0CAFC2046F6F730FD2C70BDE8F883C046F01E00203B
:20CA6000F61E0020C8130020EF1E0020401900200C010021CD1F002070B506463049307815
:20CA80000D5C401F1CD0083851D0401F4FD028464AF03AFE041C0DD130780C2808D1706898
:20CAA00030B1301D06F09EFD28464AF02DFE0446002C43D02A46204631464AF093FE37E02C
:20CAC000B07810BB307C317A2D184C10480000F00E002D1804F038002D182435E8B24AF042
:20CAE00013FE041C2AD0314618224AF07BFE04F118006060716824224AF074FE60682430F3
:20CB000060617169327C0E46D6E7012816D12435E8B24AF0F9FD041C10D0314618224AF09D
:20CB200061FE04F11800606071682422EBE7344624B10448007821464AF0DCFC70BDC04619
:20CB4000AC880100FC1E00202DE9FE4F8046314DDFF8BC9095F8FC02174609EB48066836D4
:20CB600034880191C0B1D5F81413A9B109EB880BDBF8DC0000F0FF0088478246D5F81413F8
:20CB8000DBF8DC0000F47F008847504483B21BB13088C018001D84B295F8200401280AD177
:20CBA000387A40B148447B7A067919F803000019401D84B200E00026A01980B24AF0A4FD46
:20CBC00095F800A0071C19D0002122464AF026FE002587F8008008EB090138197D704A7D0F
:20CBE000786007F1840001993E814AF0FBFD504639464AF07FFC2846BDE8FE8F8DF80080E7
:20CC000068461A2102F0C6FC1A20BDE8FE8FC046687A0100200800202DE9FF412E482D4F92
:20CC200000683E78C06B80477968401AB100B0FBF1F4B868FF680025A8464146BC4271EBED
:20CC4000080101DAB84206D82946424684428A413CDA074600E0294638463246F317001BC3
:20CC6000A94109F043F8272704464FF47A7200230D46ADF802700820ADF800002046F9F71F
:20CC8000BDFA01901548016868468847029843464FF0000100F6FC02A41A9D416042A9418A
:20CCA00011DA0F48026829462046F9F7A7FA0D4604464FF000016042A94104DA204606F0BF
:20CCC0009BFD002000E00120064908700090BDE8FF81C046301E002048190020B01A002040
:20CCE000381D00204C36002070B52B48294C20652A484FF08055A065D5F8D801284E036879
:20CD000001210A46ADF1400D30469847D5F8D80142680121304690472248281A012505606B
:20CD200008F0C4FE2149002804BF081C2C3009D01D480C224271032680F82460022380F883
:20CD400025300846FAF730FF06F080FB204608F0E9FE4FF4E1302146A061002006F0DEFFAB
:20CD600013493C22082308606846002109F03AFC4FF4C06604F5887006956A460023079009
:20CD80000C49089604F15C0009F028FC09F022FC10B070BD10010020F563010047E6000077
:20CDA00000400340FCFEE32DE81C0020DC8501003C0D0020B1170000F8B52C4E96F86B040B
:20CDC000012802D0B078012801D003F02FFB03F025FA96F8FC0218B12548016801208847EC
:20CDE000254896F86B74254D007820B9281D244B0468187808B109F0F4FAA047214AA968E3
:20CE00001378022B27D101231A4C1370A378022B03D0032B18BF062B01D18323137088473A
:20CE2000A17831F001000AD0042908D0052909D1012F07D10020607109F094F901E0F9F780
:20CE400001FDA178022903D0032918BF062903D103F020FD00E0884796F8FC0228B1D6F8C5
:20CE6000100310B1102009F055F9F8BD20080020381900200C1E0020493600208C1A00204A
:20CE80004B3600204D3600202DE9F041804608F0B7F8C01DC51098F8230000284DD198F85F
:20CEA0007E4008F0ADF8A04247DD284A5368E1100846C91891F8701004F007042141CFB2D9
:20CEC000082409E0411C04EBC000C9B2CE1896F8707088F87E00084647B9691E8142F1DCFF
:20CEE0005068002188F87E10417029E098F97E10C0000830884226DD401A79080BD298F865
:20CF00007E10401E4FEA670701F1010188F87E10F3D1BDE8F08198F87E000D49087098F836
:20CF20007E0088F8810098F87E00401C88F87E000320F8F71DFEBDE8F081002088F87E00A9
:20CF4000072005F0FDFABDE8F081C04620080020171F002003B42DE9F047304C4FF000093C
:20CF600008AF84F801903968ADF1100D02A80160B988818002A803C89A46164607F08CFF11
:20CF8000A046051C14D04C4686B12846694601224AF012FD1AF804009DF80010884205D1F9
:20CFA000641C6D1CE4B2ADB2A642EEDCA6422ED0B8F80200F61C4FF6FC7441F6F87534404A
:20CFC000001985420ADA09F0BDF8FCF7BDFAB8F8020000198542B8BF012019DB396802A8CC
:20CFE000BE88016002AD868095E803002246534601F052FE98F80100B8F80210002818BFC1
:20D00000814604D164180834A0B2A8F80200484604B0BDE8F04702B07047C046241F0020D8
:20D020002DE9B04314460F46804609F000FA81462D48027883254146381C45D0401E3DD0C6
:20D04000401E38D0401E32D0401E22D02249401E0FD0401E29D1D2B9084609F0F8F9B0B98E
:20D0600021681E4809F003FA21681D4809F0FFF92CE062B9084609F0EAF940B921681920E0
:20D0800009F0DDF921681A2009F0D9F91EE000251CE0206828B1012807D1802007F0CEFA53
:20D0A00014E0802008F070FC10E003250EE020680C4908600AE02088488207E00122C86897
:20D0C0004A746030C86001E020680860484609F09DFA2846BDE8B083C4350020FC3300203D
:20D0E000303400200C350020403600202DE9FC4707460E1C14BF4FF000084FF0E808002F6D
:20D1000050D0B8F1000F4FD17868401E78603F210170BD6D002D0CBF802000207968DFF896
:20D1200094900224083E491E7960DFF884A008703889A7F85440801C388116F8080FFF2817
:20D140002DD02A2829D1706838B3D9F814138847054678689AF80020401B78607168CC4601
:20D1600031B9DCF818C33A460023E04750B10CE0DCF818C3786871688DF800206B463A4621
:20D18000E04710B9EB20BDE8FC873889B7F85430401938815819A7F85400641ECDD1786802
:20D1A000386501E04FF0E8084046BDE8FC87C046161F002020080020F0B506460F46002506
:20D1C0001446ADF1240D8B200DF10E010095FBF79FFD8A2001A9FBF79BFD707A00282ED15C
:20D1E000387AA0B9BDF80E104FF6FE70884205DCBDF80E10884220D101A90DE020489DF8D1
:20D200000E700488BDF80E008DF812700CE0022807D0032811D1394604A84AF0A7FD09240A
:20D220000BE038888DF812008DF81040211200128DF8111005248DF81300284611E00228A2
:20D240000CBF05240924012818BF311C04D1892007A9FBF75DFD07A9224604A84AF0C2FA2C
:20D26000B07A0DEB0401C8736A4604A8214603F0F7FC002814BF281C009809B0F0BDC04660
:20D280002E0C00202DE9F0410120294E294930706FF0010008702C480068C06B8047264C2B
:20D2A000054621786068A2688B002F1AB7FBF3F058433F1A8800214902FB03F8B1FBF0F0E5
:20D2C000904201D209F08DF8ED1B1D48656008EB0501FDF7D7FE1D4C303C206BE76AA16A7B
:20D2E000404207F029F9002F08BF216B08D0216B78688142DCBF401A78603F68002FF7D19F
:20D30000606B884202D0206305F040FA05F0C0F80C4C606880470546FFF77EFCA16828462E
:20D32000884708F0F9FA00203070BDE8F081C046CD1F0020EC1E0020301E0020FFF6C2FFFD
:20D3400085D200008C1A00204819002050080020F0B5314E044696F8AA02ADF13C0D0228FE
:20D3600007D0012805D005281CBFE82086F8A9024AD196F8F00200284BD1002109A81822B4
:20D3800086F8A9124AF04AFACDF828D009A8214600F0FCFA96F8BE0296F8E812814220DD85
:20D3A000D6F8C05270B10746BDF80A006989884204D1284669464AF0ABFC90B97F1E05F1F5
:20D3C0002405F1D196F8BE02D6F8C012242210FB021069464AF006FA96F8BE02401C86F800
:20D3E000BE0296F8EA0328B19DF8340010B996F8E80228B909A8FFF73FFB96F8E80240B1E4
:20D4000096F8BE12884204D12A202070204603F0E5FF0FB0F0BDC046200800202DE9F04FE9
:20D42000044628480078ADF1140D012843D10125DFF89490DFF8948089F8005098F8000051
:20D44000012802D02846F6F735F8204604F09CFB1F4F7868804700248DF80C5083460294DF
:20D460001C498DF80D401D4D4C80286A1A4A066D02238DE818001A4B10688A4602AAB047D4
:20D48000B968E88000280CD5484604705846884740460078012802D02046F6F70BF82046D6
:20D4A0000DE0104A92F90000C5F80CA0401C10705846884702E0204604F066FB012005B075
:20D4C000BDE8F08F8B0C0020F01E0020CD1F00208C1A002018140020581D0020281900202F
:20D4E000812D0100F61E00202DE9F0412E4C2F4DA07895F86B8430F0010705D0042803D07C
:20D50000032818BF05284AD129490422677995F80C640A70791CC9B261718E423ADB0328E0
:20D5200038D0B8F1010F02D102F080FFA078042807D195F8FC0220B1D5F8481309B102206A
:20D540008847607895F81914421C9142C4BF401CC1B261706E68B8F1010F03D17068318921
:20D5600002F0CCFC716895F8FC020988090902D308B106F0FBFFA078052807D1B8F1010F96
:20D580000FD1607908F0EEFDBDE8F081F9F75AF9BDE8F081E12002F069F9BDE8F08108F01D
:20D5A00020FFBDE8F081C0460C1E0020200800204D3600202DE9B043044608F038FF8146B2
:20D5C0002A48221892F8EF10491ECFB2002F82F8EF7044D1284901EB84010D78498835F0B4
:20D5E0007F0788461AD1E90911D24FF08054D4F8B801806901464046884704F5DC74206829
:20D60000406B0146404688470228F8D121E000EB8800D0F80411002088471AE04FF0805483
:20D62000D4F8B801006A014640468847D4F8B801806A014640468847D4F8B801006B01461D
:20D640004046884701210A4A0A48116001688908FCD305F03F00152801DAFFF7ABFF4846F9
:20D6600008F0D4FF0020BDE8B083C0463C1500202820086028200840148701002DE9F84343
:20D6800014460D46804608F0D2FE04F00107C4F34006274C294681460325B1F1FF3F08D1CC
:20D6A0006168404608F016FD00280CBF2168616804E04046002206F04FFB0146002930D08F
:20D6C00091F82F0030F07F002AD0201D006888420FD04046324601F00BF808B31548007829
:20D6E00001281BD0042819D01348022108F0BBFE14E091F82F200120002F00FA07F040EA9B
:20D70000020081F82F0014BF0C480D4807F00EFD26B121684046324600F0EAFF832500E022
:20D720000425484608F072FF2846BDE8F883C046C435002040360020FC3300200100020430
:20D7400001000104F8B5234E0027E82086F85C70012186F85D7008F091F95220012108F0B1
:20D7600075F91D4D482205F1840406F16400214601F0CEFB1948C5F88800403C7461184816
:20D78000C5F890001748C5F8B4001748C5F8A8001648C5F88C001648184CC5F89400154891
:20D7A0001749C5F89C00144847F23052C5F8A40004F198004AF074FA3946A061522008F019
:20D7C00045F910494EF6602204F1BC004AF068FAE061F8BDE01900205C180020E1A9000072
:20D7E00039410100FD0F010085DC0000F5480100B9EA0000DDF700001908010058170020DA
:20D8000051590100AD5501002DE9F041064608F00EFE2A4D8046711991F8EF00421C0028FE
:20D8200081F8EF2043D1264C04EB8604277807F03F00152801DAFFF7E7FF668837F07F0004
:20D840001AD1F80911D24FF08054D4F8B801406901463046884704F5DC742068406B014669
:20D86000304688470128F8D121E005EB8605D5F80411012088471AE04FF08054D4F8B80191
:20D88000C069014630468847D4F8B801406A014630468847D4F8B801C06A014630468847DD
:20D8A0000121084A0848116001688908FCD3404608F0ACFE0020BDE8F081C0463C15002095
:20D8C000148701002820086028200840F0B585686A7D2C49ADF1140D42F000462B7DAC7D76
:20D8E000009646680027FF2C41EA03024FF00203019202D0E87DFF2800D13FB1EA7DA87DE0
:20D9000011430423039140F000400290FE2106F154004DF82310694601F0F2FD3066306E51
:20D92000002808BF381C2AD0174C29688C4214BF13220F22697D07F0B1F82868844214BF00
:20D9400014221022297D306E07F0A8F8A97DFF2902D0E87DFF2800D187B12868844214BFA6
:20D9600015221122306E07F099F82868844214BF16221222E97D306E07F090F8012005B029
:20D98000F0BDC0460000C0A000100040F8B505460E460520287096F849006968E870F06BC0
:20D9A0004861686806F128014AF0D6F9B6F842006968488196F846006968487468680024E6
:20D9C0000476214869680078C873686806F11C01193008F012FD307C696888737268696889
:20D9E00012F8010B8881696812F8013B888940EA0320888117786968F81117F00707087490
:20DA00004FF0030017FB00F1204618BF01204018C1B28918491C11F8010B287200F00702EA
:20DA2000E960401000F0380000EB420040187268318968615318834239BF2C72211C801AA6
:20DA4000091A2974F8BDC0465A0C002010F47C1F7CB524D110F00F0F24D006460024012558
:20DA600005EA0600AE436D00401E13D0401E0FD0801E0BD0001F0FD142F20500694605F080
:20DA80000DF99DF8000038B1093404E0241D02E0E41D00E0641DA4B2002EE1D133E010F013
:20DAA0000F0F01D000207CBD064602244FF4803505EA0600AE436D00B0F5803018D0B0F57F
:20DAC000803013D0B0F500300ED0B0F5802009D0B0F5002004D0B0F580100FD1072008E025
:20DAE000062006E0052004E0042002E0022000E0012000F083F90019801C84B2002ED7D1BB
:20DB0000022CD8BF002420467CBD70472DE9FF472A4C89468246211D0888401C088028493A
:20DB20000822684649F05EFE208B4FF6FF7880B165690746002628465146082207F0BCFBC2
:20DB400030B17F1E05F1080506F10106F3D100E0B0464FF6FF75454504D1207A401C20720C
:20DB60002E4627E0404602A901F080FC0646B542F6D09DF80800012807D0A16D700000EB7D
:20DB800086004018A0F8049005E0616D06EB46104018A0F81F9060696946082200EBC8008D
:20DBA00049F020FE074D68688047618B491E6183A968884730460090BDE8FF87401100206A
:20DBC000C08101008C1A002030B50546ADF12C0D08F082F9002818BFFC2051D16846294669
:20DBE000112249F0FFFDAC7C697D8DF81240687C8DF81510EB7C8DF811002A7D8DF81330DE
:20DC0000AC7D8DF81420002104B101212C7E8DF8161095F825208DF81840E87D8DF82520F7
:20DC200095F824308DF81700EC8C8DF8243005F119010B220DF11900ADF8264049F0D2FDAF
:20DC4000687C002448B9812049F03CFE0A9080B1FF21812249F0E2FD0DE09DF815000A94CC
:20DC600048B1242110FB01F080B249F02BFE0A9008B91A2403E00720694603F0E5FB20464B
:20DC80000BB030BD70B505462B4C2878ADF1200DEB2829D040B3E92806D0E12843D14FF444
:20DCA000FA7006F0C7FD3EE004F15E010878401C087094F85A00032818BF042803D14FF44F
:20DCC000FA7006F0B7FD94F85E00032809D094F85A00022827D104F10A00102149F0B2FF20
:20DCE00021E005F049FE1EE094F85A00022817D104AE6946304605F0B9FC5220002107F0E6
:20DD0000A5FE606920B1026812B1304669469047042003F0A5FD04F10A00102149F092FFEA
:20DD2000002084F85E0005488830016809B12846884708B070BDC046E0190020E019002067
:20DD40002DE9F843DFF8AC9099F84900002848D0002501212C4699F8492001FA04F0104251
:20DD600003D1641C032CF6D33BE099F849201020A040104218BF0D1C08F059FB99F849209A
:20DD80001121A14081F0FF01114089F8491008F03DFCE0B207F092FF071C22D0B87A00B38F
:20DDA00097F90960304608F0BDF938687C68012D804606D0387A022804D1F868400B01D3C8
:20DDC00003E08469384602F0EFFA012D19BF311C4FF000636FF0FE014FF00073404600226D
:20DDE000A04799F8490018B10348002108F03BFBBDE8F883403300203034002010B5401EA5
:20DE0000ADF1380D28D0401E09D0801E4FD0401E43D0401E3FD0401E3BD0002048E001A8FB
:20DE200000F05AFD04460CA942F2090004F036FF9DF83000002808BF002203D0022006F075
:20DE400016FE024601209DF83010009001AB204605F02DFA0A3028E001A800F03DFD044653
:20DE60000CA942F2080004F019FF9DF83000002808BF002203D0012006F0F9FD0246002087
:20DE80009DF83010009001AB204605F010FA001D0BE020200CE002200AE042F2130004A9D8
:20DEA00004F0FCFE04A849F0BBFC80B200E004200EB010BDFEB54FF0805684684568D6F8E8
:20DEC000D0112068C9688847216822488A6B1040886340F2F2712068204B41641E4994F896
:20DEE000210094F82020085C9A5C216810434863684608F08AFA1C4FDFF868E0D6F8D011F1
:20DF00002B7FDFF85CC06A7FA87F496857F823705EF82260AA695CF820300D4620680199BD
:20DF20003E433343A8472168C86A40F01000C8622168086B40F001000863A07D0027FF28D3
:20DF400002D0E07DFF2800D11FB1086B40F440400863FEBD0DF8FFFF66890100728901008E
:20DF60009888010050890100F4880100FEB50546687E30F07F0052D0287D0027012818BFB8
:20DF800003284CD1264CB4F8540000F0020100F00800084343D069684878C0F3810002288F
:20DFA0008DF8080006D003280ED1491D684649F0DDFE09E08A79487940EA0220ADF800002E
:20DFC000CE78087946EA0026A06F0146A8B1487E30F07F000AD0087D012818BF032805D1B0
:20DFE0004A686846314605F0B9FA28B955F80C0C00280146EBD100E02F4687B99DF80800FF
:20E000003146022818BF032809D1684602F08AF9FF2804D09DF80820002105F00DFDFEBDCD
:20E02000200800202348F8B500248460224904602848224608F001FA20480068006B8047DC
:20E040002049254B1E4D0A685F782968801A01EB1030286037B19F7827B91B490968B0EB05
:20E06000C12F21D907F0B2FAD0B1184840F60901018000F10D024480117800F10C0621F010
:20E080000F0141F001011170317864F3030131702146416008F04EF8418811F4406FFBD089
:20E0A0002C609C700120587005F006F808480460F8BDC0460C100440951901008C010010D1
:20E0C00008350020003500200C350020043600200000046054350020403600202DE9F84FD3
:20E0E0001D4691468A46044608F0A1F9834607F02FF86FF001080AAF061C3ED004F1780095
:20E1000008F08BF9C6F808A01F4886F82E90B0F91410F460491C6FF31F3181827560818A5F
:20E120001A4DB18597E80006202206F1100302EA0A0205EA0901002583E8060006F11803D8
:20E14000294686F82F502A4683E806006A46314604F0F0FD88B196F82F00B18D40F0800086
:20E1600086F82F009DF8007084F8C250A4F8C0100FB107F0EBFDB6F92C80584608F046FA23
:20E180004046BDE8F88FC046C4350020FDEFFF9F2DE9F0470F4627493A6805464FEA920951
:20E1A000494502D3387A022802D00320BDE8F08708F03DF9204C8246201D0068A84214BF4B
:20E1C00000260126B00080F004002158284606F020FC804619480268B8F1000F0CD194F823
:20E1E0003400A56240F0020084F83400504608F00DFA0020BDE8F0873968B00000EBC6002F
:20E20000001901613B7A9C35B9FBF2F10376284607F0BFFD504608F0F9F9B8F1010F06D1BC
:20E22000E06AB4F9301094F8322008F08CF88320BDE8F08740420F00903300203036002094
:20E2400098B5294C204608F002F90746012004F0A1F9606800283FD1002F39D01F48F968A7
:20E260000068884231D1684604F0E8F938B1009828B1E06818B9082006F0E0F998BD082000
:20E2800007F082FB38691649C043486038698A681043886007F1100090E80C00181CC043CE
:20E2A00041F8040C07F1100090E80C000A68181C10430860B86806F039FF204607F01AFC67
:20E2C0006060002004F066F998BD4FF4806100E00221044808F0C7F898BDC046FC340020E1
:20E2E0000C100440FC330020C435002030B5274C0120002584F85C01ADF1140D65702548DE
:20E3000084F85F51001D006884F8615180470246A06F68B1417E8B0806D341F001014176D2
:20E32000017E01F0FD01017650F80C0C0028F1D11748816810468847102007F0EBFE082009
:20E3400007F0E8FE94F86001D8B9E0238DF80F5009208DF80130B4F80E248DF8000094F8AD
:20E360002B14ADF8022094F83A548DF8041094F83B348DF8055068468DF80630FEF77CFB3A
:20E3800001E084F8605105B030BDC046200800208C1A00208C1A0020F8B5284C6068804743
:20E3A00006462148A1680278832A3AD11F4D2F797FB386210170082007F0E8F8688B1D49B7
:20E3C000401C68831A481E4FC1621B493A7891F86B34012B13D191F83B14802908DD8429A3
:20E3E00006DA40F6485191FBF2F101F6B8310BE040F6485191FBF2F101F2A32104E040F625
:20E40000485191FBF2F19631243007F093FAA16807E08522027030468847002001F026FAD6
:20E42000F8BD30468847F8BD4D3600200C1E0020B41C0020192E0100200800208C1A0020FA
:20E44000301E002090B5044600214022ADF1440D684602F09FFAA0788DF80000E0788DF89A
:20E4600001009DF8000000BB616811B101A805F041F9217A01F007028DF82820E0689DF8A9
:20E480002870C1F302118DF8301027B19DF828100B9000EB41009DF8307007B10D90207CC6
:20E4A0008DF8380067690F9719E0616811B101A805F020F9677A8DF82970A37A8DF82A30F3
:20E4C000207A8DF82800E27A8DF82B20217B8DF82C10677B8DF82D70E389ADF82E300348AE
:20E4E000006801696846884711B090BDE01E002070B50025ADF1200D07A8ADF81C5007F0D5
:20E50000A1FD254CBDF81C10B4F84000884237D194F85B00032811D004280DD0022810D146
:20E5200004AE6946304605F0A1F8606920B1026812B1304669469047042000E0032003F099
:20E540008FF9206E06F076F95220294607F07EFA07F036FC044607F033FC00EB042407F04D
:20E560002FFC4FF47A7200EB0420B0FBF2F15143401A0A3006F076F9284606F08BF909E046
:20E58000032007F0EFFC052003F06AF95220294607F05CFA08B070BDE0190020F0B5012900
:20E5A00004460546ADF1140D04D0022941D142F2030001E042F20200694604F06FFB04B1E6
:20E5C0006D1C06F01DFDC01DC010C0B2002830D000230646ADF1010C1F4618461CF801EF7A
:20E5E00000224EFA02F101F00101884211D028B97F1CBFB25CB102EBC30103E03CB102EBB8
:20E60000C301491E05F8011B091205F8011B80F00100521C082AE4DB761E03F10103DDD178
:20E6200030B12CB1D800401E05F8010B001228700FB9002005E004B12770012000EB870087
:20E6400080B205B0F0BD7047F8B50B4601460024104603B90124002200B90122DFF88CC0AE
:20E66000DFF884E0E3B19E6AD6B14F6AC7B1DC68CD68A54206D073461D68A54214BFDB689A
:20E680009B6800E00023BC086546A4EB9604E41AA54222DBB4F1704F01DB002C1DDD01246F
:20E6A000F0B1476AE7B18E6AD6B1C068C968884206D073461968814214BFD868986800E008
:20E6C0000020C0EB97006546A0EB9600854204DBB0F1704F03DB002801DC0020F8BD01222B
:20E6E0001440E0B2F8BDC04690330020FEFFFF2F2DE9F843264C814620680F469046002509
:20E70000B8420AD0206800E0006820B1016811B101688F42F8D1074606E004F1100648468A
:20E72000394607F0D7FCE0B977B310343968484607F0D0FC88B1396891F82F0040F00400D1
:20E7400081F82F00086800223860204604F0F2FA6D1CB8F1010F01D016E03F68002FE5D10C
:20E7600012E097F82F0040F0040087F82F00204607F0C0F930463946002204F0DBFA276882
:20E780006D1CB8F1010FCAD02846BDE8F883C046C4350020F8B5274C06460E220D4604F10C
:20E7A000340000F0B5FB022084F824006888A08307F006FB074607F003FB00EB072707F066
:20E7C000FFFAE26A00EB0720B0FBF2F15143401A0A3006F047F830462946FCF761FD207829
:20E7E00001280BD0687B48B9288869882A1D03F021FB011C02D00BA007F0E7FDE56806F082
:20E80000E5FD854203D806F0E1FD451B03E006F0DDFD401B451E6420E560B5FBF0F0A4F8DA
:20E820007800F8BD41757468204572726F723A20307800C05C1800201CB5214C04F5DC7016
:20E8400006F09EFA04F5CE7006F09AFA04F5EA7006F096FA0021882204F5BA7048F0DEFF8D
:20E8600007F0B8FA06F0CCFB84F89A01154984F89B011548086001200DF1010184F8F3014F
:20E8800042F2040004F00AFA42F20500694604F005FA0E489DF80110C4F8A801642011FB7C
:20E8A00000F1C4F8A0110A49C4F8C4119DF8001011FB00F0C4F8BC010648C4F8E0011CBD38
:20E8C0004011002038190020A5470100252A010091BA00008F630100F0B50446E820ADF146
:20E8E000240D08A904F04CFD9DF82000694606F0C0FB00280CBF00981D480DF12101606014
:20E90000E82004F03DFD9DF8210004A906F0B1FB58B90599C8200322B1FBF0F0401EB0FB6B
:20E92000F2F15143401AC0B200E00020207206F067FB002167686081072321700D4A6170F6
:20E940005568BD420CD1157A267AB54208D15589854205D11078207057786770084604E0B4
:20E960005B1E02F10C02EBD1012009B0F0BDC04638C40D00E41100202DE9F043254C0746AF
:20E98000243C606AADF1240D00283ED0002F3CD0387A002839D004F09DFD5FEA000834D047
:20E9A000062000250323A1468DF808002E46ADF80A30B5F5FA7F28DAD9F82400ADF80C5004
:20E9C00004AB02AA0469009392E803000A230022A047B0B9387A9DF81810814210D1022883
:20E9E00004D1BDF810103A88914207D0032807D104A93846082206F05FFC08B9284606E043
:20EA0000761CB04505F10105D3DC4FF0FF3009B0BDE8F0837C170020F0B520480127F84263
:20EA200001D004F06BFA204D204F214EBD4206D203CD0478A4003459401CA047F6E71D4888
:20EA4000002800D08047164D164FBD4202D210CDA047FAE7F0BD03251BE0416808300A1CE0
:20EA60002A400BD11A1C2A40AB4305D0046804300C600431043BF9D1131C05D004780130F2
:20EA80000C700131013BF9D1021C2A4001D0A84304300368002BE0D17047C046FFFFFFFF4A
:20EAA0000000000000000000088E0100308E0100D88D0100D5BB031070B50546244C287877
:20EAC00000283FD1A07801283CD0281DFFF754FFB0F1FF3F36D1298AC81333D001F00F01AB
:20EAE0000F292FD12046B0F840104FF6FF728A4203D0EA898A4205D102E0E989A0F84010DA
:20EB00000121C170A97C80F84210AE88A0F84460298A01F00F020F2A05D080F85820C1F3DA
:20EB2000031180F8591090F858100F290AD1012181700848064649F0DBF8012802D13046B0
:20EB400049F0E4F87434216809B12846884770BDE01900201418002003B426482DE9F0417A
:20EB6000008806AF1646ADF1080D001F84B2082C39DB3D78201F6946082280B2804648F0AF
:20EB80001BFFBDF80000C10B19D300F0FF00854215D17888BDF80210884210D1B888BDF8EB
:20EBA000041088420BD1BDF80600002E18BF40461AD1C0F30E00241A241FA0B214E0BDF82D
:20EBC000061008466FF30E0048B908460830844202DA48F023FF06E0641A083C00E0241F13
:20EBE000A4B2082CC6DA002002B0BDE8F04102B07047C046261F00202DE9F84F244C8346D9
:20EC000060688A46804706462248A16800F178021768884627B9304688470020BDE8F88FAD
:20EC2000002581462C46BC4220D0787E30F07F0018D07A685146584604F090FC90B144B13E
:20EC4000207D012812D16168087840F0100008700CE03C46607E40F010006076207E40F0DA
:20EC60008000207657F80C7C002FDED141463046884754B199F8FC0220B1D9F8100308B1FB
:20EC8000804701E0FAF798FF01252846BDE8F88F8C1A00202008002003B426482DE9F0410A
:20ECA000058806AF1446ADF1080D98464FF6FF70ADF800000222ADF802006946ADF80400AB
:20ECC00044F40040ADF80600281986B2304602F03DFABDF80600022269466FF3DF30ADF855
:20ECE0000600304602F032FAA1102846CAB2414602F02CFA387840F44040ADF80000788837
:20ED0000ADF80200B88802226946ADF80400304602F01CFABDF80000022269466FF3DF3019
:20ED2000ADF80000304602F011FA02B0BDE8F04102B07047261F00202DE9F843002A89461B
:20ED400007464CBF47F6FF75151C002F08BF002033D03888002808BF002403D02A4600F05A
:20ED600039FB0446281B002826DD388828B1291B484613A204F09CFC2418B868E0B1D7F83F
:20ED800004802E1BB8F1000F0DD0404607F0CCF8401DB04207DC291B48460AA2434604F0A3
:20EDA00087FC24182E1B122E06DBBB68291B484606A204F07DFC24182046BDE8F883C04658
:20EDC0003A2000C0222573222C2000C06C696E652025643A200070471B4838B50468B4F16E
:20EDE000FF3F08BF002406F0A9FC04282BD12048164B0025103805601868806C80471448FD
:20EE0000006820B1134800682046F7F7E5F8124812490560124C0A686FF35B4244EA0200AC
:20EE2000086010490868C0F30130012806D10A680D48104040F400320A6008600B490868AA
:20EE40000028FCD138BDFEE71C130050F001001080012843800520438C21084048200340EF
:20EE60000000390128000940EFFFFCFC0C0068429404604210B5244C08BB04F1CC021178CD
:20EE8000002004F1740360F303011170197860F303011970206794F8781004F1780241F062
:20EEA000080184F87810117860F30411F420117004F1790104F064FA44F6206019E004F156
:20EEC0007801087840F00800087094F8780020F0100084F8780048F03BFD0A2280B24FF460
:20EEE000FA6390FBF2F1514344F62062401A10FB0320064AC4F8800092F8FC1219B1D2F8B7
:20EF00005C1301B1884710BDC813002020080020002A4AD05FEA000C8B071CD1830722D15C
:20EF2000102A08D370B4103A78C978C0103AFBD270BC103238D0042A2CD3082A05D30C2ADB
:20EF400024BF08C908C008C908C008C908C092072AD0920F22E00B780370491C401C521EA6
:20EF600022D08B07F7D1C30714D18307D8D0121F12D308C903801B0C4380001D121FF8D2F8
:20EF80000AE008C903701B0A43701B0A83701B0AC370001D121FF4D2121D05D00B780370ED
:20EFA000491C401C521EF9D160467047D0B5244C04F178010F68002F3FD0002215280AD1A7
:20EFC0003B7D0126022B08D0032B06D0052B04D0042B02D000E03B7D0026984200D016B115
:20EFE0007B7E5B0905D23A4657F80C7C002FE5D123E00846394648F0EBFAF88A6760000A61
:20F0000003D397F91C0006F053FF387D022818BF052802D1012006F0B9FA6068407E30F000
:20F020007F0005D194F88300401E84F8830004E094F88200401E84F882003846D0BDC046B0
:20F0400020080020F8B5044642F209000DF1020103F024FE9DF8020050B19DF802000228C5
:20F0600033D1A08894F8271001F090FF054606E042F20D00694603F011FE9DF80050154EB6
:20F08000301D0768802D01DD07F0ABF9B847124B0E490F4A1F780D701FB91778B1684FB9E6
:20F0A00004E01778B16837F07F0703D1884701F0F9FA00E088470020A4F87C5094F821703C
:20F0C000607017B1102007F025F8F8BD4C1D00204D3600208C1A00201C0B002070B50546F6
:20F0E000204C1F48A1680068401A4FF47A7141431D48006800680E0C80472169401A48BFBF
:20F10000404240F6B831AD19A94211D306280FDAA268E1688A420BD8206848B1891A134A1F
:20F1200051438A0C02EB1141884288BF011C08E00F49486840080ED208687D2100F0FF0023
:20F140004143C82905D3B1F57A6F88BF4FF47A6103E0C82101E04FF4FA61084670BDC046A2
:20F1600030200940F0350020EC01001040420F00AC4F005003B42DE9F04307AF97F8008013
:20F180007C88BD88ADF1140DB8F1FF0F0FD14FF6FF70A0420BD1A84209D104F079F906F03E
:20F1A000D7FE19480421801C0180002027E000264BF6FF790FE06946082248F0FDFBBDF824
:20F1C00000006946022209EA0000ADF80000384601F0BCFF3E468DF80880ADF80A4002A870
:20F1E000ADF80C5003C80122FFF7B6FC071C03D1002EDAD10A2002E0BE42DCD1022005B018
:20F20000BDE8F04302B07047241F002030B5044660684078ADF1440DC0091FD31F4DB4F8D9
:20F220004200B5F80E14884218D1A878A0B995F8180498B104F1280005F06AFE70B90120DB
:20F2400000901C340194B5F80E3405F2FE3203210620F7F7E3F81FE006F0FCFA0BA8002151
:20F26000182248F0DBFA02A821460C900BA8FEF78DFB2C208DF82C000BA802F0AFF80848D1
:20F280005038007810B19DF83C0028B105208DF82C000BA8FDF7F0FB11B030BD20080020A5
:20F2A0005A0C002038B5054695F83000032839D195F83A00032835D105F128044A202146B3
:20F2C000F5F766F98A202146F8F7B8F86C686178207800EB0120ADF8000069465020F5F732
:20F2E00057F9A41C6178207800EB0120ADF8000069464B20F5F74CF98B206946F8F79EF8B2
:20F30000A41CE1202146F5F743F9641C6178207800EB0120ADF8000069465320F5F738F9BC
:20F32000002000E0E82004492A24087028462C7002F054F838BDC046C90A00202DE9F8432B
:20F340002020EFF3118780F31188214CA068012107F03CF94FF001094FF00008656921683D
:20F36000A4F81C906A1A2168A4F81E80461B401A904227D387F3118840462D18361A4846BB
:20F38000294607F01FF9B042F7D92021EFF3118781F31188E18B012903D14046294607F00F
:20F3A00011F9B0F1FF3F06D0A169801B814238BF081C291801E0A069411907F0FFF8A4F8FC
:20F3C00020902560A4F81C8087F31188BDE8F883501600207FB503461F480D4601881F48E0
:20F3E0000088144614A6984205DB32462146284604F05EF91DE0994206DB184606F026F9F3
:20F400000028F2D04268F1E715480088002808BF0CA2EBD00095002C48BF47F6FF74114E6C
:20F420000020114901946A46346802901846A047029800907FBDC0467B6D6F64756C65230A
:20F4400025647D007B6D6F64756C652D726F70653A25787D00C046C0D2880100268901009D
:20F46000E47E0100B0890100B5490100F8B50A46034621492148B1F84E70858891F809C011
:20F480008C6D8646ED18ADB25FB10020A41FA41DE67816B1A688B54208D07F1E00F10100DE
:20F4A000F5D10CF10100C0B2487206E04FF6FF7484421CBF002111701CD101201070B1F844
:20F4C0004C70BEF804604C6D4A7AF01883B267B10020213C2134A67F1EB1B4F81F50AB42B6
:20F4E00008D07F1E00F10100F4D1521CD0B248724FF6FF70F8BDC04640110020081F00200F
:20F500002DE9F843DFF87C900F4604464FF0FF31484606F07CFDDFF870801D4800210AE075
:20F52000FF2A07D00368934202D358F822600EB1002421E0491C1FB117F82120FE2AEFD193
:20F5400000202060012660600546A0600EE0FF290BD0636806FA01F048F8214018430B49DC
:20F5600060601268204604F0FDFE6D1C27B107EB85021178FE29EAD1484606F06CFF204662
:20F58000BDE8F883A8350020C0320020007FC7673C1F002090B50C46214A0178575CADF148
:20F5A0001C0D0B2F8DF8007034D0002F35D00C2F04D0112F28D148F021F925E01A2C21D0E5
:20F5C00090F89D100190C7688DF80210038A0297C28AADF80C30510904D21249827E097840
:20F5E000891A00E000218DF80E10877F8DF8107090F91F308DF81130826A0592417F8DF853
:20F600000F1001E0002001908DF801406846FDF733FA02E04470FDF783F807B090BDC04695
:20F62000897A01003C0C00202DE978411E4C012020701E480078012814BF08200220DFF879
:20F640007080002103EA010502EA00068D4208BF86420DD000214FF0E0401140184008BF89
:20F66000002905D11449088C4546401C088404E0454695F90000401E287006F031F906F01E
:20F68000BDFA0C480026067095F9000028B195F90000002804DC06F0A4FE3046F3F70AFFC5
:20F6A0002670BDE87881C046CD1F00208B0C0020F61E0020EF1E00200C1E00202DE9F0415B
:20F6C000804621483C3800680D46416927208847012404FA05F6194DC5F80064C5F87C47E7
:20F6E0000327C5F8807716480460C5F88477D5F80404012818BFC5F80444C5F8FC63114863
:20F700000460C5F800801023AB60204606F054FED5F88C074008F8D3D5F88C17204611F012
:20F72000404F09D1C5F884770021C5F8FC16D5F80024164218BF081CBDE8F08104400240D8
:20F7400000E0484200004842EC0100107CB5204C3C3CE06B0068014604208847022818D0A4
:20F76000032816D018480068C0F38150032814BF41F288324FF47A721648174C01684C3468
:20F780002046B2FBF1F106F044FE204606F043FE7CBD20680D4E406803214FF040521C23A7
:20F7A0000546009100213046A8472068406801214FF4007209230446009100213046A0475B
:20F7C000022004F0E9FD7CBDB44F005000A00C40E0010010303600204415002070B5064654
:20F7E000204D307800BB7178E8782C46012910D0022909D003292FD100204021207104F13D
:20F800000A0048F01FFA27E028B1022006F0AAFB22E0012806D05220002106F017F941F223
:20F82000883013E02021EAE75220002106F00EF97078032802D13178EA2905D001280BD1FF
:20F8400000202C46E870EAE72C46074894F85C1084F85D1005F01EF87C35296809B13046CE
:20F86000884770BDE0190020E0930400F8B5074600251F481D4C05701F4894F86B140570B1
:20F8800094F8FC0218B1D4F84003666860B9012902D0A078012801D000F0C8FD00F0BEFCB2
:20F8A0003846F8F7ABFD19E0307D35280BD1012903D17068318900F021FB7068008800094F
:20F8C00001D304F053FED4F840133846884709480078012802D02846F3F7ECFD606810B115
:20F8E000007D352801D006F089F9F8BD2008002045360020CD1F00204D360020F8B50E469D
:20F900003268916B054621F020019163286E317D012203F0F5FB286E317D012204F0A4F99E
:20F92000286E317D002205F0B9F8286EB17D002205F0B4F8A878012807D005F1CC004FF013
:20F94000FF3106F064FB306803E0306881690909FCD20D4C84420CBF10221422317D286EAF
:20F9600005F09CF8B17D0027FF2902D0F07DFF2800D13FB13068844214BF15221122286E29
:20F9800005F08CF8F8BDC04600100040F8B5054606F04DFD1F4C064604F1340220681178B8
:20F9A000A943117030B19C3006F06CFB002700B1012700E00027606838B19C3006F062FBF9
:20F9C00038434FF0000718BF012794F83400E0B9012F1AD0A06AD8B1016A89080AD24569DB
:20F9E000304606F013FEA06A00214FF400030A46A84707E0C569304606F008FEA06A022126
:20FA00000022A8470020A062F8BD304606F0FEFDF8BDC0469033002070B506467468B5688F
:20FA2000206E05F023FE29681C488A6B10408863304600F037F8304601F076FE2968C86ACA
:20FA400020F01000C862296815480A6B104008636868FDF7AFFD04F17C0006F0E6FC04F190
:20FA6000980006F0FAFCA07818B904F1CC0006F0F0FC607818B904F1E80006F0EAFC04F51B
:20FA8000827006F0C0FC06F0D2FC0021217006F0BDFD04F1680005F019FD70BD0DF8FFFF04
:20FAA000FEFCFFFF2DE9F04106467568B46806F0BEFCA96A39B921688969090903D206F0B5
:20FAC000A5FDBDE8F0810027AF6206F09FFDA17D3846FF2902D0E17DFF2900D118B1284680
:20FAE0002146FFF70BFF2168886B20F0200088632168086B20F48070086306F098FC0B4CBC
:20FB00008046207818B1022004F046FC2770404606F07CFD696A286A2F696A6A401A286225
:20FB2000296A3B4630469847BDE8F0814436002038B50C4644220546002100F02BFF04F18C
:20FB40002801284606F006F804F1320105F10A0006F000F8E06B6861B4F840002883B4F8AD
:20FB600042006883B4F84400A88394F84600A87794F84700E87794F9480085F8200094F81C
:20FB8000490085F82100B4F850006884E06C6862A07B85F8280094F8520085F82900606D6F
:20FBA0000B2204F11C01E86205F13000FFF7B0F92089A5F840006068E86338BD98B50446D2
:20FBC000217D012905D0152903D0252918BF352917D1207E000914D219484E30007858B11F
:20FBE00060781B2806D1012005F0D0FC4FF4806006F088FA0020607061782046FFF7CAFCAB
:20FC000098BD207EC20918D2012918BF152901D100090BD267781B2F06D00A48002F0CBFFA
:20FC20001A302830405C02E0232000E03120207002480078214647F05DFC98BD200800204A
:20FC40003C0C0020897A010038B504461F4800780D4601280FD004F10800690880B224BF44
:20FC600004F12C0080B2122CCCBF14210621401880B2400028E0E920694603F081FB1448B7
:20FC800090F83B04802801DD84280FDB04F10D00690880B224BF04F1260080B2122CCCBFE3
:20FCA00005210221401880B2C0000DE06001690800F5967080B224BF00F21E2080B2122C42
:20FCC000CCBF28210C21401880B238BD8B0C0020200800202DE9F04107461F49BE687C689F
:20FCE000306809688069C0F3C00018BB06F09FFB1A4D8046287820B1022004F04DFB002020
:20FD00002870404606F082FC3168886B20F0200088633168086B20F480700863206A616ADA
:20FD20002569626A401A2062216A2B4638469847BDE8F0814FF4FA70B0FBF1F1012998BF63
:20FD4000012104F58274204606F063FB204606F062FBBDE8F081C0463036002044360020E3
:20FD6000B0B504680D4617464FF0FF3104F1480006F04DF928464FF0FF35092808D0227A94
:20FD800001218140114211D111430546217210E0227A0721012303FA01F0104202D0491EC8
:20FDA000F9D503E0227A0D4610432072B5F1FF3F15D0A7B1062004F025FD29463846FFF77E
:20FDC0007DFC0746062004F0E7FA47B1217A0120A8404FF0FF3580F0FF000840207204F115
:20FDE000480006F038FB2846B0BD7CB515460E46044600E024182046694604F087FC0028BD
:20FE00002DD014F8021F8E42F4D1491E04F101041FD0491E12D0491E08D0491E18BF62208B
:20FE200027D102281BD12078287021E0032816D114F8010B28702078687019E007280ED14A
:20FE400061782078042240EA01202880A11C281D0CE0052803D120780628287001DD672066
:20FE60007CBD281D002103220160611C47F0BAFC00207CBDF8B51F4CA0F5C060D4F8B81039
:20FE8000C4F8D4000029B8BF49420028B8BF404281422BDA4FF08057D7F8A401B4F8BC10BC
:20FEA000154D40684FF47F4208230646009128463021B047D7F8A401B4F8C01040684FF49B
:20FEC000F80212230646009104212846B047D7F8A401B4F8D01040684FF440620A23064686
:20FEE000009120212846B047012000E0002084F8D800F8BD3C15002000A00C40C8B50F4672
:20FF0000082F0BDA002F3CD001787F1E91FAA1F14FEA216100F8011BF6D1C8BD414201F0C8
:20FF200003017F1A4618BBB2864203F0030200EB010709D9361A0178761E91FAA1F14FEA11
:20FF4000216100F8011BF6D123F003017F1887420AD9391AC91C8E100168761E91FAA1F1FA
:20FF600009BA40F8041BF7D1BF18874209D93F1A01787F1E91FAA1F14FEA216100F8011BC2
:20FF8000F6D1C8BD2DE9B84106F051FA1E4C1C4D804604F1E000007848B9A8680146022065
:20FFA00088470746102003F03FFB1FB31EE001F0EBFA78B9134800683221B1FBF0F101B994
:20FFC000012104F1300006F024FA04F1300006F022FA0FE0A8680022014684F8E020022089
:20FFE00088470746102003F01FFB1FB1A868014603208847404606F009FBBDE8B881C0462B
:020000040001F9
:20000000D4880100303600203C1500203EB51C4D05F5A8710878012464F30000087005F5AF
:20002000A871087864F38200087005F5A871087864F30410087005F5A871087864F38610E0
:2000400008701048022205F5A871047042F20200ADF800000DF1020047F0C4FB01A8224643
:2000600005F5A97147F0BEFBB5F83A01022806D106480068044D426A2868694690473EBDCF
:20008000C8130020181F0020581D0020481900200146F8B501F01E0201F01F00162AA4BF40
:2000A00001F01F002038184E317801F01F011629A8BF2039814225D0144F3B68144A23F08A
:2000C00010031C0A14D323F08004A2F108053C602C680DE014688142B4BF01244FF0FF3463
:2000E0000919347801F01F0504F0E004254335708842EFD11068180A04D3106810683B60B2
:2001000052F8080CF8BDC04606620840280009403420094010B51C4C207838B91B481C498A
:200120004FF47A72FEF7F4FE012020704FF00451012481F82644022381F8DA33032281F813
:20014000FE23042481F8B443052381F80034062281F8E323002081F8EC03072481F8E1431A
:20016000082381F80134092281F802240A2481F8DE430B2381F8DF330C2281F8DD23054C63
:20018000C1F8884410BDC046CE1F0020244000211C660100ED4200212DE9F8431D4C194887
:2001A000676805F07FFF1849054608680E6800F02000284006F4602614D09FB107F118012E
:2001C00091E80003A760044600201837210040EA080041EA090187E803000F484FF40051FE
:2001E00006F041F916EA05000AD0084A92F8491041EA504082F849000548002106F033F9AD
:20020000BDE8F88320000E000C1004404033002030340020C4350020FC3300209EB5194CF9
:20022000606880472146184C2289E388934225D0164B1F7817BB164B89681F7837F07F0724
:200240001DD1E28088471023124FE088ADF8003001A9ADF804003A7809880DF10207398058
:200260000D48012A18BFC838BDF804100B4F01803868426AE068694690479EBD896888474E
:200280009EBDC0468C1A00204C1D00204B3600204D3600208B0C0020C2140020481900203C
:2002A000F8B50546012003F0B1FD1D4C04F5EE7000F0FCF804F5F67000F0F8F869684A780E
:2002C000087800EB0220ADF800008F7804F5EE766FB953206946F4F75BF905F128014A2076
:2002E000F4F756F905F128018A20F7F7A7F806F1200005F11C010B2247F074FABDF80010AD
:20030000384604F097F894F80702800803D36878002105F05BFC002084F80702F8BDC0463C
:20032000200800202DE9FE430646307A02281CBFB14608240DD130880F128DF80A100DF1AC
:2003400008098DF8080004248DF80B7000128DF8090000254FF00108124F307A024605F082
:20036000B1FD08FA05F1084216D0A7F16C01022A19BF01EBC501903101EB85017431684666
:20038000224647F02FFA48466946224647F0EEF9012808BF281C03D06D1C052DDDDBFF2039
:2003A000BDE8FE83941900202DE9D841074606F03EF880468FB3B87A78B397F9091005F09F
:2003C00005F90123064603FA01F05FFA80FC46B1144C226811318B409A432260D94344F847
:2003E000041C00221146B97239723960796007F1100686E806000C49FA6001F1480291F826
:200400004A7013781843107027B191F84A00401E81F84A00604604F011F9404606F0F6F8E2
:20042000BDE8D8810C100440403300202DE9B8411848194C0578606880478046174800784E
:2004400018BB1749DFF85CC0012D0AD00F78012037F07F0713D161460F7837F07F070ED17B
:200460000CE00F78012037F07F0708D10E490F782FB961460F7837F07F0700D1002080F060
:200480000100C0B208B105F071F8A16840468847BDE8B8818B0C00208C1A00204A36002079
:2004A000493600204D3600204B36002070B504461D480078012802D00120F2F7FBFF194DA8
:2004C000281D006880471349064620460B46283105F008F920B903F12C01204605F002F9AA
:2004E000986BA04212D10C4C94F9000010F1020F0AD00B48094B006894F90010826B18684A
:2005000090476FF00100207001F0C2FFA9683046884770BD20080020ED1E0020581D0020D7
:20052000481900208C1A0020CD1F00202DE9F8438146EFF31188202080F311880124164E00
:20054000164DF461164F6C60F86A016A14208847D9F81000810C14BF000C0420A8613868C8
:2005600002682321002090470E480068C6F8804200280CBF211C03210B4807680FB141F091
:200580000401286820F4E02040EA01402860346088F31188BDE8F883000024430020094027
:2005A000840100108C8901009089010070B51B4C05461022ADF1200D04F171016846FEF798
:2005C000A7FC0026049509208DF8146004F10D018DF8160001258DF815500A680DF1170062
:2005E00002604A684260097A01720D496A46182045F0FAFD0B4918208922631D45F0F4FD08
:200600007120314605F036FDD520214605F032FD5D20294605F01AFA08B070BD408501008A
:20062000959200003D7400002DE9F041054605F0FEFE194C0126804605F19C00A67005F070
:20064000ECFE164FB7F91400B7F9161088420ED1207802280BD01248007840B1404605F02D
:20066000D5FF0720FFF792F905F0E1FE8046B7F91400B7F91610884218BF85F8C26006D1B3
:2006800005F1780005F0C9FE082003F0D7FF404605F0BCFFBDE8F08140360020C435002044
:2006A000C433002038B518481849007818B90846007828B906E00846007830F07F0001D069
:2006C00005F08FFE14490C4660688047104D2146124CEA780C3C23789A4206D10D4A8968F8
:2006E0001278D20802D288470AE08968884704F03DFF2078FCF792FE012804BF2078E87022
:2007000005F07CFA012038BD1C0B00204D360020141F00204A3600208C1A0020581D002020
:200720001D4938B5283991F8EC3201EBE30595F8AD42012203F0070302FA03F383F0FF0387
:20074000234085F8AD3291F8AA3201F52A70032B18D091F8F032012B10D0022B08D0B1F86A
:20076000E6128A409102A1EB821101F570710EE0B1F8E6229101A1EB820108E0B1F8E61265
:200780008A4001E091F81D249102A1EB82111C3005F0D0F838BDC04648080020DFF870C0B7
:2007A00098B5FF209CF85F119CF883708CF85C01012914D09CF8F5039CF81414884223D04E
:2007C00014480024047004F0D1FE01F0ABF90F480078012818D02046F2F76CFE98BD0021BE
:2007E0008CF85F1187B19CF82B148DF803009CF83A748DF800109CF83B148DF80170684614
:200800008DF8021005F09BFD98BDC046CD1F0020200800204A36002098B504462078E0282E
:200820002CD105F0C7FE19490F7908610846817801290AD04FB990F85A10012905D190F8E1
:200840005C0001281AD001200CE0114AB2F86E10491CA2F86E1047B97F1CF9B20171002341
:200860008370022005F07EFB08E0002003F0E2FF032005F077FB052000F0F2FF02480168D6
:2008800009B12046884798BD641A0020E01900205C1800201A4898B5007802282CD006284E
:2008A00028D0052805D0012827D9C11E012926D823E0144C94F86B04012820D105F06EF93A
:2008C0002146002809DD114A0F4B12781B689200B3FBF2F2801A48BF00204F7847B191F8B4
:2008E000F5130F2904D018B91C20FEF7BFFF98BD052002E0062000E00220F1F785F998BDE5
:200900000E1E00202008002048140020301E00201A4970B50A684BF2F5214843040AC2F3BE
:200920008140012813D14FF08056D6F8E011D6F8EC018D6800688047A847D6F8E011C96857
:2009400088472111C01000B2484304EBE0340D4901F1E500007830B90948006820F07F4070
:200960002418640802E0002081F8E50006480460210C41600126866070BDC046B44F00505C
:20098000102009403C1500207C600C40002213460A46194671B510F0030F0BD0002A82BF9D
:2009A00000F8011BB2F1010210F0030FF6D1002A08BF71BD11F0FF0141EA0121042A18D31E
:2009C00041EA0141082A0FD30E46102A08D30C460D46B2F10F0312F00F0272C0103BFCD86F
:2009E00012F0080F18BF42C012F0040F18BF40F8041B12F0020F18BF20F8021B12F0010F91
:200A000018BF017071BD704770B51B4E96F8F5030F2828D096F85C11FF2924D096F85E0162
:200A200070B102290CD103F0F7FB05461348D6F8544196F8EC330178083113FB01F00FE052
:200A400003F0EAFBD6F85851B6F8804096F814342D1A06EB43062D1BB6F8244101F02AF913
:200A60002D1B2D1A01D5002070BD4FF6FF70A842C8BFA8B270BDC04620080020151F002076
:200A8000F8B51C49194BDFF868C00C310C6893F86B1401290BD1614693F869740A78002F60
:200AA0000CBF2169616902EB8202521800E0226914790021032501E0491CC9B28C42D8BFD5
:200AC0004FF6FF7010DD136811FB05F69B1993F90070B842F0D1B3F801106046C01D0180C8
:200AE00010688019B0F80100F8BDC046200800204D1D00203819002070B5174817490078E2
:200B000018B90846007828B906E00846007830F07F0001D005F065FC114C60688047124E9F
:200B2000104DF1782A78914207D1104AA1681278D20803D28847012070BDA168884704F01D
:200B400015FD2878FCF76AFC012804BF2878F07005F054F870BDC0461C0B00204D36002040
:200B60008C1A00204C1D0020141F00204A36002038B51C4C002084F8610194F8F55394F880
:200B80003802401CC0B2042884F8380224D0202003F03CF994F837240F2A0AD094F8620126
:200BA00094F8F513814204DD154684F8F50303F0B9FE04EB4501B1F8245194F8F53394F8F1
:200BC00038124FF4707204F502709A40491C01FB152104F05FFB38BD03F046FCFDF786FBDD
:200BE00038BDC0462008002000B500212022ADF1240D6846FFF7CEFE1848B0F84010ADF85E
:200C0000181090F842108DF80B10B0F84400ADF80E0002218DF8161009208DF80C000121E9
:200C20008DF80D108DF81F1000208DF808008DF81B006A468DF81A0006498DF81D00182099
:200C400045F0D2FA0449B1F85400401CA1F8540009B000BD076301005C180020E019002072
:200C60002DE9F84F8346894617467120114604F0AFF881206946F8F74BF84FF0F3080025BE
:200C800007E0B8F1000F23D038686D1CEDB22C3038609DF80000A8421ADD3868066890F8FA
:200CA00004A0002402E0641C0A36E4B2A245E8DD737A002B0CBF052009208145F3D14A463D
:200CC0003046594646F052FD0128ECD14FF000084046BDE8F88F70472DE9F8431A4C0546E2
:200CE0000E46201D01681648007820B9002028603080BDE8F8838847DFF84880D8F804721F
:200D00005FFA80F908F5DC7005F05CFAD8F880214FF47A73410001EBC001B1FBF3F12960C5
:200D20005018B8F8781128608742318003D8C01B2860491C3180A16848468847BDE8F88336
:200D4000D8120020401100208C1A002038B51B4C184A0023164994F8E200136020B301283D
:200D600017D0022807D003281ED151F8350CFFF781F80B2016E051F8355C2846F7F70AFC1B
:200D800040F2FE50A84202D2C01CA842F1D2082008E051F8350CFFF7BBFD07480078002855
:200DA000E7D0052084F8E400F6F750FA38BDC0463D400C403C500C40E28801003C15002048
:200DC000154998B50F7817BB19490A784968930000FB0314114B9700B3FBF7F1814214D3A2
:200DE0000F480068C06B8047211AA1F54871090806D30C4A011B891A090828BF00F5487410
:200E000009482146FAF73EF998BD05F0EAFA07490120087098BDC046CF1F0020FFF6C2FFBC
:200E20004819002000093D00759A00004C360020301E002038B51B4C012094F8F51394F837
:200E40006B5484F861010F2927D06070202005F051F91348012DC4F820020CD094F8F513A0
:200E600094F8385204EB4101B1F82421691C5143490096310CE094F8F51394F8385204EB8F
:200E80004101B1F82421691C5143490001F2A32104F5067004F0FEF938BD03F0E5FA38BDF3
:200EA000710B0100200800202DE9F047DFF86490DFF85CA0DFF86080054600264FF0FF30EC
:200EC000192734462860E0B204F0F8FEB8B1837AABB1017A0126022915D04946DAF800205F
:200EE00040690978D26811FB072103F0EBFC41462B680A68B0FBF2F0834288BF2860641C53
:200F0000032CE0D301E0002028603046BDE8F087FC3400208A330020303600207CB542F2BC
:200F2000050001A901F0BAFE42F20100694601F0B5FE9DF8040030B3134C0098D4F88061B1
:200F400008B39DF80410B14209D8B04201D805F068FA00980021012584F8941104E001252D
:200F60009DF8040084F89451801B642104F5DC764143C4F8BC11304603F002FF304601F02E
:200F800029FD84F898517CBD4011002030B504460D4642F20900ADF12C0D09A901F07EFE67
:200FA0009DF8240008B342F20B000DF10E0101F075FE00230094BDF80E0002930004019069
:200FC000684602F0B9FB044604A942F2030001F065FE04F015F8024604A9B4FBF5F0684306
:200FE000241AE0B201F00EFE06E042F20D0003A901F054FE9DF80C000BB030BDF0B50546D5
:20100000194C2878ADF11C0DE9281CD028BB002694F85A0084F85E6002281ED104AF694663
:20102000384602F023FB5220314604F00FFD2046406920B1026812B1384669469047042004
:2010400000F00EFC09E094F85E00401C84F85E00C0B2032801D102F08FFC9434216809B196
:201060002846884707B0F0BDE0190020144998B50F780FBB1349144B0A789200B3FBF2F359
:20108000834217D34968114F00FB02143868C06B8047211AA1F54871090806D30C4A011B07
:2010A000891A090828BF00F548740B482146F9F7E9FF98BD05F095F906490120087098BD3D
:2010C000CF1F0020301E0020FFF6C2FF4819002000093D004C36002085D200002DE9F041D7
:2010E00007461748174C001D06786068804780461549A268087886281CD1104D05F11E02FB
:201100001088401C10808720087005F0C7F8A16840468847082004F099F8E879B04207D142
:2011200027B90020FEF7A2FBBDE8F0811B20F9E7E920F7E740469047BDE8F0810C1E002048
:20114000643400208C1A00204D3600202DE9FC470C46054646F048FC164F81467868164696
:201160008047804602F0CCFF8246B2002146484646F042FC504604F05FFB02E02D1D241DF1
:20118000ADB23046411ECEB278B128466946042246F012FC68462146042204F08DF800280F
:2011A000ECD00549012048700870B96840468847BDE8FC878C1A0020241F00202DE9F843BC
:2011C0000024002B16460F468046254606D5002FC3F1000302D57F42761E2D259946384642
:2011E000494602F069FC0CA0405CB7FBF9F7002F04F1010408F8010DF1D1A64205DD30210B
:20120000301B401E08F8011DFBD10DB108F8015D4046BDE8F883C0463031323334353637D7
:20122000383961626364656600007047C8B50146184AC87AC8B9B2F84E70906D4FB3801F42
:20124000801DC67826B1B1F81F2083889A4202D07F1EF5D1C8BD8A7FC270CA880280B1F89B
:201260001F208280097B8170C8BDB2F84C70506D7FB121382130867F4EB1B1F81F20B0F8A2
:201280001F309A4203D1212246F0ACFAC8BD7F1EF0D1C8BD40110020012898B528D116488A
:2012A00000680068014601208847012820D003F0A3FD134C012104F1D800017004F0C4FF05
:2012C000800917D20D4800683222B2FBF0F707B90F46083C04F1300005F09FF804F13000C8
:2012E000394605F096F804F1300005F094F801E002F068F8002098BDE00100103036002027
:2013000044150020001F06B480B280B5082802AFADF1080D26DBB0F5005F23DA00F18851B4
:20132000091F0B686A46136049685160BDF80010CA0B10D33A7801F0FF018A420BD17988C4
:20134000BDF80220914206D1B988BDF80420914208BF012007D0BDF80610401A083880B2C9
:201360000828D8DA002002B0BDE8804002B070471FB5014604208DF8000048788DF80100E1
:20138000B1F89A000DF10203ADF80C009031184604F032FB03F0BCFDC0B14FF6FF745320CE
:2013A0000DF10E01ADF80E40F3F7F2F80A4890F8F513A0F808440F2908D00F2180F8F513D3
:2013C00003F00EFF03F050F804F048FC6846FBF753FB00901FBDC04620080020194AF8B5E2
:2013E000044692F8560002EB8000D0F8AC30207800F07F0041005D182070C918497802EBD6
:201400008106D6F8AC7027B182F85610207803EB400529780B1102EB8302D2F8647137B91A
:201420000C280EDA20461821FEF7B4F8F8BD01F00F0157F821700FB904F0D3FF20463C4644
:20144000A047F8BD200800202DE9F843DFF85C90044609EB440000F16805B0F868008846D6
:2014600046F052F9074612480678B7B12A883846002146F0D3F900253C70494664187D7042
:20148000627D381D414646F0ADF93046394646F031F840B92846BDE8F8838DF80040684667
:2014A0001A21FEF777F81A20BDE8F883687A01002008002038B5194C94F8610194F83812F2
:2014C00094F86B5440B9606860B9012084F86101202004F00FFE05E0481CC0B2042884F844
:2014E000380215D0012D07D094F8F5234FF47071914001F2564106E094F8F5234FF47071F7
:20150000914001F2636104F5067004F013FA38BD202002F07BFCFCF7E9FE38BD200800201E
:201520002DE9F843174C04F1780007688046632037B300261D25397D35291CD1404639467A
:20154000324646F045F8787E30F07F0005D194F88300401E84F8830004E094F88200401E79
:2015600084F882007D7057F80C9C3846FEF726FB4F46002002E03E4657F80C7C002FDAD129
:20158000BDE8F8832008002038B5144DD5F8600101680120884701281ED0D5F82401C468D9
:2015A0000F483C2101220023A047002808BF002013D0286880470B480C4A0B4D016893689C
:2015C0001068D160A0EB9000C91A05FB01F3190C814228BF081C1060012038BD8000001067
:2015E00000A00C403020094040420F00F035002070B504F01CFF01461348007802281AD02E
:20160000084605F003F811480068006B8047104A002304F06BFB0F4A12684FF090557A262B
:2016200000232D184FEA020446EB0106ED1846EB0406341C05E004F03DFE0446084604F09B
:20164000E5FF204670BDC046403600208C01001000093D0014360020F8B50D46044604F0EC
:20166000E6FE0646E8B204F029FB8025071C1ED0B87AE0B110480078022806D03846FEF7CC
:2016800093FE00F0BDFC832511E097F909000B494FF4A06202EB002202F47F4220461143C5
:2016A000002202F0E5FF05463846FEF77DFE304604F0ACFF2846F8BD40360020010008041E
:2016C0002DE9F04180461748243007680E46ADF1300DBFB13869A8B1B8F1000F12D08EB169
:2016E00006208DF828000125ADF82A500022ADF82C2002AC00943C690AAB93E803001A2368
:20170000A04708B100200AE002A940460C22FDF7FFFB05A930460E22FDF7FAFB28460CB06B
:20172000BDE8F08158170020F8B50646B1680A687568906B20F4FA6090630968086B20F44F
:201740000070086304F073FE104C0746207820B1022002F021FE00202070384604F056FF8D
:2017600004F065FEA96B11B904F050FFF8BD0021A96304F04BFF696B286BEF686A6B401AE4
:201780002863296B3B4630469847F8BD43360020F8B5844640F6FF741CF8013B002210E084
:2017A000481B401E10F8015B7F1E01F8015BF9D103E01CF8010B01F8010B521C5B08082A3D
:2017C000EADA5808F5D21CF8010B1CF8015B05F00F07FF1CC5F30315122F45EA001508D13A
:2017E0001CF8016B300A24BF1CF8010B60F3DF16BF19AC42D4D1F8BD10B50446002128224A
:20180000ADF1280D6846FFF7C5F8134911226846FDF77EFBFF228DF8182005208DF8120050
:201820008DF8114000218DF815108DF8161009228DF8132001208DF817008DF814000B22F6
:201840000DF11900FFF7A6F8044918206A4644F0CBFC0AB010BDC04657850100C9DB00009F
:20186000B0B5184C054694F85A00A8420FD084F85B00052D84F85A5002D1002002F0F2FFA0
:20188000606920B1C16811B194F85A008847042D18BF032D10D1276904F08CFE0749C01BBC
:2018A000B0FBF1F10648B0F87A208A4204D21FB1A0F87A1000202061B0BDC046A08601003C
:2018C0005C180020E01900202DE9F0410446A56E1F461646884605B1A84704F1600003C863
:2018E00006400F4008BF002E1FD041462046802202F032FA04F1700181E8C00078B104F115
:20190000700191E8600000F1180797E8060000F11803B243A94383E80600A16E41600020BA
:20192000A06604F1400004F096FDBDE8F08170470246F8B5084611464C68203822D0401E22
:201940001DD0401E18BF6FF001001FD18D6804F06EFD0F4E07463068006901462868884770
:20196000B0F1FF3FF7D100256564E564206CA563401EA064384604F049FE2846F8BD002196
:20198000084601E00121002084F82D10F8BDC046D001001010B54FF0FF3004F043FA0446D3
:2019A0000E480F49006881420ED10E480E49002204F043FD0D490220087002F007FD18B9B5
:2019C00001F076FAFCF73CFC0948204204D009484FF0005104F047FD10BDC046143500209F
:2019E0000D2E000054350020D98F00004036002002000040FC33002010B50446012002F052
:201A000005FA208900280CBFEB2000201249607091F80702C20824BF20F0040081F8070200
:201A2000820809D2400813D32B202070EB2363702046FFF7D3FC0BE091F8070200F0FD00C2
:201A400081F80702217C6078C1F3001104F0BEF8204602F023FD10BD2008002030B5174C4B
:201A6000054605F12801ADF1140D04F2FE3046F04FF908B3EF2309208DF801306B688DF897
:201A800000005A781978181D01EB0221ADF802102A890178082A8DF8041014BF94F83A0454
:201AA000C07805F11C018DF805000DF1070004F0A4FC6846FAF7E0FF05B030BD2008002050
:201AC00010B504460320ADF1180D04F128018DF8020000208DF8030001A846F047F96068DD
:201AE000007804F11C018DF80C000DF10D0004F084FC04F1280003F00BFA58B14FF6FF7476
:201B000053206946ADF80040F2F742FD044920460A3108800DF10200FAF7AEFF06B010BDFF
:201B20001E0C002070B5134E706918B106F1140004F0A1FC134C60688047316A0A68002577
:201B4000157109683162A16888470B4A0B49107810B90846007858B1157008460570FBF720
:201B60002BF907480078012802D02846F1F7A2FC70BDC04664340020493600204B36002060
:201B8000CD1F00208C1A002010B5044613480078012808D00B2C04DB1A2CDCBF10480470CD
:201BA0001ADD04F01EFC0F4890F83B0402F090FC41680D4A006804FB01034FF47A74B3FB3A
:201BC000F4F189B204FB1130A2F85E1040037D24B0FBF4F0A2F8600010BDC0468B0C0020A6
:201BE0000E15002020080020C813002038B5124C4FF470000025E0601148A5600068656071
:201C0000C06B80470D49C0F1FF3008600D49C868657008B90C48C8600C480570012001F0C1
:201C2000EBFD30B90F2002F07DFEE068FFF7C8F838BD04F0D6FB38BD301E002008300440A0
:201C4000481900201C1D0020E12301004C36002030B50446606800252062ADF1140DA5659C
:201C60007820A4F84C0094F82C0025650F2807D004F12C0120460122F6F718FE08B116E037
:201C8000284694F83C10FF2901D1A16D21B104F13C012046FBF72AFA48B92B4601208DF85E
:201CA0000C30032101AA00902046F0F737FD05B030BD704770B5134D114968780C88083024
:201CC000444312480068104EC06B80477168401A31788900B0FBF1F10D4802783C2090407E
:201CE000B1FBF0F242436878891A00F10803B1FBF3F25A43891A401A0019083070BDC046A3
:201D0000161E0020141F0020301E002048190020340C002038B5164C04F52A7005461C3054
:201D2000FEF7C4FB02F054F8042003F08FFA94F8AA02032802D194F8A902A0B105F1450117
:201D4000E120F2F725FC05F14601E720F2F720FC94F83B0494F8EF12884204D005F14701FB
:201D6000E820F2F715FC2846FAF786FE38BDC046200800202DE9F8431D4616468946804696
:201D800004F055FB044600F07FFD07462946424648469FB138723A600C487860384600F049
:201DA0009DFDF86006B17E600949086808B93868086000F025F997F9095001E06FF00105D4
:201DC000204604F023FC2846BDE8F8831B640000FC34002038B5044642F208000DF10201B9
:201DE00000F05CFF9DF8020040B19DF8020002281ED1204602F0BEF8054606E042F20C00E1
:201E0000694600F04BFF9DF8005094F8200068B9284600F0CFFE0020A4F87C5094F8223096
:201E200020702BB1102004F075F938BD0120207038BDFEE700B5ADF1240DADF80000ADF856
:201E40000210116801A8016051684160002002460D490690887D8DF80C200D318DF80D00B9
:201E60000B680DF10E0003604B684360097A017218208DF81C2005498DF81D206A4644F047
:201E8000B3F9C0B209B000BD408501001D40000070B5FAF78DFAEFF709F8124D6868804711
:201EA000064603F053FB104C94F92A0404F000F801F092F903F054F803F066F802F090F90B
:201EC000A9683046884794F82B0400F073FE04F211415220F2F75CFB04F0DAF908B9FFF718
:201EE00085FE70BD8C1A00202008002070B50C4620B141680122A240114201D1022070BDBA
:201F00000D4E104B914300254160305D43F82450FF2804D00949096851F8201001E044F0E9
:201F200020410748FAF7D4F920464FF0FF3103F02FFC284670BDC046D8340020AC30002077
:201F4000007FC767C03200201548134A1349E4300078801E0A2807D8DFE800F019140F0678
:201F6000140F06140F0607C0FEE710688008FCD250688008FCD2F5F769B908688008FCD3B2
:201F8000F5F764B908688008FCD2F5F75FB910688008FCD3F5F75AB954600C4058600C409C
:201FA0003C1500203EB5401E4FF000040AD0401E04D0401E1CD1F5F749F919E000F0B8F9FD
:201FC000044615E0684604F0D6F901940B4D8DF800400849029401226B4605F1780001F085
:201FE00023F8054A2C21234605F19C0001F0A4FD20463EBD491F01004D0D01003C15002007
:2020000013481CB5007802281ED001281FD004281DD004F00CFA0446684602F055F800287A
:202020000C480BD0009931B904F0F7F90A48042104F019FA04E003F0ACFE01E004F0EDF950
:20204000204604F0E3FA1CBD192004F0F4F91CBD40360020B4340020FC33002070B5134810
:20206000134D06782868ADF1200DA0B1002445F06FFC0DEB04020021CB00491C20FA03F3B3
:20208000042902F8013BF7DB241DE4B2202CEEDB296868468847022E06D1064991F85001E1
:2020A00040F0040081F8500108B070BD8B0C0020B41F0020C813002010B50446012001F077
:2020C000A5FE1248FEF7F2F9208900280CBFEB2000200F49607091F80702C20824BF00F005
:2020E000FB0081F8070280080BD391F8070200F0FD0081F80702217C6078C1F3001103F0CF
:2021000065FD204602F0CAF910BDC046FC090020200800201449154898B53C2751F8202F00
:202120004C6840F8202F8B684460CC6883600B69C4604C6903618B694461CC6983617F1EB6
:20214000C461EBD1203151F8044B203040F8044B51F8043B40F8043B51F8042B40F8042B00
:202160000968016098BDC046E4690100E07F0021154909681F280ADC1F2819D00D380FD014
:202180000A380FD0001F0FD0C01E0FD01AE0253810D0001F10D0401E10D0801E10D011E080
:2021A000086870474868704788687047C8687047086970474869704788697047C8697047E3
:2021C000086A70470020704780160020F8B50646B08815460F46FDF7FDF80446002D02D432
:2021E000281B0A2806DB3368291B38460BA201F05FFA2418B08978B1002D06D4B06803F085
:2022000093FE291B401D884206DCB368291B384603A201F04DFA24182046F8BD257000C07A
:20222000282725732729000070B5124C6068F8B1124D68688047064694F883200E486168E3
:202240000078904206DCA96830468847F120F6F7D5F870BD04F1780045F098FA002394F821
:202260008300A9686360401C84F883003046884770BDC04620080020081F00208C1A0020DF
:20228000F8B5134C60680D468047124A8446A168B2F84C70506DB7B1002421382130867FC3
:2022A0006EB1B0F81F20954209D1002282774FF6FF72A0F81F20604688472046F8BD7F1E92
:2022C00004F10104EAD1604688474FF6FF70F8BD8C1A002040110020F8B50746C81D01F064
:2022E0000705C610002F4FF0010000FA05F0A0F1010C14BF0029002019D00020BEB17F1ECF
:202300003346024617F8011F941BB4F1FF3F08D10DB10CEA010104E001F1FF04401C214016
:20232000C0B20029F8D15B1E02F10102EAD1F8BD38B5134D95F8E100002410B911480078E1
:2023400060B104F074F895F8E310002906BF012185F8E310012404F059F90CB1002038BDCF
:20236000022002F04FFA0E20FBF74EFA02F014FF01280EBF0120002085F8E20038BDC04602
:202380003C150020E28801004EF68851CEF2000108684FF0F00340EA034008600C488546ED
:2023A0000C4885446F4607208743BD460A486F4607600A48002803D07946491D8E4600475C
:2023C000FCF72AFB03F086FC04F0F0F8FEE7C046003B012000050000BC1F0020F1620100F9
:2023E00070B5124C6068804711490025064648784D70A168820807D2C00814D33046884723
:202400002846F1F757F870BD3046884709480078012802D00120F1F74DF8606880470646B8
:20242000FAF7FAFBA1683046884770BD8C1A0020301E0020CD1F00202DE9F0410546002049
:202440002860114800780E46012802D00120F1F731F80E4C606880473768804630463FB1EE
:202460006A687968914203DC38463F68002FF8D1056030682F60854201D100F009F8A168BB
:2024800040468847BDE8F081CD1F00208C1A0020B0B5144C00252846A26A216BA563904235
:2024A0000CD05268914209DD01F0B6FE0146A06A42689142C8BF4160A063216BE76A37B16A
:2024C00018B142687B689A4201DD3846A06328B14068814202DD01F0CFFAB0BD02F0C8FE69
:2024E000A563B0BD2008002038B501460C684D682068002808BF4FF0FF301FD003F097FF65
:202500002168002954BF491E0021216004F07EF8206890B904F12C0003F087FF04F14800DB
:2025200003F097FF04F1640003F093FF6868FBF741F804F1180002F0C9FF002038BDFEE778
:2025400038B5134C054694F8201094F8230081421DDD94F82110A94219DD636A3BB12946F6
:2025600004F5BA72984794F8230094F8211084F8220010FB0151E06901EB81010918087898
:2025800084F82300D1F8011004F5BA70884738BD40110020C8B5064611484768FFB1416840
:2025A00091F82F1049091AD30768C7B1016891F82F10490913D201684268C968D268914274
:2025C0000DD1371C06D07F1E09D14168C16000274760C8BD03484FF4004103F044FFC8BDD6
:2025E000C4350020FC330020B0B5134C6068628808B325880021AA42C8BF01210B46AA42A2
:20260000C6BFA91A01F58061A91A8FB297B1012B04D0121902F108013A4609E01119C2F5DE
:202620008062083103F079FE606804F108012A4603F073FE6580B0BD380D0020B0B5054614
:2026400010480768C7B1B968087B012400F00F00022818BF002011D1F8680B4AC368127806
:202660008868192712FB073102F02CF9074928600968B0FBF1F001E00020044628602046C0
:20268000B0BDC046C43500208A33002030360020084608B500F0005100F00400084316D0DA
:2026A0000B4800680068014601208847012808D0084800683221B1FBF0F1074803F069FB81
:2026C00008BD064803F0A8FD054803F033FD08BDE001001030360020B43400200D2E000060
:2026E00004360020134910B5044691F80702ADF1180D40F0020081F80702012002F046FFB4
:20270000607890B9211D02A803F076F903F052FA01460120009004F110030193E38902AA63
:202720000520F3F77BFE607010B1002103F04EFA06B010BD20080020F8B506460E48104CAE
:202740000578201D006880470746012D06D10B49087820F00F0040F00100087009480068E9
:20276000094D8369286832464FF0FF319847A16838468847F8BDC0468B0C00203D14002088
:202780008C1A002048190020581D00201048F8B5066810480068104CC06B80476168401AB9
:2027A00021788900B0FBF1F0B0420ED20B4D243D686880470746A6603046FEF757FCFAF747
:2027C0002BFAA96838468847F8BD03F00AFEF8BD5008002048190020301E0020B01A0020C0
:2027E000C8B5071C23D079684878C61121D03A89F96400204B78C3F3C3030F2B08D00B78C9
:20280000C018C918801C891C80B28242F2DC01E0801C80B2824208DB79683E890918796002
:20282000311A3981A7F85000C8BD0020FAE703F0D8FDC8BD10B5044600211C22ADF1200D98
:202840006846FEF7A7F860788DF80000A0788DF80100E0788DF8020020791122611D8DF88D
:20286000030001A8FCF754FBA07D8DF8150008B1A06906900348006881696846884708B089
:2028800010BDC046E01E00202DE9F041DFF8488098F848600025012404FA05F31E4215D0A4
:2028A000E8B203F00BFA88B1877A7FB998F84A1098F84820457283F0FF038472491C88F82B
:2028C0004A10134088F84830BDE8F0816D1C032DE2D30020BDE8F0814033002010B5027AC5
:2028E000012A17D0022A18BF00201DD190F909300E484FF4A06221F470614FF6FC7402EBD0
:20290000032202F470620A4342F4005204EA0201084310BD0A2490F90930416100F1100257
:2029200004825B1D1046937010BDC04601000306F8B504460D4608461122002144F06EFFD6
:2029400094F800C0BCF1000F1AD0641C00214FF0010EE078A37843EA0023207809E0C6107C
:20296000AF5D00F00702401C0EFA02F2C0B23A43AA558342F3DA491C241DC9B28C45E8DCC4
:20298000F8BD80B502465378107840EA0320C7130F7007BFC0F3062300F0FF00C0F3C323E2
:2029A000C0F30A004B70802848800DDA02280BDB012B0CD0022B0AD0042B08D0052B06D01C
:2029C000062B04D0072B02D00022104600E0921C4A6080BD2DE9B841114C0546201D0068A5
:2029E0008047804602F012FD6F7E0146002F08BF686806D068682A69AF68401A8018C01934
:202A000068602961E96805F1140201F091FC012768686F76A168A86040468847BDE8B88168
:202A20008C1A0020114810B50078F0B1104C233C94F82A12642011FB00F0C4F8A00104F540
:202A4000CE70FFF7C7FFB4F8760194F82A22D4F87C11401C80B28918A4F8760100B900210C
:202A60000020C4F87C11FFF76BFD10BD310C00206311002038B504460F4910481430098815
:202A80000068A14213DD0E4D6868804703466946722002F09DF90099E00000EB041009185E
:202AA0000091A968184688470098001D38BD641AA1B200EBC10038BD0C1F0020401100206F
:202AC0008C1A0020042810B51AD10E4C204603F0D9FAA8B1204603F09AFC0B490968484336
:202AE000B0F5967F0CD2204603F097FC052001F089FE0649012008700548042103F0B3FCB9
:202B0000002010BDB43400203036002011350020FC33002010B5114C22685168496839B185
:202B200010B1F1F77AFA226850684068804722685168886808B9C86878B103F0E1F9216824
:202B40004868806808B1804721684868C06800B180470348503802F0E9FA10BDFC340020BF
:202B60005100070610B50446012001F04FF92078212804BFEB2060700D4991F80702C2085D
:202B800024BF20F0040081F80702800805D22B2020702046FEF722FC10BD91F8070200F0BA
:202BA000FD0081F807026078002103F00FF810BD20080020F8B5104C0646201D0568802EE1
:202BC00001DD03F00EFCA8470C4D0D49094A2F780E701FB91778A1682FB907E01778A1682D
:202BE00037F07F0702D088470120F8BD8847FDF783FFF8BD4D3600208C1A00201C0B002007
:202C00004C1D0020F8B5174604468C4600221046D7B10146DAB91CF8015B082685F0010314
:202C200003F00103C918C9B24B1EA34208D0401C761E4FEA6505C0B2F0D18742EADC03E0E3
:202C400087424FF00102E5DC0AB903F0EAFBF8BD0146104810B500784FF4C854802803DD95
:202C60008428B8BF4FF41644052909D001F030FC0949C07B0988022814BF04F57A740C441E
:202C800004F57A644FF47A6004F5FA64B4FBF0F010BDC0465B0C002036130020F8B50E4696
:202CA00002F03DFD05464FF6FF70A84208BF682013D00C4C606880470849094A074668008D
:202CC00000EBC5004018017889184278304644F089FDA168384688470020F8BD4C820100EE
:202CE0003C1300208C1A002080B502F027FD01460F4802680429C2F340674FF0FF3016D16E
:202D0000C2F30331083911D0491E0AD0891F0ED1100E04D3900E2CBF0E200D2080BD0B209F
:202D200080BD002F14BF0A20092080BD0C2080BD94120050F8B516460C46054603F077FB5A
:202D40002B461F6884460022214630460A6027B9196008B1012101700CE008B11446047030
:202D600000E03F6838680028FBD1B94208BF141C01D039600124604603F048FC2046F8BDBF
:202D8000104898B501210170022111400E4A4FF0E0471F4008BF002903D092F90010491EA5
:202DA0001170044692F9000028B192F90000002804DC03F016FB0020F0F77CFB002020701F
:202DC00098BDC046CD1F0020F61E002070B501200E4E0F4D30702878022814D100240221C4
:202DE00014EA030001EA020108BF002901D103F0F8FA084991F90000401E08702C7002F0FE
:202E000021FF347070BD03F0ECFA70BDCD1F0020CF1F0020F61E002038B50F49104C888BB9
:202E2000401C88836068804705460C480178862903D0A1682846884738BD8721017003F0BB
:202E40002DFAA16828468847082002F0FFF9E920FCF70CFD38BDC0460C1E00204D36002006
:202E60008C1A002080B507468020EFB1B97A01291AD197F909000D4A0121113001FA00F044
:202E8000C34342F8043C13681843106097F909008140C8B202F078FDF868002101F056FE6B
:202EA000812804BF0221B97280BDC0460C100440F8B5104E00241125E0B202F0FFFE071CAC
:202EC00014D0B87A012811D13846FFF7CBFF81280CD097F9090096F8491005FA00F0084354
:202EE00086F849000448002103F0BDFA641C032CE2D3F8BD4033002030340020F8B50646CB
:202F00000F4D104F7388002417E0A20002EBC402921951689068D26852B9AF420BD00A789C
:202F200055F822200346491C08461946904701E0FBF7EEFF7388641CA4B2A342E5DCF8BDE4
:202F4000D88D0100E48D010070B544680D4604F5827003F062FA0D4A667F207F0C49A369FF
:202F600012688019C01D80B204F5827445436943B1FBF3F010186330B0FBF2F1491C204669
:202F800003F047FA204603F046FA70BD3036002040420F003EB5054615F8060C03281DD1AA
:202FA0002B681869009058690190986902906C6859689A681868DB68A0472968086015F841
:202FC000080C44F073FB0446012044F09DFB011C04D042200870204644F08CFA3EBD704767
:202FE0002DE9F04117468846064602F09DFF0D4C0546002128222046FDF7CCFC31462A466D
:203000002046FBF785FF40463A46611944F0CAFD204602F00DFD02A002F00AFDBDE8F08146
:203020000D0A00C08C340020F0B515460E4604461F1CADF1240D08BF002308D068460021A0
:203040002422082303F0AEFAB8686B460690204631462A4603F0A2FA0348044902682046B9
:2030600009B00A60F0BDC0469C8901003036002000B500211A22ADF11C0D6846FDF78AFCCD
:2030800002200B4A8DF81400B2F84410ADF80C10B2F840108DF818000020ADF81610054991
:2030A0008DF8190018206A4643F09EF807B000BDE0190020116301000E49086820F00200E6
:2030C00040F4087008600C48032140F8041C41F230018160012101605022826001604FF44C
:2030E000CA62826001604FF4865282600160034801607047000004605860044000410440BB
:2031000038B50E4B1B680D461446AB4204D30C4951F82510884201D0022038BD03F087F97D
:20312000084B103B1A68AC400121A9408A4314431C6003F06BFA002038BDC0463C1F0020EA
:20314000C0320020E02002401049D0B50F68ADF1180DCFB17E69BEB1B0B106218DF8101000
:203160000226ADF812600024ADF814404388ADF8003042680192816802917C6904AE96E885
:2031800003000C226B46A04706B0D0BD7C17002070B5104D95F8F503B5F81A440F280FD048
:2031A000D5F8586101F038F80019864208D895F8F5134FF4707088402418A41B04F570744F
:2031C00005F5EE752846FDF771F92146284602F0B1FB70BD20080020104898B5877890F8B2
:2031E0006B44002F14BF802100210A4BB3F85C004FF67F72022C02EA000241EA020140EA56
:203200000100A3F85C0004D10349087867F3C710087098BD28190020181500202008002021
:2032200038B5EB2002F0F5FB0D48002404700A480078862802D12046FFF7EEFD074D686811
:20324000804708490A6A13681C7112680A62A968884702F0A7FB38BD4D3600208C1A002022
:203260004B360020643400201FB5144600900A79487940EA02208A7942EA0022C87940EAEB
:20328000022001900A78487840EA02208A7842EA0022C87840EA02200290684600F04CFA9B
:2032A000B0FBF4F16143401AC0B200901FBDF8B5051C0E4606AF04D0012D0CBF06240024B0
:2032C00000E002240EB9A41CA4B2012A06D0022A0ED15889C01D04EBE00408E038780028AE
:2032E00014BF022101210020FBF758F92418A4B22046F8BD70B50D46044603F098F8666893
:20330000A1682B468E4204D103F080F94FF0FF3070BDE1682568491CB1FBF6F27243891A60
:203320004B55A2686369E160521CA260934238BF626103F06BF9A06870BD70470F4800B588
:203340000068ADF1240D69467030F4F78BFF10B99DF80B0008B900200DE0684601F063FE3B
:203360009DF808104FF47A73B0FBF1F24A43801A091A03FB01F009B000BDC04624080020E1
:20338000F8B502F091F90D460746FF2F08BFF42011D0094C60688047084A0646B800084BED
:2033A000115C80184278C918284644F01BFAA168304688470020F8BD8C1A00208C7D0100C3
:2033C000080C002038B50D4DD5F860014268002101209047D5F8600101680120884708B141
:2033E000286880470648074CD5F86C310068083C606018688047206138BDC04680000010AC
:2034000030200940F83500202DE9F84303F029F8DFF830900C4D00240126804606FA04F06C
:2034200018EA000F06D059F8240018B107680FB12146B8472868641CE4B28442EED9BDE8FA
:20344000F883C046C03200203C1F0020B0B502F0EEFF05460B48017801290FD00A4902465F
:2034600001230878137048B1084C0746206880680146204688470C347F1EF7D1284603F099
:20348000C5F8B0BDCC1F002023890100048901002DE9F0410D4C201D00688047064600F074
:2034A0002FFE8046002044F09FFA094D686002F061F90746404602F0BFF917B10120687084
:2034C0002870A16830468847BDE8F0818C1A0020241F00200F48B0B507680025ADF1180DB4
:2034E000ADF8105097B106208DF808000223ADF80A30ADF80C5004AC00943C6902AA92E8B8
:2035000003002A46A04708B1ADF81050BDF8100006B0B0BD7C17002010B50F4C94F8070243
:20352000ADF1180DA8B940F0010084F80702012002F02CF802A801F0FFFC0120009004F53A
:20354000FE730193B4F80E34032102AA0520F2F765FF06B010BDC0462008002038B55478AC
:20356000057A0023C4F38104A54217D1022C07D0032C13D1521D114644F0E0FB03460DE07B
:2035800095795479008804EB0524844206D11479D07800EB0420884208BF0123184638BD27
:2035A00010B50446012000F031FC2078212804BFEB2060700A4991F80702C20824BF20F09D
:2035C000040081F80702800809D391F8070200F0FD0081F807026078002102F0F7FA10BD57
:2035E00020080020F8B5071C17D00D4C201D006880473E68054666B10A49091F0A6DA6F176
:203600000C00964204BF00220A650021396044F06DF9A16828468847F8BD02F0E2FEF8BD9C
:203620008C1A00202408002038B50F4C0546204602F064FEB0B9204602F003FF0446A06816
:2036400005420AD0E06822690021034628469847002818BF4FF0FF3005D1204602F0F3FE33
:20366000041CECD1002038BD3C15002038B50F4B05460C46281D03F1500144F008FBB3F897
:2036800040002880B3F84E0003F146016880201D44F0FDFA93F84200207300206073B3F8C0
:2036A00040002080B3F84400608038BDE01900200CB4F0B505AF061C0C4627F00303ADF105
:2036C000040D03F1040304D03068002818BF051C00D100253A68284602F06CFD844238BF34
:2036E000601E15B131680918316001B0BDE8F04002B0704708B50B4602F02CFA5989418182
:2037000099898181997B8173D97BC173197C002201B10122597C417459694161197E02746E
:20372000002201B10122027603F119010B221930FBF7EEFB08BD0000416882680D4B0068A3
:20374000C91AD21AC01A4A40A2EBB1425040A0EB72504140A1EBF0114A40A2EB31425040B1
:20376000A0EB32704140A1EBB04181EA0200A0EB31207047054152210C497CB5044608226B
:20378000684644F02FF80A4D0A486E8B0088A0420BDC241A6869A1B2082200EBC100694646
:2037A00001F08AFD761EB0B268837CBDC0810100401100200C1F0020F8B50D4D0446686858
:2037C00080470C4FC6B207F5CE7002F0FBFC410001EBC0014FF47A70B1FBF0F1D7F87C0138
:2037E00021604018A968206030468847F8BDC0468C1A00204011002010B5ADF1180D0C4C48
:2038000001900A4808210390002004902069ADF800101B2102900748ADF80210016868462C
:2038200088470299216106B010BDC046294C0100301E0020B01A002010B5ADF1180D0D4C64
:2038400001900A4808210A3C039000200490E068ADF800101B2102900548ADF80210016897
:20386000684688470298E06006B010BD57630100B01A0020161E00201CB50E4C0020042204
:2038800060706946207044F097F80098B0F5801F0CD020B901F070F9F5F756FE08E0FFF74D
:2038A000F7FD02F055FB0420608001E001F064F960781CBD241F002070B502F0B8FD064673
:2038C0000C48E030007850B108480068C0680546074800243C2101222346A84700B10124BF
:2038E000304602F093FE204670BDC046A401001000A00C403C150020B0B502F098FD0546ED
:20390000FDF742FE0A4C0B49A0680023E03102460B700220904707461020FFF785FE1FB10B
:20392000A068014603208847284602F06FFEB0BDD48801003C150020B0B50D46044602F04A
:2039400076FDA768294697B1226923689A5C0A7021696568A268491C521EB1FBF5F3A260DC
:203960006B43C91A216102F051FEA068B0BD02F04DFE4FF0FF30B0BD10B5002000F05AFF38
:203980005220012102F062F802F014FE094C08492061B1F86E00401CA1F86E00032002F08D
:2039A000E1FA0520FDF75CFF002084F85E0010BD5C180020E019002010B50446012000F024
:2039C00025FAEB200B49607091F80702C20824BF20F0040081F80702800809D391F80702CE
:2039E00000F0FD0081F807026078002102F0EEF810BDC046200800200D48B0B503680D48F2
:203A000002780021382411FB043090F8267037B990F82550491CAA42C9B2F4D103E090F868
:203A20002510914203D1834201D000F00DFAB0BD441900205B0C002070B504460E46104693
:203A400002F040FA0B4B0A4D012E07D00121022A01FA04F120EA010008D006E00121022A32
:203A600001FA04F141EA000000D02B46186070BDB0190020941900200C48F8B500680C4DCD
:203A80004668A868B0420DD90A4C606880470746EE603046FDF794F9F9F7BEF8A1683846EC
:203AA0008847F8BD02F09DFCF8BDC04658080020301E00208C1A00201CB50A1C17D0002387
:203AC0000124E407A04238BF041C944201D95200FBE790425B41904228BF801A914201D292
:203AE0005208F6E7191C021C081C111C1CBD00B1C843FDF79AFB1CBD00B500211822ADF146
:203B00001C0D6846FCF746FF0949B1F840006A46ADF80A0002208DF80800B1F84400054912
:203B2000ADF80000182042F05FFB07B000BDC046E019002037630100F0B514460D46064650
:203B40001F1CADF1340D08BF00230DD0684600213022082302F01EFD7B6808933868059078
:203B60003A7AADF818206B4630462946224600F0E3F90DB0F0BD00000D4910B5097804469A
:203B8000A1B1617871B9217839B194F8201021B9FEF720F90020207010BD94F87C00FFF72E
:203BA00009F810BDFBF74EFA0020607010BDC046310C002000B5ADF1140D8DF808000A4A88
:203BC000039112788DF804200823ADF800300748ADF80230243018220168ADF80620684688
:203BE000884705B000BDC046D81E00208C1A00200D4908B5D1F878020B68020F03F0FF03D3
:203C00007F2B88BF002301F099FD4FF0FF31042808D11046012804D9801E04BF0B3359B28F
:203C200000E00A21084608BDA010005098B50D4C2778002F18BF012013D16188C1F5005126
:203C400089B2884200DC58B902F07CFA00206070F5F77AFC20B9607800280CBF0127071CC9
:203C6000384698BD241F002084460B4880B5174602688A42604604D3084A52F821209042FD
:203C800001D0022080BD002307B10123044A0020E03A535480BDC0463C1F0020C0320020F6
:203CA000E0200240B0B50C460546171CADF1280D08BF00220ED0684600212822082302F0BD
:203CC00065FCFA680792386804907B680593B96806916A462846214601F080FE0AB0B0BD06
:203CE000F8B50646756802F0A2FB0B4C0746207820B1022000F050FB00202070384602F0D5
:203D000085FC696B286BEB686A6B401A2863296B30469847F8BDC0464336002002460A48D7
:203D200080B5077800206FB1084B1B78934209DD884208BF0649074B0C2012FB00300268E9
:203D4000D268904780BDC046CC1F0020238901001C88010004890100B0B517460C4A0B46BB
:203D600004460825303A3032B2F92C0083420BD12046114602F0AEF930B11FB192F82F00C8
:203D8000074201D01046B0BD6D1EECD10020B0BD082D002038B501460B4CCB8AE26860682A
:203DA000DB080ED204F1780043F0F0FC074D6868804794F88310491C84F88310A968884756
:203DC00038BD904738BDC046200800208C1A0020094A0021117009490948098890F86B34BE
:203DE000A0F80E140748022B00F15A00018002D1054824300180704764340020561D0020CA
:203E000020080020381900200E15002038B50B4C0546606880470A4B1A7885F0FF010A40E2
:203E2000A1681A708847FCF701FB06480078012802D00020EFF73EFB38BDC0468C1A002070
:203E40004A360020CD1F002080B5A0B10A494268C861476B4A6242684F6383680B62C76AC7
:203E6000036BCA620B631FB114310F60034A1160C0680349086080BD28190020B01F00208F
:203E80006008002010B50D4C94F8F503ADF1B00D0F280AD104F5EE70FCF708FBB4F81A1464
:203EA00004F5EE7001F046FD05E02F208DF800006846FDF793FA2CB010BDC0462008002098
:203EC0000C490D4880B5402751F8202F40F8202F4B6843608B688360CB68C3600B69036123
:203EE0004B6943618B698361CB697F1EC361EBD180BDC04674710100E0BF002198B50C4659
:203F000002F090F9002700B101270A4A9069211AB1F1004F08D8011B891DC90F05D1801DC0
:203F2000A04288BF041C00E0841D14600FB902F07FF998BD18200940F8B507460A480B4C98
:203F40000668E0698D00285886420AD108480090384602F017FBE0692858864218BF381CDC
:203F600000D10020F8BDC0464C80010018170020701E002010B50446E220ADF1200D05A941
:203F8000FFF7FEF9608894F8262005A9FFF76CF90446694642F20200FEF780FE01F030F8B6
:203FA000024669462046FEF72DFE08B010BD00000C4870B500F12301097803290BD0084C95
:203FC000606880470646FDF7ABFAA168054630468847284670BD012180F89711002070BDAA
:203FE0008C1A00204011002030B5054608200C46ADF1140DADF800000020ADF8020018217C
:2040000002900648ADF804100168684688479DF80C0028700498206005B030BDB01A002040
:204020001FB58DF800000A48006868B144695CB1084902A80A688988026002AB818093E891
:20404000030001226B46A04701F00AFF00901FBD7C1700207889010003B490B503AF396838
:20406000ADF10C0D68460160B98881809DE803001C4600F011FF28B1B968224643F09CFC21
:20408000002000E0012003B0BDE8904002B070470C4810B5437802788B4205D083788B42B6
:2040A00005D142F0100201E042F0080202703030044643F01DFE012802D0204643F024FEA9
:2040C00010BDC046141B00203EB50546002028606846FEF7B3FA044601A8FCF7E5FE012C92
:2040E00002D0012805D008E028B10199009A914201D8019900E0009929602043C0B23EBDE3
:20410000B0B54FF0805000F5EC74D0F8D801094D816828468847C7B257B1206842680021E5
:204120002846904720688168284688470028F9D13846B0BD0040034038B505460B4C2878FD
:2041400038B9002000F076FB0020A11C0870FDF787FB606920B1826812B12978A81C90479F
:20416000216F09B12846884738BDC046E019002038B505460120FFF749FE0A4C04F5EE7061
:20418000FCF794F904F5F670FCF790F9002084F8040284F8070268784FF6FF7100F04AF9D5
:2041A00038BDC046200800200C4838B50078012802D00120EFF77EF9064C6068804705465E
:2041C000F8F72AFDA1682846884703480068804738BDC0468C1A0020840B0020CD1F00208D
:2041E0000A4838B500F22C4190F86B44084808220D463F3043F0F6FA022C05D105482946CB
:2042000008220A3843F0EEFA38BDC04620080020481900203215002070B50A4C60688047E2
:2042200006460A480068084DC06B80476968401A29788900B0FBF1F5A1683046884728468F
:2042400070BDC0468C1A0020301E002048190020F8B50C4E446885680F4608E0216B087095
:20426000606B216B7F1E401C6063491C21633FB130680069014628688847B0F1FF3FEDD10E
:204280003846F8BDD00100102DE9B0430F46044601F072FE04F1280292E800034B4642464C
:2042A000F2F7E2FD05460B462A464046494601F01DFD17B1303484E803002846BDE8B08329
:2042C000F8B5446885680F1C11D00A4E3068216A826909782868904748B1216A606A7F1E53
:2042E00001F10101216200F101006062EED13846F8BDC046D001001080B5024653781078EA
:2043000040EA0320C7130F70C0F3C3234B70C0F30A00488005D0042B03D1802801DA022899
:2043200002DA0022104600E0921C4A6080BD000010B51446ADF1180D019000200490206805
:204340000391082202900648ADF800201B220168ADF80220684688470298206006B010BD73
:20436000B01A00200A4B10B51B6802F0FF04A34206D3084C02F0FF0354F82330984201D071
:20438000022010BD08461146F7F7A2FF002010BD3C1F0020C032002010B5044602F047F840
:2043A000094B083B1A1992F8E810491EC9B282F8E81021B99A680121A1408A439A6002F0C5
:2043C00025F9002010BDC046441500200B4801688A6800E00246506818B101F1280383421A
:2043E000F8D1507B10F00F0006D1488D40F60901814208BF012000D000207047FC3400208C
:2044000098B50146886840F603022027531C02E040687F1EFFB260B15FB10488A24218BFE7
:20442000A342F5D1C9681CC828311CC189C881E8890098BD00B50222ADF1140D8DF80100D0
:204440008DF8002008B14FF6FF71ADF8021005490B2201A8203143F0C5F96846F8F70CFB88
:2044600005B000BDFC0900200A4810B5007810B1022001F08BF82020FFF7C8FC064C04F57A
:204480000670FCF713F804F50270FCF70FF8FDF7ADFB10BD310C00202008002010B5044626
:2044A0000A48007840B1207CC00805D3B4F8421004F12800FAF7A0FBA07B0428ACBF0D207F
:2044C000122020702046F8F7D7FA10BD8A0C002010B5041C05D0042C0BDB802C01DB882C65
:2044E00001DB01F07EFF054800EB0410A0F5936010BD034800EB041010BDC046200800206C
:20450000047B010038B50B4C94F8F5030F280DD094F8140468B104F50A752846FBF7C6FFE5
:20452000B4F81A14284601F005FA38BD1020FFF76DFC38BD2008002010B5A1B10A4A0024F3
:204540001E3A13684A688B4202444A6002D1002A48BF4C604A68002A03D409680029F1D15A
:2045600010BD01F03EFF10BD760800201FB50B4A546863682189206A00910190C01A091AD2
:2045800088B2029002F22C400390606AA16A94F88C201530F7F76EFB00901FBD20080020FF
:2045A0000B4908B58A784889062A0CD14A7A022802F101024A7206DB401E80B2488106200A
:2045C000EDF722FB08BD00F045FBF9F7E5FE08BD0C1E002098B50B4C94F8FC0288B1D4F8D0
:2045E000187362686FB1D06D28B102210023B8476268D4F81873106E18B13C4608210023B5
:20460000A04798BD20080020F8B50B4E456884680F4606E005F13C02C1B21046FEF76AFEE2
:204620007F1E3FB130680069014620688847B0F1FF3FEFD1F8BDC046D001001038B50446DC
:2046400001F0F5FE084A1178054684F0FF00014011701078000903D20448082101F003FF4D
:20466000284601F0D3FF38BDF8340020FC330020F8B515460C46064601F0D9FE074608486E
:2046800000683246904205D12046294600F05EFA044600E00324384601F0B8FF2046F8BDE3
:2046A000FC340020094910B500200A4C08600120C86114342060216844F8280C04480068F6
:2046C000016A14208847206810BDC04600002443B00100101820094038B5B1F1FF3F044651
:2046E00008BF05212020EFF3118580F311880120054B61618840A061586901F03FFFA0621B
:2047000085F3118838BDC046AC16002080B502465378107840EA0320C7134FEAE0130F7009
:20472000DBB24B7000F07F00488002D12A2B00D110B90022104600E0921C4A6080BD38B55E
:2047400004460D4607202070687DA070E87DE070287E1122291D2071601D43F043F8A078A8
:2047600000280CBF81200020A075E86AA06138BD70B5044604F128020CCA0846002101F064
:20478000B5FA04F1300292E860002D1846EB0106290C30040143FFF7B1FB383484E8600065
:2047A00070BD000010B50A4C48B900F04FFE233CC4F8900194F8230048B9022005E00128E7
:2047C00005D12078022802D10320FDF7B9FE10BD631100200A4B93F8A020000601F0FF01A8
:2047E00041EA104103EB4200A0F86010521C90B22028A8BF002083F8A00000207047C0468E
:204800004011002038B5044601F011FE084A02F108031D680121A140A4182943196094F8EB
:20482000E810491C84F8E81001F0F0FE002038BD3C15002070B50A4D044605F198000646A2
:2048400043F056FA012802D1304643F05FFA34B1A869214643F054FA304643F055FA70BDD4
:204860005817002070B50A4D044605F12C00064643F03EFA012802D1304643F047FA34B13F
:20488000E868214643F03CFA304643F03DFA70BD5817002070B50A4D044605F1BC00064698
:2048A00043F026FA012802D1304643F02FFA34B1E869214643F024FA304643F025FA70BDF4
:2048C0005817002038B50C460546FCF791FE2A462146101A800801F57A72824203D26FF0DA
